
IBM(R) Linker for OS/2(R), Version 5.0 
Copyright (C) IBM Corporation 1988, 2003.
Copyright (C) Microsoft Corp. 1988, 1989.
All rights reserved.

Current option settings:
	PDD	CODE:RX	DATA:RWS
	Alignfile:0x00000010	ALIGNAddr:0x00010000	NOBASe
	NOBRowse	NODBgpack	NODEbug:none	NODEFaultlibrarysearch
	EXEPACK:2	NOEXTdictionary	NOFIxed	FReeformat	NOIGnorecase
	Linenumbers	NOLOgo	MAP:bin\Release.ACP\uniaud32.map
	OCache:0x1cbf2800	OLDcpp	NOOPTFunc	PACKCode:0xffffffff
	PACKData:0xffffffff	PMTYPE:VIO	SEGMENTS:256 	NOSEGOrder
	NOSTRictwarnings	NONOSTRictwarnings	NOSTUB	NOVERBose
	VERSION:00.00


ILink : warning LNK4019: device driver can not have a stack

 UNIAUD32

 Start         Length     Name                   Class
 0001:00000000 000000483H DATA16                 DATA16 16-bit
	at offset 00000000 00483H bytes from F:\src\os2\uniaud32\drv32\bin\Release.ACP\startup.obj (startup.asm)

 0002:00000000 000000689H CODE16                 CODE 16-bit
	at offset 00000000 00689H bytes from F:\src\os2\uniaud32\drv32\bin\Release.ACP\startup.obj (startup.asm)

 0003:00000000 000000000H FIRSTCODE32            CODE 32-bit

 0003:00000000 00008D5B6H CODE32                 CODE 32-bit
	at offset 00000000 0047DH bytes from F:\src\os2\uniaud32\drv32\bin\Release.ACP\startup.obj (startup.asm)
	at offset 0000047D 000CCH bytes from F:\src\os2\uniaud32\drv32\bin\Release.ACP\strategy.obj (F:\src\os2\uniaud32\drv32\strategy.c)
	at offset 00000549 00106H bytes from F:\src\os2\uniaud32\drv32\bin\Release.ACP\read.obj (F:\src\os2\uniaud32\drv32\read.cpp)
	at offset 0000064F 00EF4H bytes from F:\src\os2\uniaud32\drv32\bin\Release.ACP\init.obj (F:\src\os2\uniaud32\drv32\init.c)
	at offset 00001543 01F6BH bytes from F:\src\os2\uniaud32\drv32\bin\Release.ACP\parse.obj (F:\src\os2\uniaud32\drv32\parse.c)
	at offset 000034B0 0004EH bytes from F:\src\os2\uniaud32\drv32\bin\Release.ACP\devhlp.obj (devhlp.asm)
	at offset 000034FE 00839H bytes from F:\src\os2\uniaud32\drv32\bin\Release.ACP\idc.obj (F:\src\os2\uniaud32\drv32\idc.c)
	at offset 00003D37 00740H bytes from F:\src\os2\uniaud32\drv32\bin\Release.ACP\dispatch.obj (F:\src\os2\uniaud32\drv32\dispatch.c)
	at offset 00004477 00701H bytes from F:\src\os2\uniaud32\drv32\bin\Release.ACP\rmhelp.obj (F:\src\os2\uniaud32\drv32\rmhelp.cpp)
	at offset 00004B78 000D4H bytes from F:\src\os2\uniaud32\drv32\bin\Release.ACP\irq.obj (F:\src\os2\uniaud32\drv32\irq.cpp)
	at offset 00004C4C 0002DH bytes from F:\src\os2\uniaud32\drv32\bin\Release.ACP\util.obj (F:\src\os2\uniaud32\drv32\util.cpp)
	at offset 00004C79 004E6H bytes from F:\src\os2\uniaud32\lib\Release.ACP\linuxlib.lib (vsprintf.c)
	at offset 0000515F 000FBH bytes from F:\src\os2\uniaud32\lib\Release.ACP\linuxlib.lib (timer.c)
	at offset 0000525A 0004CH bytes from F:\src\os2\uniaud32\lib\Release.ACP\linuxlib.lib (strncmp.c)
	at offset 000052A6 00039H bytes from F:\src\os2\uniaud32\lib\Release.ACP\linuxlib.lib (task.c)
	at offset 000052DF 004E8H bytes from F:\src\os2\uniaud32\lib\Release.ACP\linuxlib.lib (misc.c)
	at offset 000057C7 00362H bytes from F:\src\os2\uniaud32\lib\Release.ACP\linuxlib.lib (ossidc.cpp)
	at offset 00005B29 00643H bytes from F:\src\os2\uniaud32\lib\Release.ACP\linuxlib.lib (soundmidi.c)
	at offset 0000616C 01010H bytes from F:\src\os2\uniaud32\lib\Release.ACP\linuxlib.lib (soundmixer.c)
	at offset 0000717C 0180EH bytes from F:\src\os2\uniaud32\lib\Release.ACP\linuxlib.lib (sound.c)
	at offset 0000898A 0051BH bytes from F:\src\os2\uniaud32\lib\Release.ACP\linuxlib.lib (debug.c)
	at offset 00008EA5 00CB7H bytes from F:\src\os2\uniaud32\lib\Release.ACP\linuxlib.lib (memory.cpp)
	at offset 00009B5C 01083H bytes from F:\src\os2\uniaud32\lib\Release.ACP\linuxlib.lib (ioctl.c)
	at offset 0000ABDF 00268H bytes from F:\src\os2\uniaud32\lib\Release.ACP\linuxlib.lib (irq.c)
	at offset 0000AE47 019A6H bytes from F:\src\os2\uniaud32\lib\Release.ACP\linuxlib.lib (pci.c)
	at offset 0000C7ED 00560H bytes from F:\src\os2\uniaud32\lib\Release.ACP\linuxlib.lib (malloc.cpp)
	at offset 0000CD4D 00025H bytes from F:\src\os2\uniaud32\lib\Release.ACP\linuxlib.lib (strncpy.c)
	at offset 0000CD72 00010H bytes from F:\src\os2\uniaud32\lib\Release.ACP\linuxlib.lib (waitqueue.c)
	at offset 0000CD82 00023H bytes from F:\src\os2\uniaud32\lib\Release.ACP\linuxlib.lib (spinlock.c)
	at offset 0000CDA5 008EAH bytes from F:\src\os2\uniaud32\lib\Release.ACP\core.lib (hwdep.c)
	at offset 0000D68F 024B4H bytes from F:\src\os2\uniaud32\lib\Release.ACP\core.lib (timer.c)
	at offset 0000FB43 01D21H bytes from F:\src\os2\uniaud32\lib\Release.ACP\core.lib (rawmidi.c)
	at offset 00011864 002EEH bytes from F:\src\os2\uniaud32\lib\Release.ACP\core.lib (pcm_misc.c)
	at offset 00011B52 026E0H bytes from F:\src\os2\uniaud32\lib\Release.ACP\core.lib (pcm_lib.c)
	at offset 00014232 00C4FH bytes from F:\src\os2\uniaud32\lib\Release.ACP\core.lib (pcm.c)
	at offset 00014E81 00422H bytes from F:\src\os2\uniaud32\lib\Release.ACP\core.lib (sound.c)
	at offset 000152A3 00CFFH bytes from F:\src\os2\uniaud32\lib\Release.ACP\core.lib (info.c)
	at offset 00015FA2 00386H bytes from F:\src\os2\uniaud32\lib\Release.ACP\core.lib (pcm_memory.c)
	at offset 00016328 0020EH bytes from F:\src\os2\uniaud32\lib\Release.ACP\core.lib (pcm_timer.c)
	at offset 00016536 03901H bytes from F:\src\os2\uniaud32\lib\Release.ACP\core.lib (pcm_native.c)
	at offset 00019E37 0020CH bytes from F:\src\os2\uniaud32\lib\Release.ACP\core.lib (info_oss.c)
	at offset 0001A043 0032DH bytes from F:\src\os2\uniaud32\lib\Release.ACP\core.lib (sound_oss.c)
	at offset 0001A370 00279H bytes from F:\src\os2\uniaud32\lib\Release.ACP\core.lib (device.c)
	at offset 0001A5E9 01ADDH bytes from F:\src\os2\uniaud32\lib\Release.ACP\core.lib (control.c)
	at offset 0001C0C6 003A2H bytes from F:\src\os2\uniaud32\lib\Release.ACP\core.lib (memalloc.c)
	at offset 0001C468 00C56H bytes from F:\src\os2\uniaud32\lib\Release.ACP\core.lib (init.c)
	at offset 0001D0BE 001A1H bytes from F:\src\os2\uniaud32\lib\Release.ACP\core.lib (sgbuf.c)
	at offset 0001D25F 00E4CH bytes from F:\src\os2\uniaud32\lib\Release.ACP\pci.lib (bt87x.c)
	at offset 0001E0AB 00B2CH bytes from F:\src\os2\uniaud32\lib\Release.ACP\pci.lib (als4000.c)
	at offset 0001EBD7 030C9H bytes from F:\src\os2\uniaud32\lib\Release.ACP\pci.lib (cmipci.c)
	at offset 00021CA0 01700H bytes from F:\src\os2\uniaud32\lib\Release.ACP\pci.lib (atiixp.c)
	at offset 000233A0 013FFH bytes from F:\src\os2\uniaud32\lib\Release.ACP\pci.lib (fm801.c)
	at offset 0002479F 025B3H bytes from F:\src\os2\uniaud32\lib\Release.ACP\pci.lib (via82xx.c)
	at offset 00026D52 01F46H bytes from F:\src\os2\uniaud32\lib\Release.ACP\pci.lib (maestro3.c)
	at offset 00028C98 02981H bytes from F:\src\os2\uniaud32\lib\Release.ACP\pci.lib (intel8x0.c)
	at offset 0002B619 02CCCH bytes from F:\src\os2\uniaud32\lib\Release.ACP\pci.lib (es1968.c)
	at offset 0002E2E5 01B02H bytes from F:\src\os2\uniaud32\lib\Release.ACP\pci.lib (es1938.c)
	at offset 0002FDE7 01A24H bytes from F:\src\os2\uniaud32\lib\Release.ACP\pci.lib (cs4281.c)
	at offset 0003180B 01EA7H bytes from F:\src\os2\uniaud32\lib\Release.ACP\pci.lib (ens1371.c)
	at offset 000336B2 00234H bytes from F:\src\os2\uniaud32\lib\Release.ACP\pci.lib (pci_iomap_compat.c)
	at offset 000338E6 0197BH bytes from F:\src\os2\uniaud32\lib\Release.ACP\ca0106.lib (ca0106_main.c)
	at offset 00035261 0050BH bytes from F:\src\os2\uniaud32\lib\Release.ACP\ca0106.lib (ca_midi.c)
	at offset 0003576C 00B8FH bytes from F:\src\os2\uniaud32\lib\Release.ACP\ca0106.lib (ca0106_mixer.c)
	at offset 000362FB 008F1H bytes from F:\src\os2\uniaud32\lib\Release.ACP\ca0106.lib (ca0106_proc.c)
	at offset 00036BEC 06161H bytes from F:\src\os2\uniaud32\lib\Release.ACP\hda.lib (patch_via.c)
	at offset 0003CD4D 01830H bytes from F:\src\os2\uniaud32\lib\Release.ACP\hda.lib (patch_conexant.c)
	at offset 0003E57D 001D6H bytes from F:\src\os2\uniaud32\lib\Release.ACP\hda.lib (patch_atihdmi.c)
	at offset 0003E753 04D33H bytes from F:\src\os2\uniaud32\lib\Release.ACP\hda.lib (patch_sigmatel.c)
	at offset 00043486 02631H bytes from F:\src\os2\uniaud32\lib\Release.ACP\hda.lib (patch_analog.c)
	at offset 00045AB7 00780H bytes from F:\src\os2\uniaud32\lib\Release.ACP\hda.lib (patch_cmedia.c)
	at offset 00046237 07DE2H bytes from F:\src\os2\uniaud32\lib\Release.ACP\hda.lib (patch_realtek.c)
	at offset 0004E019 0258EH bytes from F:\src\os2\uniaud32\lib\Release.ACP\hda.lib (hda_intel.c)
	at offset 000505A7 03EF8H bytes from F:\src\os2\uniaud32\lib\Release.ACP\hda.lib (hda_codec.c)
	at offset 0005449F 00270H bytes from F:\src\os2\uniaud32\lib\Release.ACP\hda.lib (hda_hwdep.c)
	at offset 0005470F 012C8H bytes from F:\src\os2\uniaud32\lib\Release.ACP\hda.lib (hda_generic.c)
	at offset 000559D7 012F0H bytes from F:\src\os2\uniaud32\lib\Release.ACP\hda.lib (hda_proc.c)
	at offset 00056CC7 0004BH bytes from F:\src\os2\uniaud32\lib\Release.ACP\sequencer.lib (seq.c)
	at offset 00056D12 00699H bytes from F:\src\os2\uniaud32\lib\Release.ACP\sequencer.lib (seq_device.c)
	at offset 000573AB 000A1H bytes from F:\src\os2\uniaud32\lib\Release.ACP\sequencer.lib (seq_info.c)
	at offset 0005744C 00212H bytes from F:\src\os2\uniaud32\lib\Release.ACP\sequencer.lib (seq_system.c)
	at offset 0005765E 00B72H bytes from F:\src\os2\uniaud32\lib\Release.ACP\sequencer.lib (seq_queue.c)
	at offset 000581D0 0077CH bytes from F:\src\os2\uniaud32\lib\Release.ACP\sequencer.lib (seq_memory.c)
	at offset 0005894C 024F9H bytes from F:\src\os2\uniaud32\lib\Release.ACP\sequencer.lib (seq_clientmgr.c)
	at offset 0005AE45 00BDCH bytes from F:\src\os2\uniaud32\lib\Release.ACP\sequencer.lib (seq_ports.c)
	at offset 0005BA21 00759H bytes from F:\src\os2\uniaud32\lib\Release.ACP\sequencer.lib (seq_timer.c)
	at offset 0005C17A 004DEH bytes from F:\src\os2\uniaud32\lib\Release.ACP\sequencer.lib (seq_prioq.c)
	at offset 0005C658 00319H bytes from F:\src\os2\uniaud32\lib\Release.ACP\sequencer.lib (seq_fifo.c)
	at offset 0005C971 003D5H bytes from F:\src\os2\uniaud32\lib\Release.ACP\opl3.lib (opl3_seq.c)
	at offset 0005CD46 0090DH bytes from F:\src\os2\uniaud32\lib\Release.ACP\opl3.lib (opl3_lib.c)
	at offset 0005D653 0029CH bytes from F:\src\os2\uniaud32\lib\Release.ACP\opl3.lib (opl3_drums.c)
	at offset 0005D8EF 00BECH bytes from F:\src\os2\uniaud32\lib\Release.ACP\opl3.lib (opl3_midi.c)
	at offset 0005E4DB 00820H bytes from F:\src\os2\uniaud32\lib\Release.ACP\opl3.lib (opl3_synth.c)
	at offset 0005ECFB 008B7H bytes from F:\src\os2\uniaud32\lib\Release.ACP\mpu401.lib (mpu401_uart.c)
	at offset 0005F5B2 001E3H bytes from F:\src\os2\uniaud32\lib\Release.ACP\cs46xx.lib (cs46xx.c)
	at offset 0005F795 02672H bytes from F:\src\os2\uniaud32\lib\Release.ACP\cs46xx.lib (cs46xx_lib.c)
	at offset 00061E07 0057BH bytes from F:\src\os2\uniaud32\lib\Release.ACP\cs5535audio.lib (cs5535audio.c)
	at offset 00062382 001A2H bytes from F:\src\os2\uniaud32\lib\Release.ACP\cs5535audio.lib (cs5535audio_pm.c)
	at offset 00062524 00518H bytes from F:\src\os2\uniaud32\lib\Release.ACP\cs5535audio.lib (cs5535audio_pcm.c)
	at offset 00062A3C 004DFH bytes from F:\src\os2\uniaud32\lib\Release.ACP\emu10k1.lib (emu10k1.c)
	at offset 00062F1B 00BF5H bytes from F:\src\os2\uniaud32\lib\Release.ACP\emu10k1.lib (p16v.c)
	at offset 00063B10 00149H bytes from F:\src\os2\uniaud32\lib\Release.ACP\emu10k1.lib (timer.c)
	at offset 00063C59 075B4H bytes from F:\src\os2\uniaud32\lib\Release.ACP\emu10k1.lib (emufx.c)
	at offset 0006B20D 01E71H bytes from F:\src\os2\uniaud32\lib\Release.ACP\emu10k1.lib (emumixer.c)
	at offset 0006D07E 027F2H bytes from F:\src\os2\uniaud32\lib\Release.ACP\emu10k1.lib (emupcm.c)
	at offset 0006F870 006ADH bytes from F:\src\os2\uniaud32\lib\Release.ACP\emu10k1.lib (emumpu401.c)
	at offset 0006FF1D 01E56H bytes from F:\src\os2\uniaud32\lib\Release.ACP\emu10k1.lib (emu10k1_main.c)
	at offset 00071D73 00B4CH bytes from F:\src\os2\uniaud32\lib\Release.ACP\emu10k1.lib (emuproc.c)
	at offset 000728BF 00A33H bytes from F:\src\os2\uniaud32\lib\Release.ACP\emu10k1.lib (io.c)
	at offset 000732F2 0025AH bytes from F:\src\os2\uniaud32\lib\Release.ACP\emu10k1.lib (voice.c)
	at offset 0007354C 0081AH bytes from F:\src\os2\uniaud32\lib\Release.ACP\emu10k1.lib (memory.c)
	at offset 00073D66 0041DH bytes from F:\src\os2\uniaud32\lib\Release.ACP\emu10k1.lib (irq.c)
	at offset 00074183 0066EH bytes from F:\src\os2\uniaud32\lib\Release.ACP\ymfpci.lib (ymfpci.c)
	at offset 000747F1 02D18H bytes from F:\src\os2\uniaud32\lib\Release.ACP\ymfpci.lib (ymfpci_main.c)
	at offset 00077509 02113H bytes from F:\src\os2\uniaud32\lib\Release.ACP\ali5451.lib (ali5451.c)
	at offset 0007961C 002E5H bytes from F:\src\os2\uniaud32\lib\Release.ACP\trident.lib (trident.c)
	at offset 00079901 0392DH bytes from F:\src\os2\uniaud32\lib\Release.ACP\trident.lib (trident_main.c)
	at offset 0007D22E 00300H bytes from F:\src\os2\uniaud32\lib\Release.ACP\trident.lib (trident_memory.c)
	at offset 0007D52E 0156BH bytes from F:\src\os2\uniaud32\lib\Release.ACP\nm256.lib (nm256.c)
	at offset 0007EA99 00CEEH bytes from F:\src\os2\uniaud32\lib\Release.ACP\sb.lib (sb_mixer.c)
	at offset 0007F787 003E3H bytes from F:\src\os2\uniaud32\lib\Release.ACP\sb.lib (sb_common.c)
	at offset 0007FB6A 037F9H bytes from F:\src\os2\uniaud32\lib\Release.ACP\core_oss.lib (pcm_oss.c)
	at offset 00083380 00140H bytes from F:\acpi\lib\acpidrv.lib (acpi)
	at offset 000834C0 002BCH bytes from F:\acpi\lib\acpidrv.lib (FindAddress)
	at offset 0008377C 00007H bytes from F:\src\os2\uniaud32\lib\Release.ACP\linuxlib.lib (semaphore.c)
	at offset 00083783 00563H bytes from F:\src\os2\uniaud32\lib\Release.ACP\core.lib (vmaster.c)
	at offset 00083CE6 00071H bytes from F:\src\os2\uniaud32\lib\Release.ACP\core.lib (misc.c)
	at offset 00083D57 000DFH bytes from F:\src\os2\uniaud32\lib\Release.ACP\core.lib (memory.c)
	at offset 00083E36 00CCBH bytes from F:\src\os2\uniaud32\lib\Release.ACP\ac97.lib (ac97_pcm.c)
	at offset 00084B01 06DC9H bytes from F:\src\os2\uniaud32\lib\Release.ACP\ac97.lib (ac97_codec.c)
	at offset 0008B8CA 0103FH bytes from F:\src\os2\uniaud32\lib\Release.ACP\ac97.lib (ac97_proc.c)
	at offset 0008C909 00B03H bytes from F:\src\os2\uniaud32\lib\Release.ACP\sequencer.lib (seq_midi_emul.c)
	at offset 0008D40C 001AAH bytes from F:\src\os2\uniaud32\lib\Release.ACP\synth.lib (util_mem.c)

 0003:0008D5C0 0000029A6H _TEXT                  CODE 32-bit
	at offset 00000000 0004FH bytes from E:\watcom\lib386\os2\clib3r.lib (i8s)
	at offset 00000050 0001CH bytes from E:\watcom\lib386\os2\clib3r.lib (i8m)
	at offset 00000070 000ADH bytes from E:\watcom\lib386\os2\clib3r.lib (strstr.c)
	at offset 00000120 00041H bytes from E:\watcom\lib386\os2\clib3r.lib (strlcpy.c)
	at offset 00000170 00091H bytes from E:\watcom\lib386\os2\clib3r.lib (sscanf.c)
	at offset 00000210 000C7H bytes from E:\watcom\lib386\os2\clib3r.lib (snprintf.c)
	at offset 000002E0 00018H bytes from E:\watcom\lib386\os2\clib3r.lib (memset.c)
	at offset 00000300 00053H bytes from E:\watcom\lib386\os2\clib3r.lib (memmove.c)
	at offset 00000360 0023DH bytes from E:\watcom\lib386\os2\clib3r.lib (strtol.c)
	at offset 000005A0 00101H bytes from E:\watcom\lib386\os2\clib3r.lib (istable.c)
	at offset 000006B0 000A3H bytes from E:\watcom\lib386\os2\clib3r.lib (__stos)
	at offset 00000760 00DCBH bytes from E:\watcom\lib386\os2\clib3r.lib (scnf.c)
	at offset 00001530 00CE4H bytes from E:\watcom\lib386\os2\clib3r.lib (prtf.c)
	at offset 00002214 0004BH bytes from E:\watcom\lib386\os2\clib3r.lib (seterrno.c)
	at offset 00002260 0000EH bytes from E:\watcom\lib386\os2\clib3r.lib (tolower.c)
	at offset 00002270 0004CH bytes from E:\watcom\lib386\os2\clib3r.lib (fdfs386)
	at offset 000022C0 00020H bytes from E:\watcom\lib386\os2\clib3r.lib (strupr.c)
	at offset 000022E0 00008H bytes from E:\watcom\lib386\os2\clib3r.lib (bits.c)
	at offset 000022F0 00042H bytes from E:\watcom\lib386\os2\clib3r.lib (noefgfmt.c)
	at offset 00002332 00128H bytes from E:\watcom\lib386\os2\clib3r.lib (maino32.c)
	at offset 00002460 0002EH bytes from E:\watcom\lib386\os2\clib3r.lib (wctomb.c)
	at offset 00002490 000BCH bytes from E:\watcom\lib386\os2\clib3r.lib (mbtowc.c)
	at offset 00002550 00017H bytes from E:\watcom\lib386\os2\clib3r.lib (mbislead.c)
	at offset 00002570 00074H bytes from E:\watcom\lib386\os2\clib3r.lib (ltoa.c)
	at offset 000025F0 00099H bytes from E:\watcom\lib386\os2\clib3r.lib (lltoa.c)
	at offset 00002690 00074H bytes from E:\watcom\lib386\os2\clib3r.lib (itoa.c)
	at offset 00002710 00070H bytes from E:\watcom\lib386\os2\clib3r.lib (xmsgo32.c)
	at offset 00002780 000B3H bytes from E:\watcom\lib386\os2\clib3r.lib (initrtns.c)
	at offset 00002833 00001H bytes from E:\watcom\lib386\os2\clib3r.lib (crwdata)
	at offset 00002840 0000BH bytes from E:\watcom\lib386\os2\clib3r.lib (cinit.c)
	at offset 0000284B 00132H bytes from E:\watcom\lib386\os2\clib3r.lib (mbinit.c)
	at offset 00002980 00026H bytes from E:\watcom\lib386\os2\clib3r.lib (enterdb.c)

 0003:0008FF68 000000000H LASTCODE32             CODE 32-bit

 0004:00000000 000000007H BEGTEXT                CODE 32-bit
	at offset 00000000 00007H bytes from E:\watcom\lib386\os2\clib3r.lib (segdefns)

 0005:00000000 000000030H BSS32                  BSS 32-bit
	at offset 00000000 00004H bytes from F:\src\os2\uniaud32\drv32\bin\Release.ACP\begin.obj (begin.asm)
	at offset 00000004 0002CH bytes from F:\acpi\lib\acpidrv.lib (acpi)

 0005:00000030 00000173CH _BSS                   BSS 32-bit
	at offset 00000000 0000CH bytes from F:\src\os2\uniaud32\drv32\bin\Release.ACP\strategy.obj (F:\src\os2\uniaud32\drv32\strategy.c)
	at offset 0000000C 0000CH bytes from F:\src\os2\uniaud32\drv32\bin\Release.ACP\read.obj (F:\src\os2\uniaud32\drv32\read.cpp)
	at offset 00000018 00008H bytes from F:\src\os2\uniaud32\drv32\bin\Release.ACP\parse.obj (F:\src\os2\uniaud32\drv32\parse.c)
	at offset 00000020 00006H bytes from F:\src\os2\uniaud32\drv32\bin\Release.ACP\idc.obj (F:\src\os2\uniaud32\drv32\idc.c)
	at offset 00000028 00054H bytes from F:\src\os2\uniaud32\drv32\bin\Release.ACP\rmhelp.obj (F:\src\os2\uniaud32\drv32\rmhelp.cpp)
	at offset 00000080 0003CH bytes from F:\src\os2\uniaud32\drv32\bin\Release.ACP\irq.obj (F:\src\os2\uniaud32\drv32\irq.cpp)
	at offset 000000BC 00028H bytes from F:\src\os2\uniaud32\lib\Release.ACP\linuxlib.lib (ossidc.cpp)
	at offset 000000E4 00004H bytes from F:\src\os2\uniaud32\lib\Release.ACP\linuxlib.lib (debug.c)
	at offset 000000E8 00008H bytes from F:\src\os2\uniaud32\lib\Release.ACP\linuxlib.lib (memory.cpp)
	at offset 000000F0 00440H bytes from F:\src\os2\uniaud32\lib\Release.ACP\linuxlib.lib (pci.c)
	at offset 00000530 0002CH bytes from F:\src\os2\uniaud32\lib\Release.ACP\linuxlib.lib (malloc.cpp)
	at offset 0000055C 00004H bytes from F:\src\os2\uniaud32\lib\Release.ACP\core.lib (hwdep.c)
	at offset 00000560 00004H bytes from F:\src\os2\uniaud32\lib\Release.ACP\core.lib (timer.c)
	at offset 00000564 00020H bytes from F:\src\os2\uniaud32\lib\Release.ACP\core.lib (rawmidi.c)
	at offset 00000584 00104H bytes from F:\src\os2\uniaud32\lib\Release.ACP\core.lib (pcm.c)
	at offset 00000688 0040CH bytes from F:\src\os2\uniaud32\lib\Release.ACP\core.lib (sound.c)
	at offset 00000A94 00010H bytes from F:\src\os2\uniaud32\lib\Release.ACP\core.lib (info.c)
	at offset 00000AA4 000C4H bytes from F:\src\os2\uniaud32\lib\Release.ACP\core.lib (info_oss.c)
	at offset 00000B68 00204H bytes from F:\src\os2\uniaud32\lib\Release.ACP\core.lib (sound_oss.c)
	at offset 00000D6C 00004H bytes from F:\src\os2\uniaud32\lib\Release.ACP\core.lib (memalloc.c)
	at offset 00000D70 0004CH bytes from F:\src\os2\uniaud32\lib\Release.ACP\core.lib (init.c)
	at offset 00000DBC 00028H bytes from F:\src\os2\uniaud32\lib\Release.ACP\pci.lib (bt87x.c)
	at offset 00000DE4 00004H bytes from F:\src\os2\uniaud32\lib\Release.ACP\pci.lib (als4000.c)
	at offset 00000DE8 00024H bytes from F:\src\os2\uniaud32\lib\Release.ACP\pci.lib (cmipci.c)
	at offset 00000E0C 00008H bytes from F:\src\os2\uniaud32\lib\Release.ACP\pci.lib (atiixp.c)
	at offset 00000E14 00024H bytes from F:\src\os2\uniaud32\lib\Release.ACP\pci.lib (fm801.c)
	at offset 00000E38 00014H bytes from F:\src\os2\uniaud32\lib\Release.ACP\pci.lib (via82xx.c)
	at offset 00000E4C 00004H bytes from F:\src\os2\uniaud32\lib\Release.ACP\pci.lib (maestro3.c)
	at offset 00000E50 00018H bytes from F:\src\os2\uniaud32\lib\Release.ACP\pci.lib (intel8x0.c)
	at offset 00000E68 00024H bytes from F:\src\os2\uniaud32\lib\Release.ACP\pci.lib (es1968.c)
	at offset 00000E8C 00004H bytes from F:\src\os2\uniaud32\lib\Release.ACP\pci.lib (es1938.c)
	at offset 00000E90 00024H bytes from F:\src\os2\uniaud32\lib\Release.ACP\pci.lib (cs4281.c)
	at offset 00000EB4 00044H bytes from F:\src\os2\uniaud32\lib\Release.ACP\pci.lib (ens1371.c)
	at offset 00000EF8 00024H bytes from F:\src\os2\uniaud32\lib\Release.ACP\ca0106.lib (ca0106_main.c)
	at offset 00000F1C 00008H bytes from F:\src\os2\uniaud32\lib\Release.ACP\hda.lib (patch_sigmatel.c)
	at offset 00000F24 00068H bytes from F:\src\os2\uniaud32\lib\Release.ACP\hda.lib (hda_intel.c)
	at offset 00000F8C 00008H bytes from F:\src\os2\uniaud32\lib\Release.ACP\sequencer.lib (seq_device.c)
	at offset 00000F94 0000CH bytes from F:\src\os2\uniaud32\lib\Release.ACP\sequencer.lib (seq_info.c)
	at offset 00000FA0 00024H bytes from F:\src\os2\uniaud32\lib\Release.ACP\sequencer.lib (seq_queue.c)
	at offset 00000FC4 003C8H bytes from F:\src\os2\uniaud32\lib\Release.ACP\sequencer.lib (seq_clientmgr.c)
	at offset 0000138C 00044H bytes from F:\src\os2\uniaud32\lib\Release.ACP\cs46xx.lib (cs46xx.c)
	at offset 000013D0 00008H bytes from F:\src\os2\uniaud32\lib\Release.ACP\cs5535audio.lib (cs5535audio.c)
	at offset 000013D8 00084H bytes from F:\src\os2\uniaud32\lib\Release.ACP\emu10k1.lib (emu10k1.c)
	at offset 0000145C 00064H bytes from F:\src\os2\uniaud32\lib\Release.ACP\ymfpci.lib (ymfpci.c)
	at offset 000014C0 00008H bytes from F:\src\os2\uniaud32\lib\Release.ACP\ali5451.lib (ali5451.c)
	at offset 000014C8 00004H bytes from F:\src\os2\uniaud32\lib\Release.ACP\trident.lib (trident.c)
	at offset 000014CC 0001CH bytes from F:\src\os2\uniaud32\lib\Release.ACP\nm256.lib (nm256.c)
	at offset 000014E8 00020H bytes from F:\src\os2\uniaud32\lib\Release.ACP\core_oss.lib (pcm_oss.c)
	at offset 00001508 00106H bytes from E:\watcom\lib386\os2\clib3r.lib (maino32.c)
	at offset 00001610 00101H bytes from E:\watcom\lib386\os2\clib3r.lib (mbislead.c)
	at offset 00001714 00004H bytes from E:\watcom\lib386\os2\clib3r.lib (mbisdbcs.c)
	at offset 00001718 00004H bytes from E:\watcom\lib386\os2\clib3r.lib (cinit.c)
	at offset 0000171C 00020H bytes from F:\src\os2\uniaud32\lib\Release.ACP\ac97.lib (ac97_codec.c)

 0005:0000176C 000000000H C_COMMON               DATA 32-bit

 0005:0000176C 000000010H c_common               DATA 32-bit
	at offset 00000000 00010H bytes from F:\acpi\lib\acpidrv.lib (acpi)

 0005:0000177C 000000090H DATA32                 DATA 32-bit
	at offset 00000000 00082H bytes from F:\src\os2\uniaud32\drv32\bin\Release.ACP\startup.obj (startup.asm)
	at offset 00000084 0000CH bytes from F:\src\os2\uniaud32\drv32\bin\Release.ACP\devhlp.obj (devhlp.asm)

 0005:00001810 000060D24H _DATA                  DATA 32-bit
	at offset 00000000 00080H bytes from F:\src\os2\uniaud32\drv32\bin\Release.ACP\strategy.obj (F:\src\os2\uniaud32\drv32\strategy.c)
	at offset 00000080 00018H bytes from F:\src\os2\uniaud32\drv32\bin\Release.ACP\parse.obj (F:\src\os2\uniaud32\drv32\parse.c)
	at offset 00000098 00004H bytes from F:\src\os2\uniaud32\drv32\bin\Release.ACP\rmhelp.obj (F:\src\os2\uniaud32\drv32\rmhelp.cpp)
	at offset 0000009C 00020H bytes from F:\src\os2\uniaud32\drv32\bin\Release.ACP\irq.obj (F:\src\os2\uniaud32\drv32\irq.cpp)
	at offset 000000BC 0000CH bytes from F:\src\os2\uniaud32\lib\Release.ACP\linuxlib.lib (timer.c)
	at offset 000000C8 00028H bytes from F:\src\os2\uniaud32\lib\Release.ACP\linuxlib.lib (task.c)
	at offset 000000F0 00414H bytes from F:\src\os2\uniaud32\lib\Release.ACP\linuxlib.lib (misc.c)
	at offset 00000504 00108H bytes from F:\src\os2\uniaud32\lib\Release.ACP\linuxlib.lib (ossidc.cpp)
	at offset 0000060C 00004H bytes from F:\src\os2\uniaud32\lib\Release.ACP\linuxlib.lib (soundmidi.c)
	at offset 00000610 001F1H bytes from F:\src\os2\uniaud32\lib\Release.ACP\linuxlib.lib (soundmixer.c)
	at offset 00000804 061D8H bytes from F:\src\os2\uniaud32\lib\Release.ACP\linuxlib.lib (sound.c)
	at offset 000069DC 00013H bytes from F:\src\os2\uniaud32\lib\Release.ACP\linuxlib.lib (debug.c)
	at offset 000069F0 0202CH bytes from F:\src\os2\uniaud32\lib\Release.ACP\linuxlib.lib (ioctl.c)
	at offset 00008A1C 00860H bytes from F:\src\os2\uniaud32\lib\Release.ACP\linuxlib.lib (irq.c)
	at offset 0000927C 03E44H bytes from F:\src\os2\uniaud32\lib\Release.ACP\linuxlib.lib (pci.c)
	at offset 0000D0C0 00004H bytes from F:\src\os2\uniaud32\lib\Release.ACP\linuxlib.lib (malloc.cpp)
	at offset 0000D0C4 00068H bytes from F:\src\os2\uniaud32\lib\Release.ACP\core.lib (hwdep.c)
	at offset 0000D12C 000ACH bytes from F:\src\os2\uniaud32\lib\Release.ACP\core.lib (timer.c)
	at offset 0000D1D8 00090H bytes from F:\src\os2\uniaud32\lib\Release.ACP\core.lib (rawmidi.c)
	at offset 0000D268 00210H bytes from F:\src\os2\uniaud32\lib\Release.ACP\core.lib (pcm_misc.c)
	at offset 0000D478 000A0H bytes from F:\src\os2\uniaud32\lib\Release.ACP\core.lib (pcm_lib.c)
	at offset 0000D518 000E0H bytes from F:\src\os2\uniaud32\lib\Release.ACP\core.lib (pcm.c)
	at offset 0000D5F8 0005CH bytes from F:\src\os2\uniaud32\lib\Release.ACP\core.lib (sound.c)
	at offset 0000D654 00048H bytes from F:\src\os2\uniaud32\lib\Release.ACP\core.lib (info.c)
	at offset 0000D69C 00008H bytes from F:\src\os2\uniaud32\lib\Release.ACP\core.lib (pcm_memory.c)
	at offset 0000D6A4 00030H bytes from F:\src\os2\uniaud32\lib\Release.ACP\core.lib (pcm_timer.c)
	at offset 0000D6D4 00144H bytes from F:\src\os2\uniaud32\lib\Release.ACP\core.lib (pcm_native.c)
	at offset 0000D818 0000CH bytes from F:\src\os2\uniaud32\lib\Release.ACP\core.lib (info_oss.c)
	at offset 0000D824 0000CH bytes from F:\src\os2\uniaud32\lib\Release.ACP\core.lib (sound_oss.c)
	at offset 0000D830 00060H bytes from F:\src\os2\uniaud32\lib\Release.ACP\core.lib (control.c)
	at offset 0000D890 0001CH bytes from F:\src\os2\uniaud32\lib\Release.ACP\core.lib (memalloc.c)
	at offset 0000D8AC 00058H bytes from F:\src\os2\uniaud32\lib\Release.ACP\core.lib (init.c)
	at offset 0000D904 00264H bytes from F:\src\os2\uniaud32\lib\Release.ACP\pci.lib (bt87x.c)
	at offset 0000DB68 00164H bytes from F:\src\os2\uniaud32\lib\Release.ACP\pci.lib (als4000.c)
	at offset 0000DCCC 00D81H bytes from F:\src\os2\uniaud32\lib\Release.ACP\pci.lib (cmipci.c)
	at offset 0000EA50 00320H bytes from F:\src\os2\uniaud32\lib\Release.ACP\pci.lib (atiixp.c)
	at offset 0000ED70 0046CH bytes from F:\src\os2\uniaud32\lib\Release.ACP\pci.lib (fm801.c)
	at offset 0000F1DC 005D4H bytes from F:\src\os2\uniaud32\lib\Release.ACP\pci.lib (via82xx.c)
	at offset 0000F7B0 00528H bytes from F:\src\os2\uniaud32\lib\Release.ACP\pci.lib (maestro3.c)
	at offset 0000FCD8 00D10H bytes from F:\src\os2\uniaud32\lib\Release.ACP\pci.lib (intel8x0.c)
	at offset 000109E8 00244H bytes from F:\src\os2\uniaud32\lib\Release.ACP\pci.lib (es1968.c)
	at offset 00010C2C 00861H bytes from F:\src\os2\uniaud32\lib\Release.ACP\pci.lib (es1938.c)
	at offset 00011490 00298H bytes from F:\src\os2\uniaud32\lib\Release.ACP\pci.lib (cs4281.c)
	at offset 00011728 0040CH bytes from F:\src\os2\uniaud32\lib\Release.ACP\pci.lib (ens1371.c)
	at offset 00011B34 004B4H bytes from F:\src\os2\uniaud32\lib\Release.ACP\ca0106.lib (ca0106_main.c)
	at offset 00011FE8 00020H bytes from F:\src\os2\uniaud32\lib\Release.ACP\ca0106.lib (ca_midi.c)
	at offset 00012008 00634H bytes from F:\src\os2\uniaud32\lib\Release.ACP\ca0106.lib (ca0106_mixer.c)
	at offset 0001263C 00058H bytes from F:\src\os2\uniaud32\lib\Release.ACP\ca0106.lib (ca0106_proc.c)
	at offset 00012694 029D4H bytes from F:\src\os2\uniaud32\lib\Release.ACP\hda.lib (patch_via.c)
	at offset 00015068 0276CH bytes from F:\src\os2\uniaud32\lib\Release.ACP\hda.lib (patch_conexant.c)
	at offset 000177D4 00160H bytes from F:\src\os2\uniaud32\lib\Release.ACP\hda.lib (patch_atihdmi.c)
	at offset 00017934 02800H bytes from F:\src\os2\uniaud32\lib\Release.ACP\hda.lib (patch_sigmatel.c)
	at offset 0001A134 07788H bytes from F:\src\os2\uniaud32\lib\Release.ACP\hda.lib (patch_analog.c)
	at offset 000218BC 00794H bytes from F:\src\os2\uniaud32\lib\Release.ACP\hda.lib (patch_cmedia.c)
	at offset 00022050 1ECE3H bytes from F:\src\os2\uniaud32\lib\Release.ACP\hda.lib (patch_realtek.c)
	at offset 00040D34 002D8H bytes from F:\src\os2\uniaud32\lib\Release.ACP\hda.lib (hda_intel.c)
	at offset 0004100C 00477H bytes from F:\src\os2\uniaud32\lib\Release.ACP\hda.lib (hda_codec.c)
	at offset 00041484 00090H bytes from F:\src\os2\uniaud32\lib\Release.ACP\hda.lib (hda_generic.c)
	at offset 00041514 000E0H bytes from F:\src\os2\uniaud32\lib\Release.ACP\hda.lib (hda_proc.c)
	at offset 000415F4 0005CH bytes from F:\src\os2\uniaud32\lib\Release.ACP\sequencer.lib (seq.c)
	at offset 00041650 00028H bytes from F:\src\os2\uniaud32\lib\Release.ACP\sequencer.lib (seq_device.c)
	at offset 00041678 00008H bytes from F:\src\os2\uniaud32\lib\Release.ACP\sequencer.lib (seq_system.c)
	at offset 00041680 00004H bytes from F:\src\os2\uniaud32\lib\Release.ACP\sequencer.lib (seq_queue.c)
	at offset 00041684 00140H bytes from F:\src\os2\uniaud32\lib\Release.ACP\sequencer.lib (seq_clientmgr.c)
	at offset 000417C4 00030H bytes from F:\src\os2\uniaud32\lib\Release.ACP\opl3.lib (opl3_seq.c)
	at offset 000417F4 00074H bytes from F:\src\os2\uniaud32\lib\Release.ACP\opl3.lib (opl3_lib.c)
	at offset 00041868 000A7H bytes from F:\src\os2\uniaud32\lib\Release.ACP\opl3.lib (opl3_drums.c)
	at offset 00041910 000E8H bytes from F:\src\os2\uniaud32\lib\Release.ACP\opl3.lib (opl3_midi.c)
	at offset 000419F8 00024H bytes from F:\src\os2\uniaud32\lib\Release.ACP\opl3.lib (opl3_synth.c)
	at offset 00041A1C 00028H bytes from F:\src\os2\uniaud32\lib\Release.ACP\mpu401.lib (mpu401_uart.c)
	at offset 00041A44 000ACH bytes from F:\src\os2\uniaud32\lib\Release.ACP\cs46xx.lib (cs46xx.c)
	at offset 00041AF0 0DBC4H bytes from F:\src\os2\uniaud32\lib\Release.ACP\cs46xx.lib (cs46xx_lib.c)
	at offset 0004F6B4 000C4H bytes from F:\src\os2\uniaud32\lib\Release.ACP\cs5535audio.lib (cs5535audio.c)
	at offset 0004F778 00110H bytes from F:\src\os2\uniaud32\lib\Release.ACP\cs5535audio.lib (cs5535audio_pcm.c)
	at offset 0004F888 000ECH bytes from F:\src\os2\uniaud32\lib\Release.ACP\emu10k1.lib (emu10k1.c)
	at offset 0004F974 002E8H bytes from F:\src\os2\uniaud32\lib\Release.ACP\emu10k1.lib (p16v.c)
	at offset 0004FC5C 00030H bytes from F:\src\os2\uniaud32\lib\Release.ACP\emu10k1.lib (timer.c)
	at offset 0004FC8C 001C0H bytes from F:\src\os2\uniaud32\lib\Release.ACP\emu10k1.lib (emufx.c)
	at offset 0004FE4C 0169CH bytes from F:\src\os2\uniaud32\lib\Release.ACP\emu10k1.lib (emumixer.c)
	at offset 000514E8 00334H bytes from F:\src\os2\uniaud32\lib\Release.ACP\emu10k1.lib (emupcm.c)
	at offset 0005181C 00020H bytes from F:\src\os2\uniaud32\lib\Release.ACP\emu10k1.lib (emumpu401.c)
	at offset 0005183C 00894H bytes from F:\src\os2\uniaud32\lib\Release.ACP\emu10k1.lib (emu10k1_main.c)
	at offset 000520D0 00270H bytes from F:\src\os2\uniaud32\lib\Release.ACP\emu10k1.lib (emuproc.c)
	at offset 00052340 00280H bytes from F:\src\os2\uniaud32\lib\Release.ACP\emu10k1.lib (io.c)
	at offset 000525C0 0008CH bytes from F:\src\os2\uniaud32\lib\Release.ACP\ymfpci.lib (ymfpci.c)
	at offset 0005264C 006D8H bytes from F:\src\os2\uniaud32\lib\Release.ACP\ymfpci.lib (ymfpci_main.c)
	at offset 00052D24 002B0H bytes from F:\src\os2\uniaud32\lib\Release.ACP\ali5451.lib (ali5451.c)
	at offset 00052FD4 000CCH bytes from F:\src\os2\uniaud32\lib\Release.ACP\trident.lib (trident.c)
	at offset 000530A0 004ECH bytes from F:\src\os2\uniaud32\lib\Release.ACP\trident.lib (trident_main.c)
	at offset 0005358C 0C798H bytes from F:\src\os2\uniaud32\lib\Release.ACP\nm256.lib (nm256.c)
	at offset 0005FD24 004B8H bytes from F:\src\os2\uniaud32\lib\Release.ACP\sb.lib (sb_mixer.c)
	at offset 000601DC 00014H bytes from F:\src\os2\uniaud32\lib\Release.ACP\sb.lib (sb_common.c)
	at offset 000601F0 00080H bytes from F:\src\os2\uniaud32\lib\Release.ACP\core_oss.lib (pcm_oss.c)
	at offset 00060270 0008CH bytes from E:\watcom\lib386\os2\clib3r.lib (strtol.c)
	at offset 000602FC 00008H bytes from E:\watcom\lib386\os2\clib3r.lib (noefgfmt.c)
	at offset 00060304 00040H bytes from E:\watcom\lib386\os2\clib3r.lib (maino32.c)
	at offset 00060344 0004AH bytes from E:\watcom\lib386\os2\clib3r.lib (crwdata)
	at offset 00060390 00004H bytes from E:\watcom\lib386\os2\clib3r.lib (mbinit.c)
	at offset 00060394 00001H bytes from E:\watcom\lib386\os2\clib3r.lib (enterdb.c)
	at offset 00060398 00004H bytes from E:\watcom\lib386\os2\clib3r.lib (amblksiz.c)
	at offset 0006039C 00051H bytes from F:\src\os2\uniaud32\lib\Release.ACP\ac97.lib (ac97_pcm.c)
	at offset 000603F0 00802H bytes from F:\src\os2\uniaud32\lib\Release.ACP\ac97.lib (ac97_codec.c)
	at offset 00060BF4 00110H bytes from F:\src\os2\uniaud32\lib\Release.ACP\ac97.lib (ac97_proc.c)
	at offset 00060D04 00018H bytes from F:\src\os2\uniaud32\lib\Release.ACP\sequencer.lib (seq_midi_emul.c)
	at offset 00060D1C 00008H bytes from F:\src\os2\uniaud32\lib\Release.ACP\synth.lib (util_mem.c)

 0005:00062534 000012745H CONST                  DATA 32-bit
	at offset 00000000 00038H bytes from F:\src\os2\uniaud32\drv32\bin\Release.ACP\init.obj (F:\src\os2\uniaud32\drv32\init.c)
	at offset 00000038 00073H bytes from F:\src\os2\uniaud32\drv32\bin\Release.ACP\parse.obj (F:\src\os2\uniaud32\drv32\parse.c)
	at offset 000000AB 00096H bytes from F:\src\os2\uniaud32\drv32\bin\Release.ACP\dispatch.obj (F:\src\os2\uniaud32\drv32\dispatch.c)
	at offset 00000141 0006AH bytes from F:\src\os2\uniaud32\drv32\bin\Release.ACP\rmhelp.obj (F:\src\os2\uniaud32\drv32\rmhelp.cpp)
	at offset 000001AC 00029H bytes from F:\src\os2\uniaud32\lib\Release.ACP\linuxlib.lib (vsprintf.c)
	at offset 000001D8 00054H bytes from F:\src\os2\uniaud32\lib\Release.ACP\linuxlib.lib (misc.c)
	at offset 0000022C 0005AH bytes from F:\src\os2\uniaud32\lib\Release.ACP\linuxlib.lib (ossidc.cpp)
	at offset 00000288 000BBH bytes from F:\src\os2\uniaud32\lib\Release.ACP\linuxlib.lib (soundmidi.c)
	at offset 00000344 0022FH bytes from F:\src\os2\uniaud32\lib\Release.ACP\linuxlib.lib (soundmixer.c)
	at offset 00000574 0057FH bytes from F:\src\os2\uniaud32\lib\Release.ACP\linuxlib.lib (sound.c)
	at offset 00000AF4 00101H bytes from F:\src\os2\uniaud32\lib\Release.ACP\linuxlib.lib (ioctl.c)
	at offset 00000BF8 00057H bytes from F:\src\os2\uniaud32\lib\Release.ACP\linuxlib.lib (irq.c)
	at offset 00000C50 0012BH bytes from F:\src\os2\uniaud32\lib\Release.ACP\linuxlib.lib (pci.c)
	at offset 00000D7B 000A1H bytes from F:\src\os2\uniaud32\lib\Release.ACP\linuxlib.lib (malloc.cpp)
	at offset 00000E1C 000E9H bytes from F:\src\os2\uniaud32\lib\Release.ACP\core.lib (hwdep.c)
	at offset 00000F08 00146H bytes from F:\src\os2\uniaud32\lib\Release.ACP\core.lib (timer.c)
	at offset 00001050 002F3H bytes from F:\src\os2\uniaud32\lib\Release.ACP\core.lib (rawmidi.c)
	at offset 00001344 00083H bytes from F:\src\os2\uniaud32\lib\Release.ACP\core.lib (pcm_lib.c)
	at offset 000013C8 001FCH bytes from F:\src\os2\uniaud32\lib\Release.ACP\core.lib (pcm.c)
	at offset 000015C4 000DEH bytes from F:\src\os2\uniaud32\lib\Release.ACP\core.lib (sound.c)
	at offset 000016A4 000B4H bytes from F:\src\os2\uniaud32\lib\Release.ACP\core.lib (info.c)
	at offset 00001758 0006AH bytes from F:\src\os2\uniaud32\lib\Release.ACP\core.lib (pcm_timer.c)
	at offset 000017C4 000A4H bytes from F:\src\os2\uniaud32\lib\Release.ACP\core.lib (pcm_native.c)
	at offset 00001868 000F2H bytes from F:\src\os2\uniaud32\lib\Release.ACP\core.lib (info_oss.c)
	at offset 0000195C 00068H bytes from F:\src\os2\uniaud32\lib\Release.ACP\core.lib (sound_oss.c)
	at offset 000019C4 000BDH bytes from F:\src\os2\uniaud32\lib\Release.ACP\core.lib (device.c)
	at offset 00001A84 000D9H bytes from F:\src\os2\uniaud32\lib\Release.ACP\core.lib (control.c)
	at offset 00001B60 0005BH bytes from F:\src\os2\uniaud32\lib\Release.ACP\core.lib (memalloc.c)
	at offset 00001BBC 0022FH bytes from F:\src\os2\uniaud32\lib\Release.ACP\core.lib (init.c)
	at offset 00001DEC 00311H bytes from F:\src\os2\uniaud32\lib\Release.ACP\pci.lib (bt87x.c)
	at offset 00002100 00103H bytes from F:\src\os2\uniaud32\lib\Release.ACP\pci.lib (als4000.c)
	at offset 00002204 00578H bytes from F:\src\os2\uniaud32\lib\Release.ACP\pci.lib (cmipci.c)
	at offset 0000277C 00228H bytes from F:\src\os2\uniaud32\lib\Release.ACP\pci.lib (atiixp.c)
	at offset 000029A4 0027EH bytes from F:\src\os2\uniaud32\lib\Release.ACP\pci.lib (fm801.c)
	at offset 00002C24 00471H bytes from F:\src\os2\uniaud32\lib\Release.ACP\pci.lib (via82xx.c)
	at offset 00003098 001EAH bytes from F:\src\os2\uniaud32\lib\Release.ACP\pci.lib (maestro3.c)
	at offset 00003284 00A12H bytes from F:\src\os2\uniaud32\lib\Release.ACP\pci.lib (intel8x0.c)
	at offset 00003C98 002FBH bytes from F:\src\os2\uniaud32\lib\Release.ACP\pci.lib (es1968.c)
	at offset 00003F94 00422H bytes from F:\src\os2\uniaud32\lib\Release.ACP\pci.lib (es1938.c)
	at offset 000043B8 002CBH bytes from F:\src\os2\uniaud32\lib\Release.ACP\pci.lib (cs4281.c)
	at offset 00004684 00266H bytes from F:\src\os2\uniaud32\lib\Release.ACP\pci.lib (ens1371.c)
	at offset 000048EC 002D4H bytes from F:\src\os2\uniaud32\lib\Release.ACP\ca0106.lib (ca0106_main.c)
	at offset 00004BC0 00045H bytes from F:\src\os2\uniaud32\lib\Release.ACP\ca0106.lib (ca_midi.c)
	at offset 00004C08 0067DH bytes from F:\src\os2\uniaud32\lib\Release.ACP\ca0106.lib (ca0106_mixer.c)
	at offset 00005288 003C4H bytes from F:\src\os2\uniaud32\lib\Release.ACP\ca0106.lib (ca0106_proc.c)
	at offset 0000564C 00560H bytes from F:\src\os2\uniaud32\lib\Release.ACP\hda.lib (patch_via.c)
	at offset 00005BAC 0054DH bytes from F:\src\os2\uniaud32\lib\Release.ACP\hda.lib (patch_conexant.c)
	at offset 000060FC 00048H bytes from F:\src\os2\uniaud32\lib\Release.ACP\hda.lib (patch_atihdmi.c)
	at offset 00006144 00AF9H bytes from F:\src\os2\uniaud32\lib\Release.ACP\hda.lib (patch_sigmatel.c)
	at offset 00006C40 00891H bytes from F:\src\os2\uniaud32\lib\Release.ACP\hda.lib (patch_analog.c)
	at offset 000074D4 0016DH bytes from F:\src\os2\uniaud32\lib\Release.ACP\hda.lib (patch_cmedia.c)
	at offset 00007644 012FCH bytes from F:\src\os2\uniaud32\lib\Release.ACP\hda.lib (patch_realtek.c)
	at offset 00008940 00762H bytes from F:\src\os2\uniaud32\lib\Release.ACP\hda.lib (hda_intel.c)
	at offset 000090A4 00840H bytes from F:\src\os2\uniaud32\lib\Release.ACP\hda.lib (hda_codec.c)
	at offset 000098E4 0000DH bytes from F:\src\os2\uniaud32\lib\Release.ACP\hda.lib (hda_hwdep.c)
	at offset 000098F4 001CAH bytes from F:\src\os2\uniaud32\lib\Release.ACP\hda.lib (hda_generic.c)
	at offset 00009AC0 00784H bytes from F:\src\os2\uniaud32\lib\Release.ACP\hda.lib (hda_proc.c)
	at offset 0000A244 00163H bytes from F:\src\os2\uniaud32\lib\Release.ACP\sequencer.lib (seq_device.c)
	at offset 0000A3A8 00015H bytes from F:\src\os2\uniaud32\lib\Release.ACP\sequencer.lib (seq_info.c)
	at offset 0000A3C0 00016H bytes from F:\src\os2\uniaud32\lib\Release.ACP\sequencer.lib (seq_system.c)
	at offset 0000A3D8 00156H bytes from F:\src\os2\uniaud32\lib\Release.ACP\sequencer.lib (seq_queue.c)
	at offset 0000A530 0011AH bytes from F:\src\os2\uniaud32\lib\Release.ACP\sequencer.lib (seq_memory.c)
	at offset 0000A64C 001FBH bytes from F:\src\os2\uniaud32\lib\Release.ACP\sequencer.lib (seq_clientmgr.c)
	at offset 0000A848 00060H bytes from F:\src\os2\uniaud32\lib\Release.ACP\sequencer.lib (seq_ports.c)
	at offset 0000A8A8 00127H bytes from F:\src\os2\uniaud32\lib\Release.ACP\sequencer.lib (seq_timer.c)
	at offset 0000A9D0 000C3H bytes from F:\src\os2\uniaud32\lib\Release.ACP\sequencer.lib (seq_prioq.c)
	at offset 0000AA94 00027H bytes from F:\src\os2\uniaud32\lib\Release.ACP\sequencer.lib (seq_fifo.c)
	at offset 0000AABC 00028H bytes from F:\src\os2\uniaud32\lib\Release.ACP\opl3.lib (opl3_seq.c)
	at offset 0000AAE4 0014DH bytes from F:\src\os2\uniaud32\lib\Release.ACP\opl3.lib (opl3_lib.c)
	at offset 0000AC34 0000FH bytes from F:\src\os2\uniaud32\lib\Release.ACP\opl3.lib (opl3_synth.c)
	at offset 0000AC44 000E6H bytes from F:\src\os2\uniaud32\lib\Release.ACP\mpu401.lib (mpu401_uart.c)
	at offset 0000AD2C 00035H bytes from F:\src\os2\uniaud32\lib\Release.ACP\cs46xx.lib (cs46xx.c)
	at offset 0000AD64 00474H bytes from F:\src\os2\uniaud32\lib\Release.ACP\cs46xx.lib (cs46xx_lib.c)
	at offset 0000B1D8 00129H bytes from F:\src\os2\uniaud32\lib\Release.ACP\cs5535audio.lib (cs5535audio.c)
	at offset 0000B304 000C2H bytes from F:\src\os2\uniaud32\lib\Release.ACP\cs5535audio.lib (cs5535audio_pm.c)
	at offset 0000B3C8 0005CH bytes from F:\src\os2\uniaud32\lib\Release.ACP\cs5535audio.lib (cs5535audio_pcm.c)
	at offset 0000B424 000BBH bytes from F:\src\os2\uniaud32\lib\Release.ACP\emu10k1.lib (emu10k1.c)
	at offset 0000B4E0 00189H bytes from F:\src\os2\uniaud32\lib\Release.ACP\emu10k1.lib (p16v.c)
	at offset 0000B66C 00016H bytes from F:\src\os2\uniaud32\lib\Release.ACP\emu10k1.lib (timer.c)
	at offset 0000B684 00B47H bytes from F:\src\os2\uniaud32\lib\Release.ACP\emu10k1.lib (emufx.c)
	at offset 0000C1CC 01071H bytes from F:\src\os2\uniaud32\lib\Release.ACP\emu10k1.lib (emumixer.c)
	at offset 0000D240 0009DH bytes from F:\src\os2\uniaud32\lib\Release.ACP\emu10k1.lib (emupcm.c)
	at offset 0000D2E0 00082H bytes from F:\src\os2\uniaud32\lib\Release.ACP\emu10k1.lib (emumpu401.c)
	at offset 0000D364 006A2H bytes from F:\src\os2\uniaud32\lib\Release.ACP\emu10k1.lib (emu10k1_main.c)
	at offset 0000DA08 00831H bytes from F:\src\os2\uniaud32\lib\Release.ACP\emu10k1.lib (emuproc.c)
	at offset 0000E23C 0009CH bytes from F:\src\os2\uniaud32\lib\Release.ACP\emu10k1.lib (io.c)
	at offset 0000E2D8 0008CH bytes from F:\src\os2\uniaud32\lib\Release.ACP\emu10k1.lib (memory.c)
	at offset 0000E364 000C9H bytes from F:\src\os2\uniaud32\lib\Release.ACP\emu10k1.lib (irq.c)
	at offset 0000E430 00128H bytes from F:\src\os2\uniaud32\lib\Release.ACP\ymfpci.lib (ymfpci.c)
	at offset 0000E558 00374H bytes from F:\src\os2\uniaud32\lib\Release.ACP\ymfpci.lib (ymfpci_main.c)
	at offset 0000E8CC 00425H bytes from F:\src\os2\uniaud32\lib\Release.ACP\ali5451.lib (ali5451.c)
	at offset 0000ECF4 00068H bytes from F:\src\os2\uniaud32\lib\Release.ACP\trident.lib (trident.c)
	at offset 0000ED5C 00442H bytes from F:\src\os2\uniaud32\lib\Release.ACP\trident.lib (trident_main.c)
	at offset 0000F1A0 00035H bytes from F:\src\os2\uniaud32\lib\Release.ACP\trident.lib (trident_memory.c)
	at offset 0000F1D8 003AFH bytes from F:\src\os2\uniaud32\lib\Release.ACP\nm256.lib (nm256.c)
	at offset 0000F588 0036EH bytes from F:\src\os2\uniaud32\lib\Release.ACP\sb.lib (sb_mixer.c)
	at offset 0000F8F8 00134H bytes from F:\src\os2\uniaud32\lib\Release.ACP\sb.lib (sb_common.c)
	at offset 0000FA2C 00227H bytes from F:\src\os2\uniaud32\lib\Release.ACP\core_oss.lib (pcm_oss.c)
	at offset 0000FC54 00025H bytes from E:\watcom\lib386\os2\clib3r.lib (alphabet.c)
	at offset 0000FC7C 0001AH bytes from F:\src\os2\uniaud32\lib\Release.ACP\core.lib (vmaster.c)
	at offset 0000FC98 0008CH bytes from F:\src\os2\uniaud32\lib\Release.ACP\ac97.lib (ac97_pcm.c)
	at offset 0000FD24 01DD2H bytes from F:\src\os2\uniaud32\lib\Release.ACP\ac97.lib (ac97_codec.c)
	at offset 00011AF8 00BFFH bytes from F:\src\os2\uniaud32\lib\Release.ACP\ac97.lib (ac97_proc.c)
	at offset 000126F8 0004DH bytes from F:\src\os2\uniaud32\lib\Release.ACP\sequencer.lib (seq_midi_emul.c)

 0005:00074C80 00000675AH CONST2                 DATA 32-bit
	at offset 00000000 0017BH bytes from F:\src\os2\uniaud32\drv32\bin\Release.ACP\init.obj (F:\src\os2\uniaud32\drv32\init.c)
	at offset 0000017C 00040H bytes from F:\src\os2\uniaud32\lib\Release.ACP\core.lib (info.c)
	at offset 000001BC 00004H bytes from F:\src\os2\uniaud32\lib\Release.ACP\core.lib (pcm_memory.c)
	at offset 000001C0 0000CH bytes from F:\src\os2\uniaud32\lib\Release.ACP\core.lib (pcm_native.c)
	at offset 000001CC 001C0H bytes from F:\src\os2\uniaud32\lib\Release.ACP\pci.lib (bt87x.c)
	at offset 0000038C 00060H bytes from F:\src\os2\uniaud32\lib\Release.ACP\pci.lib (als4000.c)
	at offset 000003EC 00100H bytes from F:\src\os2\uniaud32\lib\Release.ACP\pci.lib (cmipci.c)
	at offset 000004EC 0008CH bytes from F:\src\os2\uniaud32\lib\Release.ACP\pci.lib (atiixp.c)
	at offset 00000578 00064H bytes from F:\src\os2\uniaud32\lib\Release.ACP\pci.lib (fm801.c)
	at offset 000005DC 00064H bytes from F:\src\os2\uniaud32\lib\Release.ACP\pci.lib (via82xx.c)
	at offset 00000640 001B8H bytes from F:\src\os2\uniaud32\lib\Release.ACP\pci.lib (maestro3.c)
	at offset 000007F8 002A0H bytes from F:\src\os2\uniaud32\lib\Release.ACP\pci.lib (intel8x0.c)
	at offset 00000A98 00070H bytes from F:\src\os2\uniaud32\lib\Release.ACP\pci.lib (es1968.c)
	at offset 00000B08 00048H bytes from F:\src\os2\uniaud32\lib\Release.ACP\pci.lib (es1938.c)
	at offset 00000B50 00048H bytes from F:\src\os2\uniaud32\lib\Release.ACP\pci.lib (cs4281.c)
	at offset 00000B98 00080H bytes from F:\src\os2\uniaud32\lib\Release.ACP\pci.lib (ens1371.c)
	at offset 00000C18 00058H bytes from F:\src\os2\uniaud32\lib\Release.ACP\ca0106.lib (ca0106_main.c)
	at offset 00000C70 00020H bytes from F:\src\os2\uniaud32\lib\Release.ACP\ca0106.lib (ca0106_mixer.c)
	at offset 00000C90 00108H bytes from F:\src\os2\uniaud32\lib\Release.ACP\hda.lib (patch_conexant.c)
	at offset 00000D98 00068H bytes from F:\src\os2\uniaud32\lib\Release.ACP\hda.lib (patch_realtek.c)
	at offset 00000E00 00428H bytes from F:\src\os2\uniaud32\lib\Release.ACP\hda.lib (hda_intel.c)
	at offset 00001228 00070H bytes from F:\src\os2\uniaud32\lib\Release.ACP\cs46xx.lib (cs46xx.c)
	at offset 00001298 00054H bytes from F:\src\os2\uniaud32\lib\Release.ACP\cs5535audio.lib (cs5535audio.c)
	at offset 000012EC 00070H bytes from F:\src\os2\uniaud32\lib\Release.ACP\emu10k1.lib (emu10k1.c)
	at offset 0000135C 00010H bytes from F:\src\os2\uniaud32\lib\Release.ACP\emu10k1.lib (p16v.c)
	at offset 0000136C 00814H bytes from F:\src\os2\uniaud32\lib\Release.ACP\emu10k1.lib (emufx.c)
	at offset 00001B80 00010H bytes from F:\src\os2\uniaud32\lib\Release.ACP\emu10k1.lib (emumixer.c)
	at offset 00001B90 000C4H bytes from F:\src\os2\uniaud32\lib\Release.ACP\ymfpci.lib (ymfpci.c)
	at offset 00001C54 00010H bytes from F:\src\os2\uniaud32\lib\Release.ACP\ymfpci.lib (ymfpci_main.c)
	at offset 00001C64 00038H bytes from F:\src\os2\uniaud32\lib\Release.ACP\ali5451.lib (ali5451.c)
	at offset 00001C9C 00070H bytes from F:\src\os2\uniaud32\lib\Release.ACP\trident.lib (trident.c)
	at offset 00001D0C 00020H bytes from F:\src\os2\uniaud32\lib\Release.ACP\trident.lib (trident_main.c)
	at offset 00001D2C 00070H bytes from F:\src\os2\uniaud32\lib\Release.ACP\nm256.lib (nm256.c)
	at offset 00001D9C 00018H bytes from F:\src\os2\uniaud32\lib\Release.ACP\ac97.lib (ac97_pcm.c)
	at offset 00001DB4 049A6H bytes from F:\src\os2\uniaud32\lib\Release.ACP\ac97.lib (ac97_codec.c)

 0005:0007B3DC 000000004H LASTDATA32             DATA 32-bit
	at offset 00000000 00004H bytes from F:\src\os2\uniaud32\drv32\bin\Release.ACP\end.obj (end.asm)

 0005:0007B3E0 000000000H XIB                    DATA 32-bit

 0005:0007B3E0 000000006H XI                     DATA 32-bit
	at offset 00000000 00006H bytes from E:\watcom\lib386\os2\clib3r.lib (mbislead.c)

 0005:0007B3E6 000000000H XIE                    DATA 32-bit

 0005:0007B3E6 000000000H TIB                    DATA 32-bit

 0005:0007B3E6 000000000H TI                     DATA 32-bit

 0005:0007B3E6 000000000H TIE                    DATA 32-bit

 0005:0007B3E6 000000000H YIB                    DATA 32-bit

 0005:0007B3E6 000000000H YI                     DATA 32-bit

 0005:0007B3E6 000000000H YIE                    DATA 32-bit

 0005:0007B3E6 000000000H DATA                   DATA 32-bit

 0005:0007B3E8 000000000H CONST32                CONST 32-bit

 0005:0007B3E8 000000045H CONST32_RO             CONST 32-bit
	at offset 00000000 00045H bytes from F:\acpi\lib\acpidrv.lib (acpi)

 0005:0007B430 000000004H _NULL                  BEGDATA 32-bit
	at offset 00000000 00004H bytes from E:\watcom\lib386\os2\clib3r.lib (segdefns)

 0005:0007B434 000000000H _AFTERNULL             BEGDATA 32-bit

 0005:0007B440 000010000H STACK                  STACK 32-bit
	at offset 00000000 10000H bytes from E:\watcom\lib386\os2\clib3r.lib (segdefns)


 Origin   Group
 0000:0   FLAT
 0003:0   CGROUP
 0005:0   DGROUP


 Address         Publics by Name
 0003:00083380       ACPIFindPCIDevice
 0003:00008EA5       AddBaseAddress_
 0003:00005223       add_timer_
 0003:0000CD73       add_wait_queue_
 0003:0000CD74       add_wait_queue_exclusive_
 0003:0000974F       alloc_pages_
 0003:000073FC       ALSAToOSSDataType_
 0003:0000747A       ALSAToOSSRateFlags_
 0003:00004C07       ALSA_FreeIrq_
 0003:000035F2       ALSA_IDC
 0003:00004C25       ALSA_Interrupt
 0003:00004B78       ALSA_SetIrq_
 0003:00000524       ALSA_STRATEGY
 0003:0000515F       ALSA_TIMER_
 0005:0000176C       BootCode
 0003:000056CC       cancel_delayed_work_
 0003:000356B2       ca_midi_init_
 0003:00008B4A       CharOut_
 0003:00058A3D       client_init_data_
 0003:0000616C       ConvertVolume_
 0003:0000984E       copy_from_user_
 0003:00083DC5       copy_from_user_toio_
 0003:000097EE       copy_to_user_
 0003:00083D57       copy_to_user_fromio_
 0003:000053B7       create_proc_entry_
 0003:00005529       create_workqueue_
 0003:0000898A       DecLongToASCII_
 0003:00005224       del_timer_
 0003:00005575       destroy_workqueue_
 0005:00001800       DevHelp32
 0001:0000003C       DevHelpInit
 0003:00000010       DevHlp
 0003:00000030       DevHlp_ModifiedDS
 0003:00005404       disable_dma_
 0003:0000AE46       disable_irq_
 0000:00000000  Imp  DOS32FLATDS          (DOSCALLS.370)
 0000:00000000  Imp  DOSCLOSE             (DOSCALLS.59)
 0000:00000000  Imp  DosExit              (DOSCALLS.234)
 0000:00000000  Imp  DOSIODELAYCNT        (DOSCALLS.427)
 0000:00000000  Imp  DOSOPEN              (DOSCALLS.70)
 0000:00000000  Imp  DosQueryCp           (DOSCALLS.291)
 0000:00000000  Imp  DosQueryDBCSEnv      (NLS.6)
 0000:00000000  Imp  DosQuerySysInfo      (DOSCALLS.348)
 0000:00000000  Imp  DOSWRITE             (DOSCALLS.138)
 0000:00000000  Imp  DosWrite             (DOSCALLS.282)
 0003:0008377E       down_
 0003:00083780       down_interruptible_
 0003:000051E7       do_gettimeofday_
 0003:00005403       enable_dma_
 0003:0000AD61       eoi_irq_
 0003:000053FB       fasync_helper_
 0001:00000465       FileName
 0003:0000A0D6       FillCaps_
 0003:00083510       FindAddress
 0003:000054DA       flush_workqueue_
 0001:00000040       fOpen
 0003:00005402       free_dma_
 0003:0000ACFA       free_irq_
 0003:0000962F       free_pages_
 0003:00005751       gcd_
 0003:00008ED9       GetBaseAddress_
 0003:00009D61       GetMaxChannels_
 0003:00009CAC       GetNumberOfCards_
 0003:00009CB2       GetNumberOfPcm_
 0003:000027B9       GetParms_
 0003:00009CD6       GetPcmForChannels_
 0003:000034B0       GetTKSSBase
 0003:0000A2F9       GetUniaudCardInfo_
 0003:0000A670       GetUniaudControlInfo_
 0003:0000A3D5       GetUniaudControlNum_
 0003:0000A508       GetUniaudControls_
 0003:0000A751       GetUniaudControlValueGet_
 0003:0000A836       GetUniaudControlValuePut_
 0003:00009DDD       GetUniaudPcmCaps1_
 0003:0000A128       GetUniaudPcmCaps_
 0001:00000000       help_header
 0002:00000000       help_stub_strategy
 0003:00008A6C       HexLongToASCII_
 0003:0000535B       hweight32_
 0003:000000E0       IDC_
 0003:000559E5       ilog2_
 0003:00083422       InitACPICall
 0001:00000046       InitPktOff
 0001:00000044       InitPktSeg
 0003:0008377C       init_MUTEX_
 0003:0008377D       init_MUTEX_LOCKED_
 0003:0000CD7E       init_waitqueue_entry_
 0003:0000CD72       init_waitqueue_head_
 0003:0000CD7C       interruptible_sleep_on_
 0003:0000CD76       interruptible_sleep_on_timeout_
 0005:00001804       intSwitchStack
 0003:0000AE40       in_interrupt_
 0003:000034F0       iodelay32_
 0003:0003373B       ioport_map_
 0003:0003374B       ioport_unmap_
 0003:000336CD       ioread16_
 0003:000336EA       ioread32_
 0003:000336B2       ioread8_
 0003:000097AC       iounmap_
 0003:00033713       iowrite16_
 0003:00033728       iowrite32_
 0003:00033700       iowrite8_
 0003:000097BF       is_access_ok_
 0003:0008FCA0       itoa_
 0003:00009AC8       kcalloc_
 0000:00000000  Imp  KernLinToPageList    (KEE.64)
 0000:00000000  Imp  KernSelToFlat        (KEE.66)
 0000:00000000  Imp  KernThunkStackTo16   (KEE.40)
 0000:00000000  Imp  KernThunkStackTo32   (KEE.41)
 0000:00000000  Imp  KernVMAlloc          (KEE.60)
 0000:00000000  Imp  KernVMFree           (KEE.61)
 0000:00000000  Imp  KernVMLock           (KEE.62)
 0003:000053FE       kill_fasync_
 0003:0000557A       kstrdup_
 0003:000099D4       kzalloc_
 0003:0008FC20       lltoa_
 0003:0008FB80       ltoa_
 0003:0008FA50       mbtowc_
 0003:000051BE       mdelay_
 0003:00005689       memdup_user_
 0003:0008D8C0       memmove_
 0003:0008D8A0       memset_
 0003:000055B5       mod_firmware_load_
 0003:00005227       mod_timer_
 0003:00005228       msleep_
 0003:00005AE3       MyDevBlock_
 0002:00000388       MY_DEVHELP_ATTACHDD
 0003:00004C73       os2gettimemsec_
 0003:00004C6D       os2gettimesec_
 0003:0000C759       OSS32_APMResume_
 0003:0000C79E       OSS32_APMSuspend_
 0003:00005AA8       OSS32_CloseUNI16_
 0003:00005B12       OSS32_DebugString_
 0003:000057FC       OSS32_Initialize_
 0003:00005EA6       OSS32_MidiClose_
 0003:00006045       OSS32_MidiCommand_
 0003:00005B39       OSS32_MidiOpen_
 0003:00006021       OSS32_MidiQueryCaps_
 0003:00005FD2       OSS32_MidiRead_
 0003:00005FCC       OSS32_MidiWrite_
 0003:0000668B       OSS32_MixClose_
 0003:00006D7D       OSS32_MixGetProperty_
 0003:000066E1       OSS32_MixGetVolume_
 0003:00006190       OSS32_MixOpen_
 0003:00006E80       OSS32_MixQueryCaps_
 0003:00006F15       OSS32_MixQueryName_
 0003:00006A50       OSS32_MixSetProperty_
 0003:0000673C       OSS32_MixSetVolume_
 0003:00005A33       OSS32_ProcessIRQ_
 0003:00005A6E       OSS32_ProcessMIDIIRQ_
 0003:00007550       OSS32_QueryDevCaps_
 0003:00007007       OSS32_QueryNames_
 0003:000052CF       OSS32_SetFileId_
 0003:000059A0       OSS32_Shutdown_
 0003:0000857B       OSS32_WaveAddBuffer_
 0003:00007A87       OSS32_WaveClose_
 0003:00008868       OSS32_WaveGetHwPtr_
 0003:0000879C       OSS32_WaveGetPosition_
 0003:00008802       OSS32_WaveGetSpace_
 0003:000088CE       OSS32_WaveGetStatus_
 0003:000078C1       OSS32_WaveOpen_
 0003:00007C64       OSS32_WavePause_
 0003:00007B55       OSS32_WavePrepare_
 0003:00007CBA       OSS32_WaveResume_
 0003:00007D13       OSS32_WaveSetHwParams_
 0003:00008929       OSS32_WaveSetVolume_
 0003:00007BB8       OSS32_WaveStart_
 0003:00007C0E       OSS32_WaveStop_
 0003:00006D9C       OSSToALSAVolume_
 0003:0000B51E       pcibios_present_
 0003:0000AFBC       pcidev_activate_
 0003:0000AFC2       pcidev_deactivate_
 0003:0000AFB6       pcidev_prepare_
 0003:0000B9A6       pci_alloc_consistent_
 0003:0000BBD7       pci_disable_device_
 0003:0000B549       pci_dma_supported_
 0003:0000B761       pci_enable_device_
 0003:0000B55E       pci_find_capability_
 0003:0000B3BC       pci_find_device_
 0003:0000B535       pci_find_slot_
 0003:0000BA62       pci_free_consistent_
 0003:0000BA88       pci_get_dma_mask_
 0003:0000BA7D       pci_get_driver_data_
 0003:0000B4F8       pci_get_flags_
 0003:0003374C       pci_iomap_
 0003:000338D7       pci_iounmap_
 0003:0000C64D       pci_match_device_
 0003:0000B8B2       pci_module_init_
 0003:0000BAD5       pci_orig_restore_state_
 0003:0000BAA9       pci_orig_save_state_
 0003:0000AE47       pci_read_config_byte_
 0003:0000AEC9       pci_read_config_dword_
 0003:0000AE87       pci_read_config_word_
 0003:0000B79F       pci_register_driver_
 0003:0000C633       pci_release_regions_
 0003:0000C2C9       pci_release_region_
 0003:0000C5F8       pci_request_regions_
 0003:0000BC13       pci_request_region_
 0003:0000BB83       pci_restore_state_
 0003:0000BB38       pci_save_state_
 0003:0000BA72       pci_set_driver_data_
 0003:0000BA96       pci_set_latency_time_
 0003:0000B951       pci_set_master_
 0003:0000B5ED       pci_set_power_state_
 0003:0000B8C1       pci_unregister_driver_
 0003:0000AF00       pci_write_config_byte_
 0003:0000AF81       pci_write_config_dword_
 0003:0000AF40       pci_write_config_word_
 0003:00014D7F       pcm_info_
 0003:00014E1B       pcm_instances_
 0005:0000178C       PDDName
 0001:0000045E       pddname16
 0003:00008FD8       phys_to_virt_
 0003:0000B98D       pm_register_
 0003:0000B990       pm_unregister_
 0003:00005357       poll_wait_
 0003:0000AD6E       process_interrupt_
 0003:000053F5       proc_register_
 0003:000053F8       proc_unregister_
 0003:000516DD       query_amp_caps_
 0003:000578F3       queueptr_
 0003:00005709       queue_delayed_work_
 0003:00005446       queue_work_
 0003:0000717C       register_chrdev_
 0003:00005405       register_reboot_notifier_
 0003:0000724C       register_sound_dsp_
 0003:00007217       register_sound_midi_
 0003:000071E2       register_sound_mixer_
 0003:000071AD       register_sound_special_
 0003:0000727E       register_sound_synth_
 0003:00083CE6       release_and_free_resource_
 0003:00005671       release_firmware_
 0003:0000BA93       release_resource_
 0003:00009752       remap_page_range_
 0003:000053F4       remove_proc_entry_
 0003:0000CD75       remove_wait_queue_
 0003:000053FF       request_dma_
 0003:000055F2       request_firmware_
 0003:0000ABFD       request_irq_
 0005:00001790       RMAllocResource1632
 0005:000017A8       RMCreateAdapter1632
 0005:000017A0       RMCreateDevice1632
 0005:000017B0       RMCreateDriver1632
 0005:00001798       RMDeallocResource1632
 0005:000017B8       RMDestroyDriver1632
 0005:000017C8       RMDevIDToHandleList1632
 0003:000047F8       RMDone_
 0005:000017C0       RMGetNodeInfo1632
 0005:000017D0       RMHandleToResourceHandleList1632
 0003:00004477       RMInit_
 0003:000045EE       RMRequestIO_
 0003:00004727       RMRequestIRQ_
 0003:00004692       RMRequestMem_
 0003:00005356       schedule_
 0003:0000519B       schedule_timeout_
 0003:000056EE       schedule_work_
 0003:00009CB7       SetPCMInstance_
 0003:0008A435       snd_ac97_bus_
 0003:0008C8F5       snd_ac97_bus_proc_done_
 0003:0008C89A       snd_ac97_bus_proc_init_
 0003:0008A1BF       snd_ac97_get_name_
 0003:0008A352       snd_ac97_get_short_name_
 0003:0008A4B8       snd_ac97_mixer_
 0003:000843F9       snd_ac97_pcm_assign_
 0003:00084A00       snd_ac97_pcm_close_
 0003:00084AC8       snd_ac97_pcm_double_rate_rules_
 0003:00084774       snd_ac97_pcm_open_
 0003:0008C877       snd_ac97_proc_done_
 0003:0008C793       snd_ac97_proc_init_
 0003:00088068       snd_ac97_read_
 0003:0008B039       snd_ac97_resume_
 0003:0008403B       snd_ac97_set_rate_
 0003:0008AF36       snd_ac97_suspend_
 0003:0008B7A4       snd_ac97_tune_hardware_
 0003:00088138       snd_ac97_update_
 0003:000881B8       snd_ac97_update_bits_
 0003:00088202       snd_ac97_update_bits_nolock_
 0003:0008800B       snd_ac97_write_
 0003:000880E2       snd_ac97_write_cache_
 0003:000150C8       snd_add_device_sysfs_file_
 0003:000543C8       snd_array_free_
 0003:0005434A       snd_array_new_
 0003:00033A41       snd_ca0106_i2c_write_
 0003:000360AB       snd_ca0106_mixer_
 0003:00036283       snd_ca0106_mixer_resume_
 0003:0003624A       snd_ca0106_mixer_suspend_
 0003:00036AD6       snd_ca0106_proc_init_
 0003:000338FB       snd_ca0106_ptr_read_
 0003:00033935       snd_ca0106_ptr_write_
 0003:0003396F       snd_ca0106_spi_write_
 0003:0001C506       snd_card_create_
 0003:0001C842       snd_card_disconnect_
 0003:0001CF13       snd_card_file_add_
 0003:0001CF87       snd_card_file_remove_
 0003:0001CA41       snd_card_free_
 0003:0001C9F1       snd_card_free_when_closed_
 0003:0001CE36       snd_card_info_done_
 0003:0001CDB8       snd_card_info_init_
 0003:0001CD2F       snd_card_info_read_oss_
 0003:0001C76B       snd_card_locked_
 0003:00015E3B       snd_card_proc_new_
 0003:0001CC51       snd_card_register_
 0003:0001CC2B       snd_card_set_id_
 0003:0001CE4D       snd_component_add_
 0003:000619D3       snd_cs46xx_create_
 0003:0005FC7F       snd_cs46xx_download_
 0003:0005FCB8       snd_cs46xx_download_image_
 0003:00061173       snd_cs46xx_gameport_
 0003:000610BC       snd_cs46xx_midi_
 0003:00060CB5       snd_cs46xx_mixer_
 0003:00060A42       snd_cs46xx_pcm_
 0003:00061899       snd_cs46xx_resume_
 0003:00061547       snd_cs46xx_start_dsp_
 0003:000617DA       snd_cs46xx_suspend_
 0003:00062979       snd_cs5535audio_pcm_
 0003:0006243B       snd_cs5535audio_resume_
 0003:00062397       snd_cs5535audio_suspend_
 0003:0001AB08       snd_ctl_add_
 0003:0001C088       snd_ctl_boolean_mono_info_
 0003:0001C0A7       snd_ctl_boolean_stereo_info_
 0003:0001C070       snd_ctl_create_
 0003:0001ADCC       snd_ctl_find_id_
 0003:0001AD9F       snd_ctl_find_numid_
 0003:0001AA3F       snd_ctl_free_one_
 0003:00083C24       snd_ctl_make_virtual_master_
 0003:0001A96E       snd_ctl_new1_
 0003:0001A80C       snd_ctl_notify_
 0003:0001BF0A       snd_ctl_register_ioctl_
 0003:0001AC1B       snd_ctl_remove_
 0003:0001AC86       snd_ctl_remove_id_
 0003:0001AD43       snd_ctl_rename_id_
 0003:0001BF64       snd_ctl_unregister_ioctl_
 0003:0001A465       snd_device_disconnect_
 0003:0001A567       snd_device_disconnect_all_
 0003:0001A3CE       snd_device_free_
 0003:0001A59F       snd_device_free_all_
 0003:0001A37B       snd_device_new_
 0003:0001A4CF       snd_device_register_
 0003:0001A529       snd_device_register_all_
 0003:0001C1AE       snd_dma_alloc_pages_
 0003:0001C23D       snd_dma_alloc_pages_fallback_
 0003:0001C29D       snd_dma_free_pages_
 0003:0001C2F0       snd_dma_get_reserved_buf_
 0003:0001C3A1       snd_dma_reserve_buf_
 0003:00072DD2       snd_emu1010_fpga_link_dst_src_write_
 0003:00072D5B       snd_emu1010_fpga_read_
 0003:00072CD0       snd_emu1010_fpga_write_
 0003:00073219       snd_emu10k1_ac97_read_
 0003:0007325B       snd_emu10k1_ac97_write_
 0003:000738C9       snd_emu10k1_alloc_pages_
 0003:0006FE85       snd_emu10k1_audigy_midi_
 0003:000715D6       snd_emu10k1_create_
 0003:0007068F       snd_emu10k1_done_
 0003:0006AE3E       snd_emu10k1_efx_alloc_pm_buffer_
 0003:0006AEE5       snd_emu10k1_efx_free_pm_buffer_
 0003:0006412C       snd_emu10k1_efx_read_
 0003:0006B039       snd_emu10k1_efx_resume_
 0003:0006AF16       snd_emu10k1_efx_suspend_
 0003:0006A5C9       snd_emu10k1_free_efx_
 0003:000739BA       snd_emu10k1_free_pages_
 0003:0006AD8D       snd_emu10k1_fx8010_new_
 0003:00063F32       snd_emu10k1_fx8010_register_irq_handler_
 0003:0006A603       snd_emu10k1_fx8010_tram_setup_
 0003:00063FD3       snd_emu10k1_fx8010_unregister_irq_handler_
 0003:00072BC5       snd_emu10k1_i2c_write_
 0003:0006A591       snd_emu10k1_init_efx_
 0003:00073D66       snd_emu10k1_interrupt_
 0003:00072E5F       snd_emu10k1_intr_disable_
 0003:00072E26       snd_emu10k1_intr_enable_
 0003:00073829       snd_emu10k1_memblk_map_
 0003:0006FE38       snd_emu10k1_midi_
 0003:0006C7D8       snd_emu10k1_mixer_
 0003:0006ED90       snd_emu10k1_pcm_
 0003:0006F729       snd_emu10k1_pcm_efx_
 0003:0006EF8D       snd_emu10k1_pcm_mic_
 0003:0006EEB0       snd_emu10k1_pcm_multi_
 0003:00072698       snd_emu10k1_proc_init_
 0003:00072A4F       snd_emu10k1_ptr20_read_
 0003:00072A8F       snd_emu10k1_ptr20_write_
 0003:000728BF       snd_emu10k1_ptr_read_
 0003:0007297B       snd_emu10k1_ptr_write_
 0003:0007329D       snd_emu10k1_rate_to_pitch_
 0003:00071C61       snd_emu10k1_resume_init_
 0003:00071CC5       snd_emu10k1_resume_regs_
 0003:00072ACF       snd_emu10k1_spi_write_
 0003:00071BD2       snd_emu10k1_suspend_regs_
 0003:000739BF       snd_emu10k1_synth_alloc_
 0003:00073C64       snd_emu10k1_synth_bzero_
 0003:00073CD8       snd_emu10k1_synth_copy_from_user_
 0003:00073A1F       snd_emu10k1_synth_free_
 0003:00063BB1       snd_emu10k1_timer_
 0003:00073479       snd_emu10k1_voice_alloc_
 0003:00073157       snd_emu10k1_voice_clear_loop_stop_
 0003:00073507       snd_emu10k1_voice_free_
 0003:00073092       snd_emu10k1_voice_half_loop_intr_ack_
 0003:0007302B       snd_emu10k1_voice_half_loop_intr_disable_
 0003:00072FC6       snd_emu10k1_voice_half_loop_intr_enable_
 0003:0006FF1D       snd_emu10k1_voice_init_
 0003:00072F66       snd_emu10k1_voice_intr_ack_
 0003:00072EFF       snd_emu10k1_voice_intr_disable_
 0003:00072E9A       snd_emu10k1_voice_intr_enable_
 0003:000730F2       snd_emu10k1_voice_set_loop_stop_
 0003:000731BE       snd_emu10k1_wait_
 0003:0001C179       snd_free_dev_pages_
 0003:0001C112       snd_free_pages_
 0003:0001D0FA       snd_free_sgbuf_pages_
 0003:0005060A       snd_hda_add_codec_preset_
 0003:000535E7       snd_hda_add_new_ctls_
 0003:00051F1F       snd_hda_add_nid_
 0003:00051030       snd_hda_add_pincfg_
 0003:00052159       snd_hda_add_vmaster_
 0003:00052E20       snd_hda_build_controls_
 0003:000534FF       snd_hda_build_pcms_
 0003:00050BA5       snd_hda_bus_new_
 0003:00053883       snd_hda_bus_reboot_notify_
 0003:00052EB1       snd_hda_calc_stream_format_
 0003:000535A1       snd_hda_check_board_codec_sid_config_
 0003:00053526       snd_hda_check_board_config_
 0003:0005368B       snd_hda_ch_mode_get_
 0003:00053654       snd_hda_ch_mode_info_
 0003:000536AF       snd_hda_ch_mode_put_
 0003:00051936       snd_hda_codec_amp_read_
 0003:00051A1D       snd_hda_codec_amp_stereo_
 0003:00051976       snd_hda_codec_amp_update_
 0003:00052E7D       snd_hda_codec_build_controls_
 0003:0005344C       snd_hda_codec_build_pcms_
 0003:000515F0       snd_hda_codec_cleanup_stream_
 0003:000514E5       snd_hda_codec_configure_
 0003:000510D1       snd_hda_codec_get_pincfg_
 0003:0005125C       snd_hda_codec_new_
 0003:00056C7B       snd_hda_codec_proc_new_
 0003:000507D8       snd_hda_codec_read_
 0003:00052000       snd_hda_codec_reset_
 0003:00051A68       snd_hda_codec_resume_amp_
 0003:00052BD7       snd_hda_codec_resume_cache_
 0003:000515AA       snd_hda_codec_setup_stream_
 0003:000510BC       snd_hda_codec_set_pincfg_
 0003:00052B61       snd_hda_codec_update_cache_
 0003:00050805       snd_hda_codec_write_
 0003:00052AEB       snd_hda_codec_write_cache_
 0003:00054622       snd_hda_create_hwdep_
 0003:00052A45       snd_hda_create_spdif_in_ctls_
 0003:0005286E       snd_hda_create_spdif_out_ctls_
 0003:00052954       snd_hda_create_spdif_share_sw_
 0003:00051F60       snd_hda_ctls_clear_
 0003:00051EB2       snd_hda_ctl_add_
 0003:0005063A       snd_hda_delete_codec_preset_
 0003:00051EA8       snd_hda_find_mixer_ctl_
 0003:000508A3       snd_hda_get_connections_
 0003:000506AB       snd_hda_get_jack_connectivity_
 0003:00050662       snd_hda_get_jack_location_
 0003:000506B9       snd_hda_get_jack_type_
 0003:0005086B       snd_hda_get_sub_nodes_
 0003:000536F8       snd_hda_input_mux_info_
 0003:00053747       snd_hda_input_mux_put_
 0003:00053204       snd_hda_is_supported_format_
 0003:0005183C       snd_hda_jack_detect_
 0003:00052215       snd_hda_mixer_amp_switch_get_
 0003:000521E5       snd_hda_mixer_amp_switch_info_
 0003:000522AC       snd_hda_mixer_amp_switch_put_
 0003:00051D49       snd_hda_mixer_amp_tlv_
 0003:00051C00       snd_hda_mixer_amp_volume_get_
 0003:00051B1B       snd_hda_mixer_amp_volume_info_
 0003:00051C9A       snd_hda_mixer_amp_volume_put_
 0003:0005247B       snd_hda_mixer_bind_ctls_get_
 0003:00052443       snd_hda_mixer_bind_ctls_info_
 0003:000524B4       snd_hda_mixer_bind_ctls_put_
 0003:00052367       snd_hda_mixer_bind_switch_get_
 0003:000523A2       snd_hda_mixer_bind_switch_put_
 0003:00052522       snd_hda_mixer_bind_tlv_
 0003:00053C16       snd_hda_multi_out_analog_cleanup_
 0003:00053966       snd_hda_multi_out_analog_open_
 0003:00053A7A       snd_hda_multi_out_analog_prepare_
 0003:00053916       snd_hda_multi_out_dig_cleanup_
 0003:00053944       snd_hda_multi_out_dig_close_
 0003:000538AC       snd_hda_multi_out_dig_open_
 0003:000538E6       snd_hda_multi_out_dig_prepare_
 0003:0005174E       snd_hda_override_amp_caps_
 0003:00055939       snd_hda_parse_generic_codec_
 0003:00053D59       snd_hda_parse_pin_def_config_
 0003:000517E6       snd_hda_pin_sense_
 0003:000517CB       snd_hda_query_pin_caps_
 0003:00050AC2       snd_hda_queue_unsol_event_
 0003:00054327       snd_hda_resume_
 0003:0005083E       snd_hda_sequence_write_
 0003:00052C24       snd_hda_sequence_write_cache_
 0003:00051E0C       snd_hda_set_vmaster_tlv_
 0003:00051162       snd_hda_shutup_pins_
 0003:00054304       snd_hda_suspend_
 0003:0000D35D       snd_hwdep_new_
 0003:00015AF8       snd_info_card_create_
 0003:00015BB2       snd_info_card_disconnect_
 0003:00015C06       snd_info_card_free_
 0003:00015B73       snd_info_card_id_change_
 0003:00015B5A       snd_info_card_register_
 0003:000152C2       snd_info_check_reserved_words_
 0003:00015DAA       snd_info_create_card_entry_
 0003:00015D90       snd_info_create_module_entry_
 0003:00015AAA       snd_info_done_
 0003:00015E93       snd_info_free_entry_
 0003:00015C26       snd_info_get_line_
 0003:00015CB1       snd_info_get_str_
 0003:00015A0E       snd_info_init_
 0003:00019FDD       snd_info_minor_register_
 0003:0001A031       snd_info_minor_unregister_
 0003:00015ED6       snd_info_register_
 0003:0001279D       snd_interval_div_
 0003:00012E3C       snd_interval_list_
 0003:00012856       snd_interval_muldivk_
 0003:00012905       snd_interval_mulkdiv_
 0003:000126FF       snd_interval_mul_
 0003:000129C7       snd_interval_ratnum_
 0003:000125A9       snd_interval_refine_
 0003:00008CD3       snd_iprintf_
 0003:00014E81       snd_lookup_minor_data_
 0003:0001A043       snd_lookup_oss_minor_data_
 0003:0001C13C       snd_malloc_dev_pages_
 0003:0001C0E6       snd_malloc_pages_
 0003:0001D140       snd_malloc_sgbuf_pages_
 0003:0008D399       snd_midi_channel_alloc_set_
 0003:0008D3F0       snd_midi_channel_free_set_
 0003:0008CEF1       snd_midi_channel_set_clear_
 0003:0008C909       snd_midi_process_event_
 0003:00015203       snd_minor_info_done_
 0003:000151C2       snd_minor_info_init_
 0003:0001A363       snd_minor_info_oss_done_
 0003:0001A320       snd_minor_info_oss_init_
 0003:0005EDAF       snd_mpu401_uart_interrupt_
 0003:0005EDC1       snd_mpu401_uart_interrupt_tx_
 0003:0005F343       snd_mpu401_uart_new_
 0003:0005D8EF       snd_opl3_calc_volume_
 0003:0005E8BD       snd_opl3_clear_patches_
 0003:0005E472       snd_opl3_control_
 0003:0005D2C5       snd_opl3_create_
 0003:0005D842       snd_opl3_drum_switch_
 0003:0005E848       snd_opl3_find_patch_
 0003:0005D44B       snd_opl3_hwdep_new_
 0003:0005D254       snd_opl3_init_
 0003:0005D15E       snd_opl3_interrupt_
 0003:0005E4DE       snd_opl3_ioctl_
 0003:0005E343       snd_opl3_key_press_
 0003:0005D7D1       snd_opl3_load_drums_
 0003:0005E75E       snd_opl3_load_patch_
 0003:0005D1D1       snd_opl3_new_
 0003:0005E313       snd_opl3_note_off_
 0003:0005DC40       snd_opl3_note_on_
 0003:0005E4D7       snd_opl3_nrpn_
 0003:0005E4DB       snd_opl3_open_
 0003:0005E65A       snd_opl3_release_
 0003:0005E8FB       snd_opl3_reset_
 0003:0005CA38       snd_opl3_synth_cleanup_
 0003:0005C98E       snd_opl3_synth_setup_
 0003:0005C98D       snd_opl3_synth_use_dec_
 0003:0005C971       snd_opl3_synth_use_inc_
 0003:0005E4D8       snd_opl3_sysex_
 0003:0005E344       snd_opl3_terminate_note_
 0003:0005DB38       snd_opl3_timer_func_
 0003:0005D40E       snd_opl3_timer_new_
 0003:0005E668       snd_opl3_write_
 0003:00019E37       snd_oss_info_register_
 0003:00063A75       snd_p16v_alloc_pm_buffer_
 0003:00063650       snd_p16v_free_
 0003:00063A97       snd_p16v_free_pm_buffer_
 0003:00063A36       snd_p16v_mixer_
 0003:00063661       snd_p16v_pcm_
 0003:00063AD4       snd_p16v_resume_
 0003:00063AA2       snd_p16v_suspend_
 0003:0000C74C       snd_pci_compat_get_pci_driver_
 0003:0000C6F1       snd_pci_dev_present_
 0003:00083D3A       snd_pci_quirk_lookup_
 0003:00083CFB       snd_pci_quirk_lookup_id_
 0003:00014759       snd_pcm_attach_substream_
 0003:000149CA       snd_pcm_detach_substream_
 0003:000179A8       snd_pcm_drain_done_
 0003:000118D7       snd_pcm_format_big_endian_
 0003:0001189F       snd_pcm_format_linear_
 0003:000118AF       snd_pcm_format_little_endian_
 0003:000144B2       snd_pcm_format_name_
 0003:00011912       snd_pcm_format_physical_width_
 0003:0001197B       snd_pcm_format_set_silence_
 0003:00011864       snd_pcm_format_signed_
 0003:00011950       snd_pcm_format_silence_64_
 0003:0001193A       snd_pcm_format_size_
 0003:0001188C       snd_pcm_format_unsigned_
 0003:000118EA       snd_pcm_format_width_
 0003:00018AC9       snd_pcm_hw_constraints_complete_
 0003:00018786       snd_pcm_hw_constraints_init_
 0003:000130C4       snd_pcm_hw_constraint_integer_
 0003:0001314F       snd_pcm_hw_constraint_list_
 0003:00013077       snd_pcm_hw_constraint_mask64_
 0003:0001304A       snd_pcm_hw_constraint_mask_
 0003:000130E3       snd_pcm_hw_constraint_minmax_
 0003:000132AE       snd_pcm_hw_constraint_msbits_
 0003:0001333A       snd_pcm_hw_constraint_pow2_
 0003:00013261       snd_pcm_hw_constraint_ratdens_
 0003:000131D8       snd_pcm_hw_constraint_ratnums_
 0003:000132F3       snd_pcm_hw_constraint_step_
 0003:0001360E       snd_pcm_hw_params_choose_
 0003:0001353A       snd_pcm_hw_param_first_
 0003:000135D7       snd_pcm_hw_param_last_
 0003:000133FC       snd_pcm_hw_param_value_
 0003:00016A37       snd_pcm_hw_refine_
 0003:00012F32       snd_pcm_hw_rule_add_
 0003:0001691A       snd_pcm_info_
 0003:000169DB       snd_pcm_info_user_
 0003:00019C07       snd_pcm_kernel_ioctl_
 0003:00016285       snd_pcm_lib_free_pages_
 0003:0001630B       snd_pcm_lib_free_vmalloc_buffer_
 0003:0001378D       snd_pcm_lib_ioctl_
 0003:000161BA       snd_pcm_lib_malloc_pages_
 0003:00016064       snd_pcm_lib_preallocate_free_
 0003:0001606C       snd_pcm_lib_preallocate_free_for_all_
 0003:000160CE       snd_pcm_lib_preallocate_pages_
 0003:000160E6       snd_pcm_lib_preallocate_pages_for_all_
 0003:000141E0       snd_pcm_lib_readv_
 0003:000140B2       snd_pcm_lib_read_
 0003:00013DCD       snd_pcm_lib_writev_
 0003:00013C62       snd_pcm_lib_write_
 0003:00011AB4       snd_pcm_limit_hw_rates_
 0003:000145E8       snd_pcm_new_
 0003:000144BA       snd_pcm_new_stream_
 0003:00014C24       snd_pcm_notify_
 0003:00018CC9       snd_pcm_open_substream_
 0003:00081561       snd_pcm_oss_read3_
 0003:00081652       snd_pcm_oss_readv3_
 0003:00081502       snd_pcm_oss_write3_
 0003:000815F3       snd_pcm_oss_writev3_
 0003:000137CB       snd_pcm_period_elapsed_
 0003:00011F84       snd_pcm_playback_silence_
 0003:00011B1C       snd_pcm_rate_to_rate_bit_
 0003:00018C60       snd_pcm_release_substream_
 0003:00012482       snd_pcm_set_ops_
 0003:000124A7       snd_pcm_set_sync_
 0003:00016164       snd_pcm_sgbuf_get_chunk_size_
 0003:00016146       snd_pcm_sgbuf_ops_page_
 0003:000178DF       snd_pcm_start_
 0003:000172FB       snd_pcm_status_
 0003:00017997       snd_pcm_stop_
 0003:00017B76       snd_pcm_suspend_
 0003:00017BC7       snd_pcm_suspend_all_
 0003:00016516       snd_pcm_timer_done_
 0003:0001641D       snd_pcm_timer_init_
 0003:00016328       snd_pcm_timer_resolution_change_
 0003:00012478       snd_pcm_update_hw_ptr_
 0003:0001223A       snd_pcm_update_state_
 0003:0001D03A       snd_power_wait_
 0003:00054444       snd_print_pcm_bits_
 0003:000543E9       snd_print_pcm_rates_
 0003:0000FDFB       snd_rawmidi_drain_input_
 0003:0000FD87       snd_rawmidi_drain_output_
 0003:0000FD45       snd_rawmidi_drop_output_
 0003:00010508       snd_rawmidi_info_select_
 0003:000106AE       snd_rawmidi_input_params_
 0003:0000FFE0       snd_rawmidi_kernel_open_
 0003:00010A96       snd_rawmidi_kernel_read_
 0003:000103F8       snd_rawmidi_kernel_release_
 0003:00010EFB       snd_rawmidi_kernel_write_
 0003:000112C7       snd_rawmidi_new_
 0003:0001060A       snd_rawmidi_output_params_
 0003:000107F8       snd_rawmidi_receive_
 0003:000117B0       snd_rawmidi_set_ops_
 0003:00010D7E       snd_rawmidi_transmit_
 0003:00010D03       snd_rawmidi_transmit_ack_
 0003:00010BDC       snd_rawmidi_transmit_empty_
 0003:00010C25       snd_rawmidi_transmit_peek_
 0003:00014F8B       snd_register_device_for_dev_
 0003:0001A11E       snd_register_oss_device_
 0003:0007F787       snd_sbdsp_command_
 0003:0007FA1A       snd_sbdsp_create_
 0003:0007F7DA       snd_sbdsp_get_byte_
 0003:0007F822       snd_sbdsp_reset_
 0003:0007F3B5       snd_sbmixer_add_ctl_
 0003:0007F4DA       snd_sbmixer_new_
 0003:0007EAD9       snd_sbmixer_read_
 0003:0007F710       snd_sbmixer_resume_
 0003:0007F699       snd_sbmixer_suspend_
 0003:0007EAAE       snd_sbmixer_write_
 0003:0005AE32       snd_sequencer_device_done_
 0003:0005ADD9       snd_sequencer_device_init_
 0003:000588DD       snd_sequencer_memory_done_
 0003:000588DA       snd_sequencer_memory_init_
 0003:00058387       snd_seq_cell_free_
 0003:00057969       snd_seq_check_queue_
 0003:00059B48       snd_seq_client_notify_subscription_
 0003:000589CA       snd_seq_client_use_ptr_
 0003:00058035       snd_seq_control_queue_
 0003:0005A8A9       snd_seq_create_kernel_client_
 0003:0005AF72       snd_seq_create_port_
 0003:0005B25E       snd_seq_delete_all_ports_
 0003:0005A983       snd_seq_delete_kernel_client_
 0003:0005B1D7       snd_seq_delete_port_
 0003:00056DA7       snd_seq_device_load_drivers_
 0003:00056DA8       snd_seq_device_new_
 0003:00056F79       snd_seq_device_register_driver_
 0003:000570B5       snd_seq_device_unregister_driver_
 0003:000592AD       snd_seq_dispatch_event_
 0003:000581ED       snd_seq_dump_var_event_
 0003:00057A49       snd_seq_enqueue_event_
 0003:000584FA       snd_seq_event_dup_
 0003:0005B94F       snd_seq_event_port_attach_
 0003:0005B9DD       snd_seq_event_port_detach_
 0003:000582DE       snd_seq_expand_var_event_
 0003:0005C80E       snd_seq_fifo_cell_out_
 0003:0005C899       snd_seq_fifo_cell_putback_
 0003:0005C725       snd_seq_fifo_clear_
 0003:0005C6DC       snd_seq_fifo_delete_
 0003:0005C75D       snd_seq_fifo_event_in_
 0003:0005C658       snd_seq_fifo_new_
 0003:0005C8CD       snd_seq_fifo_poll_wait_
 0003:0005C8E8       snd_seq_fifo_resize_
 0003:0005B39C       snd_seq_get_port_info_
 0003:0005ACB7       snd_seq_info_clients_read_
 0003:0005742B       snd_seq_info_done_
 0003:000573EA       snd_seq_info_init_
 0003:000588DE       snd_seq_info_pool_
 0003:0005808A       snd_seq_info_queues_read_
 0003:0005C0E9       snd_seq_info_timer_read_
 0003:0005AA63       snd_seq_kernel_client_ctl_
 0003:0005AA20       snd_seq_kernel_client_dispatch_
 0003:0005A9FF       snd_seq_kernel_client_enqueue_
 0003:0005AA0B       snd_seq_kernel_client_enqueue_blocking_
 0003:0005AA76       snd_seq_kernel_client_write_poll_
 0003:000588BB       snd_seq_pool_delete_
 0003:00058794       snd_seq_pool_done_
 0003:000586F6       snd_seq_pool_init_
 0003:0005884F       snd_seq_pool_new_
 0003:000586D6       snd_seq_pool_poll_wait_
 0003:0005B587       snd_seq_port_connect_
 0003:0005B7EB       snd_seq_port_disconnect_
 0003:0005B90B       snd_seq_port_get_subscription_
 0003:0005AED5       snd_seq_port_query_nearest_
 0003:0005AE77       snd_seq_port_use_ptr_
 0003:0005C3B3       snd_seq_prioq_avail_
 0003:0005C290       snd_seq_prioq_cell_in_
 0003:0005C35C       snd_seq_prioq_cell_out_
 0003:0005C3D1       snd_seq_prioq_cell_peek_
 0003:0005C1E5       snd_seq_prioq_delete_
 0003:0005C431       snd_seq_prioq_leave_
 0003:0005C19B       snd_seq_prioq_new_
 0003:0005C5A9       snd_seq_prioq_remove_events_
 0003:0005786B       snd_seq_queues_delete_
 0003:00057868       snd_seq_queues_init_
 0003:0005788B       snd_seq_queue_alloc_
 0003:00057B42       snd_seq_queue_check_access_
 0003:00057DB6       snd_seq_queue_client_leave_
 0003:00057E45       snd_seq_queue_client_leave_cells_
 0003:00057D53       snd_seq_queue_client_termination_
 0003:000578CA       snd_seq_queue_delete_
 0003:0005792C       snd_seq_queue_find_name_
 0003:000576AE       snd_seq_queue_get_cur_queues_
 0003:00057D1F       snd_seq_queue_is_used_
 0003:00057E83       snd_seq_queue_remove_cells_
 0003:00057B7C       snd_seq_queue_set_owner_
 0003:00057C06       snd_seq_queue_timer_close_
 0003:00057BCB       snd_seq_queue_timer_open_
 0003:00057C1D       snd_seq_queue_timer_set_tempo_
 0003:00057C8B       snd_seq_queue_use_
 0003:0005B311       snd_seq_set_port_info_
 0003:0005A0EB       snd_seq_set_queue_tempo_
 0003:000574A4       snd_seq_system_broadcast_
 0003:0005763C       snd_seq_system_client_done_
 0003:00057512       snd_seq_system_client_init_
 0003:000574D1       snd_seq_system_notify_
 0003:0005BEED       snd_seq_timer_close_
 0003:0005C004       snd_seq_timer_continue_
 0003:0005BB83       snd_seq_timer_defaults_
 0003:0005BB4A       snd_seq_timer_delete_
 0003:0005C0E5       snd_seq_timer_get_cur_tick_
 0003:0005C055       snd_seq_timer_get_cur_time_
 0003:0005BB06       snd_seq_timer_new_
 0003:0005BDF1       snd_seq_timer_open_
 0003:0005BBE2       snd_seq_timer_reset_
 0003:0005BD41       snd_seq_timer_set_position_tick_
 0003:0005BD71       snd_seq_timer_set_position_time_
 0003:0005BCE0       snd_seq_timer_set_ppq_
 0003:0005BDAB       snd_seq_timer_set_skew_
 0003:0005BCA3       snd_seq_timer_set_tempo_
 0003:0005BFBB       snd_seq_timer_start_
 0003:0005BF10       snd_seq_timer_stop_
 0003:0000DA3E       snd_timer_close_
 0003:0000DF13       snd_timer_continue_
 0003:0000E6C8       snd_timer_global_free_
 0003:0000E693       snd_timer_global_new_
 0003:0000E6CD       snd_timer_global_register_
 0003:0000E0A1       snd_timer_interrupt_
 0003:0000E2E9       snd_timer_new_
 0003:0000E59D       snd_timer_notify_
 0003:0000D8E8       snd_timer_open_
 0003:0000DF8D       snd_timer_pause_
 0003:0000DB96       snd_timer_resolution_
 0003:0000DD71       snd_timer_start_
 0003:0000DECD       snd_timer_stop_
 0003:0007D4C0       snd_trident_alloc_pages_
 0003:0007CEEF       snd_trident_alloc_voice_
 0003:0007C9BA       snd_trident_create_
 0003:0007C388       snd_trident_create_gameport_
 0003:0007B43E       snd_trident_foldback_pcm_
 0003:0007D4CF       snd_trident_free_pages_
 0003:0007CF9F       snd_trident_free_voice_
 0003:0007B2E8       snd_trident_pcm_
 0003:0007D15E       snd_trident_resume_
 0003:0007B5E1       snd_trident_spdif_pcm_
 0003:00079BA4       snd_trident_start_voice_
 0003:00079BCF       snd_trident_stop_voice_
 0003:0007D0DC       snd_trident_suspend_
 0003:00079CE0       snd_trident_write_voice_regs_
 0003:00015079       snd_unregister_device_
 0003:0001A1A9       snd_unregister_oss_device_
 0003:0008D44A       snd_util_memhdr_free_
 0003:0008D417       snd_util_memhdr_new_
 0003:0008D528       snd_util_mem_alloc_
 0003:0008D58D       snd_util_mem_avail_
 0003:0008D56C       snd_util_mem_free_
 0003:000772BA       snd_ymfpci_create_
 0003:00074183       snd_ymfpci_free_gameport_
 0003:0007673D       snd_ymfpci_mixer_
 0003:00075D21       snd_ymfpci_pcm2_
 0003:00075C50       snd_ymfpci_pcm_
 0003:00075E9A       snd_ymfpci_pcm_4ch_
 0003:00075DDB       snd_ymfpci_pcm_spdif_
 0003:000771D0       snd_ymfpci_resume_
 0003:00077107       snd_ymfpci_suspend_
 0003:000769F8       snd_ymfpci_timer_
 0003:0008D870       snprintf_
 0003:0000CD89       spin_lock_
 0003:0000CD93       spin_lock_flag_
 0003:0000CD82       spin_lock_init_
 0003:0000CD9D       spin_trylock_
 0003:0000CDA0       spin_unlock_
 0003:00005139       sprintf_
 0003:0008D7A0       sscanf_
 0005:0000177C       stackbase
 0005:00001780       stacksel
 0003:00000080       STRATEGY_
 0003:0000525A       strcmp_
 0003:0000576A       strict_strtoul_
 0003:00008B8C       StringOut_
 0003:0008D6E0       strlcpy_
 0003:000834C0       StrLen
 0003:000834E0       StrNCmp
 0003:0000527D       strncmp_
 0003:0000CD4D       strncpy_
 0003:0008D630       strstr_
 0003:0008DB50       strtol_
 0003:0008DB40       strtoul_
 0003:0008F880       strupr_
 0003:000052A6       tasklet_hi_schedule_
 0003:000052BB       tasklet_init_
 0003:00000024       thunk1632_devhelp
 0003:00000044       thunk1632_devhelp_modified_ds
 0002:000001A0       thunk3216_devhelp
 0002:000001B2       thunk3216_devhelp_modified_ds
 0003:00000140       TIMER_
 0003:0008F820       tolower_
 0003:0008FBB0       ulltoa_
 0003:0008FB30       ultoa_
 0003:0000AB72       UniaudCloseAll_
 0003:0000A171       UniaudCtlGetPowerState_
 0003:0000A235       UniaudCtlSetPowerState_
 0003:0000A96B       UniaudIoctlHWParamSet_
 0003:0000A91B       UniaudIoctlHWRefine_
 0003:0000AB41       UniaudIoctlPCMDrop_
 0003:0000AAAC       UniaudIoctlPCMPrepare_
 0003:0000AA7C       UniaudIoctlPCMRead_
 0003:0000AADD       UniaudIoctlPCMResume_
 0003:0000AB10       UniaudIoctlPCMStart_
 0003:0000AA0B       UniaudIoctlPCMStatus_
 0003:0000AA4C       UniaudIoctlPCMWrite_
 0003:0000A9BB       UniaudIoctlSWParamSet_
 0001:0000001E       uniaud_header
 0003:00009B5C       uniaud_set_interrupted_substream_
 0002:0000010A       uniaud_stub_idc
 0002:00000096       uniaud_stub_strategy
 0002:00000128       uniaud_stub_timer
 0003:00007321       UNIXToOSSError_
 0003:00007195       unregister_chrdev_
 0003:00005408       unregister_reboot_notifier_
 0003:000072F5       unregister_sound_dsp_
 0003:000072DF       unregister_sound_midi_
 0003:000072C9       unregister_sound_mixer_
 0003:000072B3       unregister_sound_special_
 0003:0000730B       unregister_sound_synth_
 0003:0008377F       up_
 0003:0008FC50       utoa_
 0003:0000971E       vfree_
 0003:00008FAA       virt_to_phys_
 0003:0000965C       vmalloc_
 0003:00009014       VMAlloc_
 0003:0000907A       VMFree_
 0003:0008D810       vsnprintf_
 0003:00004E8A       vsprintf_
 0003:0008D770       vsscanf_
 0003:00004C61       W?$dln(pnv)v
 0003:00004C5C       W?$nwn(ui)pnv
 0003:00004C66       W?$nwn(uipnv)pnv
 0005:0000056C       W?acHeap$npnuc
 0003:000057C7       W?CallOSS16$n(ululul)ul
 0003:0000167A       W?CheckCardName$n(pfa)v
 0003:0000CA6A       W?compact$n()v
 0005:00000030       W?deviceOwner$nul
 0003:0000064F       W?DevSaveMessage$n(pfai)v
 0003:00000771       W?DiscardableInit$n(pf$RPInit$$)ul
 0003:000018B1       W?DoParm$n(apfa)i
 0003:0000C7ED       W?dumpheap$n()v
 0005:000000EC       W?fnCardExitCall$n[]pn()v
 0005:000018A4       W?ForceCard$ni
 0003:0000CB0E       W?free$n(pnv)v
 0003:0000C863       W?HeapCheck$n(pna)v
 0003:0000CCED       W?HeapInit$n(ul)ul
 0003:0000CCCD       W?IsHeapAddr$n(ul)ul
 0003:00001621       W?IsWhitespace$n(a)i
 0003:000006CF       W?LockSegments$n()i
 0003:0000C939       W?malloc$n(ul)pnv
 0003:00001551       W?mymemchr$n(pfaaus)pfa
 0003:0000C8BC       W?npvAllocateBlock$n(pn$_MEMBLOCK$$ulpn$1$)pnv
 0005:00000034       W?numOS2Opens$nul
 0003:00003A26       W?OSS32IDC$n(ulpn$__6ikc0pIDC32_PACKET$$)ul
 0003:00001B8E       W?ParseParm$n(pfai)i
 0005:00000564       W?pmbFree$npn$_MEMBLOCK$$
 0005:00000560       W?pmbUsed$npn$_MEMBLOCK$$
 0003:0000CC5A       W?realloc$n(pnvul)pnv
 0003:0000CA3C       W?remove$n(pn$_MEMBLOCK$$)v
 0005:00000064       W?RMFlags$nul
 0005:00000058       W?RM_Help$npn()i
 0005:0000005C       W?RM_Help0$npn()i
 0005:00000060       W?RM_Help3$npn()i
 0003:0000C81E       W?SignatureCheck$n(pn$_MEMBLOCK$$pna)s
 0003:0000163A       W?SkipWhite$n(pfa)pfa
 0003:00004448       W?StratClose$n(pf$RP$$)ul
 0005:00001810       W?StratDispatch$n[]pn(pf$RP$$)ul
 0003:000004A2       W?StratInit$n(pf$RP$$)ul
 0003:000004A7       W?StratInitComplete$n(pf$RP$$)ul
 0003:00003D37       W?StratIOCtl$n(pf$RP$$)ul
 0003:0000047D       W?StratOpen$n(pf$RP$$)ul
 0003:00000549       W?StratRead$n(pf$RP$$)ul
 0003:0000050A       W?StratShutdown$n(pf$RP$$)ul
 0003:00001589       W?sz2us$n(pfai)us
 0003:00001543       W?toupper$n(i)i
 0005:00000574       W?ulcAlloc$nul
 0005:00000580       W?ulcFree$nul
 0005:0000E8D0       W?ulcTotalHeap$nul
 0005:00000570       W?ulnAlloc$nul
 0005:00000578       W?ulnAllocCalls$nul
 0005:00000588       W?ulnCompact$nul
 0005:0000057C       W?ulnFree$nul
 0005:00000584       W?ulnFreeCalls$nul
 0005:00000568       W?uMemFree$nui
 0003:0000CC48       W?_memfree$n()ui
 0003:0000CC4E       W?_msize$n(pnv)ui
 0003:00009B8F       WaitForControlChange_
 0003:00009BEC       WaitForPCMInterrupt_
 0003:0000CD7F       waitqueue_active_
 0003:0008FA20       wctomb_
 0005:00002154       _alsa_fops
 0005:00042C37       _auto_pin_cfg_labels
 0003:00000050       _CallPDD16
 0002:00000448       _CallRM
 0005:00001D14       _cardcalls
 0005:0000A224       _card_id_changed
 0005:0000A220       _control_id_changed
 0005:000081E4       _CountWv
 0005:000018FC       _current
 0005:000018D8       _current_task
 0005:00000114       _DebugLevel
 0005:0008B440       _edata
 0005:0008B440       _end
 0005:0000004C       _fDebug
 0005:0000A22C       _fInInterrupt
 0005:00000110       _fStrategyInit
 0005:0000D4CC       _fSuspended
 0005:00000048       _fVerbose
 0005:000081EC       _hextab
 0005:00000050       _idc16_PddHandler
 0005:00001CC4       _iLastError
 0005:00000038       _InitCompleteWas
 0005:00001AA2       _iomem_resource
 0005:00001A86       _ioport_resource
 0003:0008FB10       _ismbblead_
 0005:000017DE       _ISR00
 0005:000017E2       _ISR01
 0005:000017E6       _ISR02
 0005:000017EA       _ISR03
 0005:000017EE       _ISR04
 0005:000017F2       _ISR05
 0005:000017F6       _ISR06
 0005:000017FA       _ISR07
 0005:000018D4       _jiffies
 0000:00000000  Imp  _KernSISData         (KEE.90)
 0005:000081E8       _LockAdd
 0005:000081FD       _MAGIC_COMM_PORT
 0005:00001ABE       _mem_map
 0001:00000058       _MESSAGE_STR
 0005:00001E1C       _midi_port
 0001:00000458       _MSG_TABLE16
 0005:00001788       _MSG_TABLE32
 0005:0000010C       _nrCardsDetected
 0005:00002168       _opened_handles
 0005:00042FD8       _opl3_ops
 0005:00002014       _oss_devices
 0005:0000AA8C       _pci_devices
 0005:00008200       _pcmcaps
 0005:00002160       _pcm_device
 0005:00002158       _per_bytes
 0005:0000215C       _prev_size
 0003:000052FE       _printk
 0005:00001CC8       _proc_root
 0003:000098A4       _put_user_
 0005:0000003C       _rdOffset
 0003:00000230       _RMAllocResource
 0002:00000204       _RMAllocResource16
 0002:000001C8       _RMAllocResourceOrg
 0003:000002F8       _RMCreateAdapter
 0002:00000264       _RMCreateAdapter16
 0002:00000228       _RMCreateAdapterOrg
 0003:000002B0       _RMCreateDevice
 0002:000002CC       _RMCreateDevice16
 0002:00000290       _RMCreateDeviceOrg
 0003:00000340       _RMCreateDriver
 0002:00000428       _RMCreateDriver16
 0002:000003AE       _RMCreateDriverOrg
 0003:00000270       _RMDeallocResource
 0002:00000368       _RMDeallocResource16
 0002:0000033E       _RMDeallocResourceOrg
 0002:00000322       _RMDestroyDevice16
 0002:000002F8       _RMDestroyDeviceOrg
 0003:00000380       _RMDestroyDriver
 0002:000004A6       _RMDestroyDriver16
 0002:0000047C       _RMDestroyDriverOrg
 0003:000003EC       _RMDevIDToHandleList
 0002:00000556       _RMDevIDToHandleList16
 0001:00000054       _RMFlags
 0003:000003AC       _RMGetNodeInfo
 0002:000004FA       _RMGetNodeInfo16
 0003:00000440       _RMHandleToResourceHandleList
 0002:000005CA       _RMHandleToResourceHandleList16
 0001:00000048       _RM_Help0
 0001:0000004C       _RM_Help1
 0001:00000050       _RM_Help3
 0005:000000E8       _SaveIRQCounter
 0005:00042E04       _seq_client_load
 0005:00042E48       _seq_default_timer_card
 0005:00042E40       _seq_default_timer_class
 0005:00042E4C       _seq_default_timer_device
 0005:00042E54       _seq_default_timer_resolution
 0005:00042E44       _seq_default_timer_sclass
 0005:00042E50       _seq_default_timer_subdevice
 0005:000000B0       _sISRHigh
 0005:00000DC0       _snd_cards
 0003:00083A6B       _snd_ctl_add_slave_
 0005:00000ABC       _snd_ecards_limit
 0005:0004297B       _snd_hda_bind_sw
 0005:0004296B       _snd_hda_bind_vol
 0005:00042BD7       _snd_hda_pcm_type_name
 0005:00000AC0       _snd_major
 0005:00043208       _snd_opl3_regmap
 0005:00000ACC       _snd_oss_root
 0005:000005B4       _snd_pcm_devices_os2
 0005:0000EFA8       _snd_pcm_f_ops
 0003:000133B6       _snd_pcm_hw_params_any_
 0003:00013473       _snd_pcm_hw_param_setempty_
 0003:000806D7       _snd_pcm_hw_param_set_
 0005:00074E40       _snd_pcm_known_rates
 0003:000162C5       _snd_pcm_lib_alloc_vmalloc_buffer_
 0005:0000EEE4       _snd_pcm_link_rwlock
 0005:00000AD0       _snd_seq_root
 0005:00008220       _substream_int
 0005:00001900       _system_utsname
 0005:00001BC2       _szLastALSAError1
 0005:00001C43       _szLastALSAError2
 0005:00001C42       _szOverrunTest1
 0005:00001CC3       _szOverrunTest2
 0005:00000044       _szprintBuf
 0005:00001F88       _szRecSources
 0005:00001AC2       _this_module
 0005:000017D8       _TimerHandler16
 0005:00001808       _TKSSBase
 0005:00002164       _total
 0005:0000011C       _ulget_free_pagesMemUsed
 0005:0000A228       _unlock_all
 0005:00042FD4       _use_internal_drums
 0005:00000040       _wrOffset
 0005:00061B30       __AccessFHeap
 0005:00061B1C       __AccessFileH
 0005:00061B24       __AccessIOB
 0005:00061B2C       __AccessNHeap
 0005:00061B3C       __AccessTDList
 0005:00061BA8       __amblksiz
 0005:00061B80       __ASTACKPTR
 0005:00061B7C       __ASTACKSIZ
 0003:0008F8A0       __Bits
 0005:00061B84       __cbyte
 0005:00061B88       __cbyte2
 0003:00005358       __check_region_
 0005:00061B8C       __child
 0003:0008FE00       __CommonInit_
 0003:0000B991       __compat_get_order_
 0003:000097C5       __copy_user_
 0003:00009819       __copy_user_zeroing_
 0005:00061B58       __curbrk
 0000:00001234  Abs  __DOSseg__
 0005:00061B54       __dynend
 0005:0007B3E6       __End_XI
 0005:0007B3E6       __End_YI
 0003:0008FF40       __EnterWVIDEO_
 0005:00061B92       __Envptr
 0005:00061B96       __Envseg
 0003:0008F9D6       __exit_
 0003:0008FCD0       __exit_with_msg_
 0003:0008FD20       __fatal_runtime_error_
 0003:0008F830       __FDFS
 0003:0008FDA0       __FiniRtns
 0003:00000000       __GETDS
 0003:00009088       __get_free_dma_pages_
 0003:00009273       __get_free_pages_
 0003:00009879       __get_user_
 0003:0008D5F5       __I8LS
 0003:0008D610       __I8M
 0003:0008D5DA       __I8RS
 0003:0008FD50       __InitRtns
 0003:00009755       __ioremap_
 0003:0008DB60       __IsTable
 0003:0000998F       __kfree_
 0003:000098B4       __kmalloc_
 0005:00061B5C       __LpCmdLine
 0005:00061B64       __LpDllName
 0005:00061B60       __LpPgmName
 0005:00061B68       __LpwCmdLine
 0005:00061B70       __LpwDllName
 0005:00061B6C       __LpwPgmName
 0003:0008FE45       __mbinit_
 0005:00061B90       __no87
 0005:0007B430       __nullarea
 0003:00000000       __OffBeginCS32
 0005:00000000       __OffBeginDS32
 0002:00000689       __OffFinalCS16
 0003:0008FF68       __OffFinalCS32
 0001:00000483       __OffFinalDS16
 0005:0007B3DC       __OffFinalDS32
 0005:00001784       __OffsetFinalCS16
 0005:00001786       __OffsetFinalDS16
 0003:0008F9B9       __OS2Fini_
 0003:0008F97B       __OS2Init_
 0003:0008F90C       __OS2MainInit_
 0005:00061B98       __osmajor
 0005:00061B99       __osminor
 0003:0008EAF0       __prtf_
 0005:00061B38       __ReleaseFHeap
 0005:00061B20       __ReleaseFileH
 0005:00061B28       __ReleaseIOB
 0005:00061B34       __ReleaseNHeap
 0005:00061B40       __ReleaseTDList
 0003:0000B4CD       __release_region_
 0003:0000B453       __request_region_
 0003:0008E880       __scnf_
 0003:0008F811       __set_doserrno_
 0003:0008F7E2       __set_EDOM_
 0003:0008F7FE       __set_EINVAL_
 0003:0008F7F0       __set_ERANGE_
 0003:0008F7D4       __set_errno_
 0003:0008F9C1       __shutdown_stack_checking_
 0003:0008D4D2       __snd_util_memblk_new_
 0003:0008D47E       __snd_util_mem_alloc_
 0003:0008D54B       __snd_util_mem_free_
 0005:00061B74       __STACKLOW
 0005:00061B78       __STACKTOP
 0005:0007B3E0       __Start_XI
 0005:0007B3E6       __Start_YI
 0003:0008DC70       __STOSB
 0003:0008DCA7       __STOSD
 0003:0008F903       __threadid_
 0003:0008F8FC       __threadstack_
 0005:00061B4C       __threadstksize
 0003:0008D5F5       __U8LS
 0003:0008D610       __U8M
 0003:0008D5C0       __U8RS
 0003:000051AA       __udelay_
 0003:0000CD7D       __wake_up_
 0003:00004C50       __wcpp_2_pure_error__
 0003:00004C4C       __wcpp_2_undefed_cdtor__
 0003:00004C4E       __wcpp_2_undefined_member_function__
 0003:00004C52       __wcpp_2_undef_vfun__
 0003:00004C58       __wcpp_4_pure_error__
 0003:00004C54       __wcpp_4_undefed_cdtor__
 0003:00004C56       __wcpp_4_undefined_member_function__
 0003:00004C5A       __wcpp_4_undef_vfun__
 0005:00072188       ___Alphabet
 0004:00000003       ___begtext
 0005:00061B0C       ___EFG_printf
 0005:00061B10       ___EFG_scanf
 0005:000623FE       ___exitcall_alsa_ac97_exit
 0005:000547E0       ___exitcall_alsa_card_ali_exit
 0005:0000F4D8       ___exitcall_alsa_card_als4000_exit
 0005:0001057C       ___exitcall_alsa_card_atiixp_exit
 0005:00042818       ___exitcall_alsa_card_azx_exit
 0005:0000F374       ___exitcall_alsa_card_bt87x_exit
 0005:000137F4       ___exitcall_alsa_card_ca0106_exit
 0005:00010259       ___exitcall_alsa_card_cmipci_exit
 0005:00012F34       ___exitcall_alsa_card_cs4281_exit
 0005:000432FC       ___exitcall_alsa_card_cs46xx_exit
 0005:00050F84       ___exitcall_alsa_card_cs5535audio_exit
 0005:00051180       ___exitcall_alsa_card_emu10k1_exit
 0005:00013340       ___exitcall_alsa_card_ens137x_exit
 0005:00012C99       ___exitcall_alsa_card_es1938_exit
 0005:00012438       ___exitcall_alsa_card_es1968_exit
 0005:000109E8       ___exitcall_alsa_card_fm801_exit
 0005:000121F4       ___exitcall_alsa_card_intel8x0_exit
 0005:000114E4       ___exitcall_alsa_card_m3_exit
 0005:00061530       ___exitcall_alsa_card_nm256_exit
 0005:000548AC       ___exitcall_alsa_card_trident_exit
 0005:00010FBC       ___exitcall_alsa_card_via82xx_exit
 0005:00053E58       ___exitcall_alsa_card_ymfpci_exit
 0005:0000E938       ___exitcall_alsa_hwdep_exit
 0005:00043250       ___exitcall_alsa_mpu401_uart_exit
 0005:00043074       ___exitcall_alsa_opl3_exit
 0005:00043000       ___exitcall_alsa_opl3_seq_exit
 0005:0000EE04       ___exitcall_alsa_pcm_exit
 0005:00061A7C       ___exitcall_alsa_pcm_oss_exit
 0005:0000EA74       ___exitcall_alsa_rawmidi_exit
 0005:000619FC       ___exitcall_alsa_sb_common_exit
 0005:00042E84       ___exitcall_alsa_seq_device_exit
 0005:00042E5C       ___exitcall_alsa_seq_exit
 0005:00062528       ___exitcall_alsa_seq_midi_emul_exit
 0005:0000EE60       ___exitcall_alsa_sound_exit
 0005:0000E9E4       ___exitcall_alsa_timer_exit
 0005:00062530       ___exitcall_alsa_util_mem_exit
 0005:000230C8       ___exitcall_patch_analog_exit
 0005:00019140       ___exitcall_patch_atihdmi_exit
 0005:0002385C       ___exitcall_patch_cmedia_exit
 0005:00018FE0       ___exitcall_patch_conexant_exit
 0005:0004253F       ___exitcall_patch_realtek_exit
 0005:0001B940       ___exitcall_patch_sigmatel_exit
 0005:00016874       ___exitcall_patch_via_exit
 0005:0000F0B8       ___exitcall_snd_mem_exit
 0005:00061B14       ___FirstThreadData
 0005:00061B9A       ___FPE_handler
 0005:00061B18       ___GetThreadPtr
 0005:00001748       ___hmodule
 0005:000623FA       ___initcall_alsa_ac97_init
 0005:000547DC       ___initcall_alsa_card_ali_init
 0005:0000F4D4       ___initcall_alsa_card_als4000_init
 0005:00010578       ___initcall_alsa_card_atiixp_init
 0005:00042814       ___initcall_alsa_card_azx_init
 0005:0000F370       ___initcall_alsa_card_bt87x_init
 0005:000137F0       ___initcall_alsa_card_ca0106_init
 0005:00010255       ___initcall_alsa_card_cmipci_init
 0005:00012F30       ___initcall_alsa_card_cs4281_init
 0005:000432F8       ___initcall_alsa_card_cs46xx_init
 0005:00050F80       ___initcall_alsa_card_cs5535audio_init
 0005:0005117C       ___initcall_alsa_card_emu10k1_init
 0005:0001333C       ___initcall_alsa_card_ens137x_init
 0005:00012C95       ___initcall_alsa_card_es1938_init
 0005:00012434       ___initcall_alsa_card_es1968_init
 0005:000109E4       ___initcall_alsa_card_fm801_init
 0005:000121F0       ___initcall_alsa_card_intel8x0_init
 0005:000114E0       ___initcall_alsa_card_m3_init
 0005:0006152C       ___initcall_alsa_card_nm256_init
 0005:000548A8       ___initcall_alsa_card_trident_init
 0005:00010FB8       ___initcall_alsa_card_via82xx_init
 0005:00053E54       ___initcall_alsa_card_ymfpci_init
 0005:0000E934       ___initcall_alsa_hwdep_init
 0005:0004324C       ___initcall_alsa_mpu401_uart_init
 0005:00043070       ___initcall_alsa_opl3_init
 0005:00042FFC       ___initcall_alsa_opl3_seq_init
 0005:0000EE00       ___initcall_alsa_pcm_init
 0005:00061A78       ___initcall_alsa_pcm_oss_init
 0005:0000EA70       ___initcall_alsa_rawmidi_init
 0005:000619F8       ___initcall_alsa_sb_common_init
 0005:00042E80       ___initcall_alsa_seq_device_init
 0005:00042E58       ___initcall_alsa_seq_init
 0005:00062524       ___initcall_alsa_seq_midi_emul_init
 0005:0000EE5C       ___initcall_alsa_sound_init
 0005:0000E9E0       ___initcall_alsa_timer_init
 0005:0006252C       ___initcall_alsa_util_mem_init
 0005:000230C4       ___initcall_patch_analog_init
 0005:0001913C       ___initcall_patch_atihdmi_init
 0005:00023858       ___initcall_patch_cmedia_init
 0005:00018FDC       ___initcall_patch_conexant_init
 0005:0004253B       ___initcall_patch_realtek_init
 0005:0001B93C       ___initcall_patch_sigmatel_init
 0005:00016870       ___initcall_patch_via_init
 0005:0000F0B4       ___initcall_snd_mem_init
 0005:00001744       ___IsDBCS
 0005:00001538       ___Is_DLL
 0005:00061BA0       ___MBCodePage
 0005:00001640       ___MBCSIsTable
 0005:00061B50       ___process_fini
 0005:0000153C       ___saved_CS
 0005:00061B48       ___sig_fini_rtn
 0005:00061B44       ___sig_init_rtn
 0005:00061BA4       ___WD_Present


 Address         Publics by Value
 0000:00000000  Imp  KernThunkStackTo32   (KEE.41)
 0000:00000000  Imp  DOSOPEN              (DOSCALLS.70)
 0000:00000000  Imp  DosQueryCp           (DOSCALLS.291)
 0000:00000000  Imp  DosQueryDBCSEnv      (NLS.6)
 0000:00000000  Imp  KernVMLock           (KEE.62)
 0000:00000000  Imp  DosExit              (DOSCALLS.234)
 0000:00000000  Imp  KernVMFree           (KEE.61)
 0000:00000000  Imp  DosQuerySysInfo      (DOSCALLS.348)
 0000:00000000  Imp  DOSWRITE             (DOSCALLS.138)
 0000:00000000  Imp  KernVMAlloc          (KEE.60)
 0000:00000000  Imp  KernLinToPageList    (KEE.64)
 0000:00000000  Imp  _KernSISData         (KEE.90)
 0000:00000000  Imp  KernSelToFlat        (KEE.66)
 0000:00000000  Imp  DOSCLOSE             (DOSCALLS.59)
 0000:00000000  Imp  DosWrite             (DOSCALLS.282)
 0000:00000000  Imp  DOSIODELAYCNT        (DOSCALLS.427)
 0000:00000000  Imp  DOS32FLATDS          (DOSCALLS.370)
 0000:00000000  Imp  KernThunkStackTo16   (KEE.40)
 0000:00001234  Abs  __DOSseg__
 0001:00000000       help_header
 0001:0000001E       uniaud_header
 0001:0000003C       DevHelpInit
 0001:00000040       fOpen
 0001:00000044       InitPktSeg
 0001:00000046       InitPktOff
 0001:00000048       _RM_Help0
 0001:0000004C       _RM_Help1
 0001:00000050       _RM_Help3
 0001:00000054       _RMFlags
 0001:00000058       _MESSAGE_STR
 0001:00000458       _MSG_TABLE16
 0001:0000045E       pddname16
 0001:00000465       FileName
 0001:00000483       __OffFinalDS16
 0002:00000000       help_stub_strategy
 0002:00000096       uniaud_stub_strategy
 0002:0000010A       uniaud_stub_idc
 0002:00000128       uniaud_stub_timer
 0002:000001A0       thunk3216_devhelp
 0002:000001B2       thunk3216_devhelp_modified_ds
 0002:000001C8       _RMAllocResourceOrg
 0002:00000204       _RMAllocResource16
 0002:00000228       _RMCreateAdapterOrg
 0002:00000264       _RMCreateAdapter16
 0002:00000290       _RMCreateDeviceOrg
 0002:000002CC       _RMCreateDevice16
 0002:000002F8       _RMDestroyDeviceOrg
 0002:00000322       _RMDestroyDevice16
 0002:0000033E       _RMDeallocResourceOrg
 0002:00000368       _RMDeallocResource16
 0002:00000388       MY_DEVHELP_ATTACHDD
 0002:000003AE       _RMCreateDriverOrg
 0002:00000428       _RMCreateDriver16
 0002:00000448       _CallRM
 0002:0000047C       _RMDestroyDriverOrg
 0002:000004A6       _RMDestroyDriver16
 0002:000004FA       _RMGetNodeInfo16
 0002:00000556       _RMDevIDToHandleList16
 0002:000005CA       _RMHandleToResourceHandleList16
 0002:00000689       __OffFinalCS16
 0003:00000000       __OffBeginCS32
 0003:00000000       __GETDS
 0003:00000010       DevHlp
 0003:00000024       thunk1632_devhelp
 0003:00000030       DevHlp_ModifiedDS
 0003:00000044       thunk1632_devhelp_modified_ds
 0003:00000050       _CallPDD16
 0003:00000080       STRATEGY_
 0003:000000E0       IDC_
 0003:00000140       TIMER_
 0003:00000230       _RMAllocResource
 0003:00000270       _RMDeallocResource
 0003:000002B0       _RMCreateDevice
 0003:000002F8       _RMCreateAdapter
 0003:00000340       _RMCreateDriver
 0003:00000380       _RMDestroyDriver
 0003:000003AC       _RMGetNodeInfo
 0003:000003EC       _RMDevIDToHandleList
 0003:00000440       _RMHandleToResourceHandleList
 0003:0000047D       W?StratOpen$n(pf$RP$$)ul
 0003:000004A2       W?StratInit$n(pf$RP$$)ul
 0003:000004A7       W?StratInitComplete$n(pf$RP$$)ul
 0003:0000050A       W?StratShutdown$n(pf$RP$$)ul
 0003:00000524       ALSA_STRATEGY
 0003:00000549       W?StratRead$n(pf$RP$$)ul
 0003:0000064F       W?DevSaveMessage$n(pfai)v
 0003:000006CF       W?LockSegments$n()i
 0003:00000771       W?DiscardableInit$n(pf$RPInit$$)ul
 0003:00001543       W?toupper$n(i)i
 0003:00001551       W?mymemchr$n(pfaaus)pfa
 0003:00001589       W?sz2us$n(pfai)us
 0003:00001621       W?IsWhitespace$n(a)i
 0003:0000163A       W?SkipWhite$n(pfa)pfa
 0003:0000167A       W?CheckCardName$n(pfa)v
 0003:000018B1       W?DoParm$n(apfa)i
 0003:00001B8E       W?ParseParm$n(pfai)i
 0003:000027B9       GetParms_
 0003:000034B0       GetTKSSBase
 0003:000034F0       iodelay32_
 0003:000035F2       ALSA_IDC
 0003:00003A26       W?OSS32IDC$n(ulpn$__6ikc0pIDC32_PACKET$$)ul
 0003:00003D37       W?StratIOCtl$n(pf$RP$$)ul
 0003:00004448       W?StratClose$n(pf$RP$$)ul
 0003:00004477       RMInit_
 0003:000045EE       RMRequestIO_
 0003:00004692       RMRequestMem_
 0003:00004727       RMRequestIRQ_
 0003:000047F8       RMDone_
 0003:00004B78       ALSA_SetIrq_
 0003:00004C07       ALSA_FreeIrq_
 0003:00004C25       ALSA_Interrupt
 0003:00004C4C       __wcpp_2_undefed_cdtor__
 0003:00004C4E       __wcpp_2_undefined_member_function__
 0003:00004C50       __wcpp_2_pure_error__
 0003:00004C52       __wcpp_2_undef_vfun__
 0003:00004C54       __wcpp_4_undefed_cdtor__
 0003:00004C56       __wcpp_4_undefined_member_function__
 0003:00004C58       __wcpp_4_pure_error__
 0003:00004C5A       __wcpp_4_undef_vfun__
 0003:00004C5C       W?$nwn(ui)pnv
 0003:00004C61       W?$dln(pnv)v
 0003:00004C66       W?$nwn(uipnv)pnv
 0003:00004C6D       os2gettimesec_
 0003:00004C73       os2gettimemsec_
 0003:00004E8A       vsprintf_
 0003:00005139       sprintf_
 0003:0000515F       ALSA_TIMER_
 0003:0000519B       schedule_timeout_
 0003:000051AA       __udelay_
 0003:000051BE       mdelay_
 0003:000051E7       do_gettimeofday_
 0003:00005223       add_timer_
 0003:00005224       del_timer_
 0003:00005227       mod_timer_
 0003:00005228       msleep_
 0003:0000525A       strcmp_
 0003:0000527D       strncmp_
 0003:000052A6       tasklet_hi_schedule_
 0003:000052BB       tasklet_init_
 0003:000052CF       OSS32_SetFileId_
 0003:000052FE       _printk
 0003:00005356       schedule_
 0003:00005357       poll_wait_
 0003:00005358       __check_region_
 0003:0000535B       hweight32_
 0003:000053B7       create_proc_entry_
 0003:000053F4       remove_proc_entry_
 0003:000053F5       proc_register_
 0003:000053F8       proc_unregister_
 0003:000053FB       fasync_helper_
 0003:000053FE       kill_fasync_
 0003:000053FF       request_dma_
 0003:00005402       free_dma_
 0003:00005403       enable_dma_
 0003:00005404       disable_dma_
 0003:00005405       register_reboot_notifier_
 0003:00005408       unregister_reboot_notifier_
 0003:00005446       queue_work_
 0003:000054DA       flush_workqueue_
 0003:00005529       create_workqueue_
 0003:00005575       destroy_workqueue_
 0003:0000557A       kstrdup_
 0003:000055B5       mod_firmware_load_
 0003:000055F2       request_firmware_
 0003:00005671       release_firmware_
 0003:00005689       memdup_user_
 0003:000056CC       cancel_delayed_work_
 0003:000056EE       schedule_work_
 0003:00005709       queue_delayed_work_
 0003:00005751       gcd_
 0003:0000576A       strict_strtoul_
 0003:000057C7       W?CallOSS16$n(ululul)ul
 0003:000057FC       OSS32_Initialize_
 0003:000059A0       OSS32_Shutdown_
 0003:00005A33       OSS32_ProcessIRQ_
 0003:00005A6E       OSS32_ProcessMIDIIRQ_
 0003:00005AA8       OSS32_CloseUNI16_
 0003:00005AE3       MyDevBlock_
 0003:00005B12       OSS32_DebugString_
 0003:00005B39       OSS32_MidiOpen_
 0003:00005EA6       OSS32_MidiClose_
 0003:00005FCC       OSS32_MidiWrite_
 0003:00005FD2       OSS32_MidiRead_
 0003:00006021       OSS32_MidiQueryCaps_
 0003:00006045       OSS32_MidiCommand_
 0003:0000616C       ConvertVolume_
 0003:00006190       OSS32_MixOpen_
 0003:0000668B       OSS32_MixClose_
 0003:000066E1       OSS32_MixGetVolume_
 0003:0000673C       OSS32_MixSetVolume_
 0003:00006A50       OSS32_MixSetProperty_
 0003:00006D7D       OSS32_MixGetProperty_
 0003:00006D9C       OSSToALSAVolume_
 0003:00006E80       OSS32_MixQueryCaps_
 0003:00006F15       OSS32_MixQueryName_
 0003:00007007       OSS32_QueryNames_
 0003:0000717C       register_chrdev_
 0003:00007195       unregister_chrdev_
 0003:000071AD       register_sound_special_
 0003:000071E2       register_sound_mixer_
 0003:00007217       register_sound_midi_
 0003:0000724C       register_sound_dsp_
 0003:0000727E       register_sound_synth_
 0003:000072B3       unregister_sound_special_
 0003:000072C9       unregister_sound_mixer_
 0003:000072DF       unregister_sound_midi_
 0003:000072F5       unregister_sound_dsp_
 0003:0000730B       unregister_sound_synth_
 0003:00007321       UNIXToOSSError_
 0003:000073FC       ALSAToOSSDataType_
 0003:0000747A       ALSAToOSSRateFlags_
 0003:00007550       OSS32_QueryDevCaps_
 0003:000078C1       OSS32_WaveOpen_
 0003:00007A87       OSS32_WaveClose_
 0003:00007B55       OSS32_WavePrepare_
 0003:00007BB8       OSS32_WaveStart_
 0003:00007C0E       OSS32_WaveStop_
 0003:00007C64       OSS32_WavePause_
 0003:00007CBA       OSS32_WaveResume_
 0003:00007D13       OSS32_WaveSetHwParams_
 0003:0000857B       OSS32_WaveAddBuffer_
 0003:0000879C       OSS32_WaveGetPosition_
 0003:00008802       OSS32_WaveGetSpace_
 0003:00008868       OSS32_WaveGetHwPtr_
 0003:000088CE       OSS32_WaveGetStatus_
 0003:00008929       OSS32_WaveSetVolume_
 0003:0000898A       DecLongToASCII_
 0003:00008A6C       HexLongToASCII_
 0003:00008B4A       CharOut_
 0003:00008B8C       StringOut_
 0003:00008CD3       snd_iprintf_
 0003:00008EA5       AddBaseAddress_
 0003:00008ED9       GetBaseAddress_
 0003:00008FAA       virt_to_phys_
 0003:00008FD8       phys_to_virt_
 0003:00009014       VMAlloc_
 0003:0000907A       VMFree_
 0003:00009088       __get_free_dma_pages_
 0003:00009273       __get_free_pages_
 0003:0000962F       free_pages_
 0003:0000965C       vmalloc_
 0003:0000971E       vfree_
 0003:0000974F       alloc_pages_
 0003:00009752       remap_page_range_
 0003:00009755       __ioremap_
 0003:000097AC       iounmap_
 0003:000097BF       is_access_ok_
 0003:000097C5       __copy_user_
 0003:000097EE       copy_to_user_
 0003:00009819       __copy_user_zeroing_
 0003:0000984E       copy_from_user_
 0003:00009879       __get_user_
 0003:000098A4       _put_user_
 0003:000098B4       __kmalloc_
 0003:0000998F       __kfree_
 0003:000099D4       kzalloc_
 0003:00009AC8       kcalloc_
 0003:00009B5C       uniaud_set_interrupted_substream_
 0003:00009B8F       WaitForControlChange_
 0003:00009BEC       WaitForPCMInterrupt_
 0003:00009CAC       GetNumberOfCards_
 0003:00009CB2       GetNumberOfPcm_
 0003:00009CB7       SetPCMInstance_
 0003:00009CD6       GetPcmForChannels_
 0003:00009D61       GetMaxChannels_
 0003:00009DDD       GetUniaudPcmCaps1_
 0003:0000A0D6       FillCaps_
 0003:0000A128       GetUniaudPcmCaps_
 0003:0000A171       UniaudCtlGetPowerState_
 0003:0000A235       UniaudCtlSetPowerState_
 0003:0000A2F9       GetUniaudCardInfo_
 0003:0000A3D5       GetUniaudControlNum_
 0003:0000A508       GetUniaudControls_
 0003:0000A670       GetUniaudControlInfo_
 0003:0000A751       GetUniaudControlValueGet_
 0003:0000A836       GetUniaudControlValuePut_
 0003:0000A91B       UniaudIoctlHWRefine_
 0003:0000A96B       UniaudIoctlHWParamSet_
 0003:0000A9BB       UniaudIoctlSWParamSet_
 0003:0000AA0B       UniaudIoctlPCMStatus_
 0003:0000AA4C       UniaudIoctlPCMWrite_
 0003:0000AA7C       UniaudIoctlPCMRead_
 0003:0000AAAC       UniaudIoctlPCMPrepare_
 0003:0000AADD       UniaudIoctlPCMResume_
 0003:0000AB10       UniaudIoctlPCMStart_
 0003:0000AB41       UniaudIoctlPCMDrop_
 0003:0000AB72       UniaudCloseAll_
 0003:0000ABFD       request_irq_
 0003:0000ACFA       free_irq_
 0003:0000AD61       eoi_irq_
 0003:0000AD6E       process_interrupt_
 0003:0000AE40       in_interrupt_
 0003:0000AE46       disable_irq_
 0003:0000AE47       pci_read_config_byte_
 0003:0000AE87       pci_read_config_word_
 0003:0000AEC9       pci_read_config_dword_
 0003:0000AF00       pci_write_config_byte_
 0003:0000AF40       pci_write_config_word_
 0003:0000AF81       pci_write_config_dword_
 0003:0000AFB6       pcidev_prepare_
 0003:0000AFBC       pcidev_activate_
 0003:0000AFC2       pcidev_deactivate_
 0003:0000B3BC       pci_find_device_
 0003:0000B453       __request_region_
 0003:0000B4CD       __release_region_
 0003:0000B4F8       pci_get_flags_
 0003:0000B51E       pcibios_present_
 0003:0000B535       pci_find_slot_
 0003:0000B549       pci_dma_supported_
 0003:0000B55E       pci_find_capability_
 0003:0000B5ED       pci_set_power_state_
 0003:0000B761       pci_enable_device_
 0003:0000B79F       pci_register_driver_
 0003:0000B8B2       pci_module_init_
 0003:0000B8C1       pci_unregister_driver_
 0003:0000B951       pci_set_master_
 0003:0000B98D       pm_register_
 0003:0000B990       pm_unregister_
 0003:0000B991       __compat_get_order_
 0003:0000B9A6       pci_alloc_consistent_
 0003:0000BA62       pci_free_consistent_
 0003:0000BA72       pci_set_driver_data_
 0003:0000BA7D       pci_get_driver_data_
 0003:0000BA88       pci_get_dma_mask_
 0003:0000BA93       release_resource_
 0003:0000BA96       pci_set_latency_time_
 0003:0000BAA9       pci_orig_save_state_
 0003:0000BAD5       pci_orig_restore_state_
 0003:0000BB38       pci_save_state_
 0003:0000BB83       pci_restore_state_
 0003:0000BBD7       pci_disable_device_
 0003:0000BC13       pci_request_region_
 0003:0000C2C9       pci_release_region_
 0003:0000C5F8       pci_request_regions_
 0003:0000C633       pci_release_regions_
 0003:0000C64D       pci_match_device_
 0003:0000C6F1       snd_pci_dev_present_
 0003:0000C74C       snd_pci_compat_get_pci_driver_
 0003:0000C759       OSS32_APMResume_
 0003:0000C79E       OSS32_APMSuspend_
 0003:0000C7ED       W?dumpheap$n()v
 0003:0000C81E       W?SignatureCheck$n(pn$_MEMBLOCK$$pna)s
 0003:0000C863       W?HeapCheck$n(pna)v
 0003:0000C8BC       W?npvAllocateBlock$n(pn$_MEMBLOCK$$ulpn$1$)pnv
 0003:0000C939       W?malloc$n(ul)pnv
 0003:0000CA3C       W?remove$n(pn$_MEMBLOCK$$)v
 0003:0000CA6A       W?compact$n()v
 0003:0000CB0E       W?free$n(pnv)v
 0003:0000CC48       W?_memfree$n()ui
 0003:0000CC4E       W?_msize$n(pnv)ui
 0003:0000CC5A       W?realloc$n(pnvul)pnv
 0003:0000CCCD       W?IsHeapAddr$n(ul)ul
 0003:0000CCED       W?HeapInit$n(ul)ul
 0003:0000CD4D       strncpy_
 0003:0000CD72       init_waitqueue_head_
 0003:0000CD73       add_wait_queue_
 0003:0000CD74       add_wait_queue_exclusive_
 0003:0000CD75       remove_wait_queue_
 0003:0000CD76       interruptible_sleep_on_timeout_
 0003:0000CD7C       interruptible_sleep_on_
 0003:0000CD7D       __wake_up_
 0003:0000CD7E       init_waitqueue_entry_
 0003:0000CD7F       waitqueue_active_
 0003:0000CD82       spin_lock_init_
 0003:0000CD89       spin_lock_
 0003:0000CD93       spin_lock_flag_
 0003:0000CD9D       spin_trylock_
 0003:0000CDA0       spin_unlock_
 0003:0000D35D       snd_hwdep_new_
 0003:0000D8E8       snd_timer_open_
 0003:0000DA3E       snd_timer_close_
 0003:0000DB96       snd_timer_resolution_
 0003:0000DD71       snd_timer_start_
 0003:0000DECD       snd_timer_stop_
 0003:0000DF13       snd_timer_continue_
 0003:0000DF8D       snd_timer_pause_
 0003:0000E0A1       snd_timer_interrupt_
 0003:0000E2E9       snd_timer_new_
 0003:0000E59D       snd_timer_notify_
 0003:0000E693       snd_timer_global_new_
 0003:0000E6C8       snd_timer_global_free_
 0003:0000E6CD       snd_timer_global_register_
 0003:0000FD45       snd_rawmidi_drop_output_
 0003:0000FD87       snd_rawmidi_drain_output_
 0003:0000FDFB       snd_rawmidi_drain_input_
 0003:0000FFE0       snd_rawmidi_kernel_open_
 0003:000103F8       snd_rawmidi_kernel_release_
 0003:00010508       snd_rawmidi_info_select_
 0003:0001060A       snd_rawmidi_output_params_
 0003:000106AE       snd_rawmidi_input_params_
 0003:000107F8       snd_rawmidi_receive_
 0003:00010A96       snd_rawmidi_kernel_read_
 0003:00010BDC       snd_rawmidi_transmit_empty_
 0003:00010C25       snd_rawmidi_transmit_peek_
 0003:00010D03       snd_rawmidi_transmit_ack_
 0003:00010D7E       snd_rawmidi_transmit_
 0003:00010EFB       snd_rawmidi_kernel_write_
 0003:000112C7       snd_rawmidi_new_
 0003:000117B0       snd_rawmidi_set_ops_
 0003:00011864       snd_pcm_format_signed_
 0003:0001188C       snd_pcm_format_unsigned_
 0003:0001189F       snd_pcm_format_linear_
 0003:000118AF       snd_pcm_format_little_endian_
 0003:000118D7       snd_pcm_format_big_endian_
 0003:000118EA       snd_pcm_format_width_
 0003:00011912       snd_pcm_format_physical_width_
 0003:0001193A       snd_pcm_format_size_
 0003:00011950       snd_pcm_format_silence_64_
 0003:0001197B       snd_pcm_format_set_silence_
 0003:00011AB4       snd_pcm_limit_hw_rates_
 0003:00011B1C       snd_pcm_rate_to_rate_bit_
 0003:00011F84       snd_pcm_playback_silence_
 0003:0001223A       snd_pcm_update_state_
 0003:00012478       snd_pcm_update_hw_ptr_
 0003:00012482       snd_pcm_set_ops_
 0003:000124A7       snd_pcm_set_sync_
 0003:000125A9       snd_interval_refine_
 0003:000126FF       snd_interval_mul_
 0003:0001279D       snd_interval_div_
 0003:00012856       snd_interval_muldivk_
 0003:00012905       snd_interval_mulkdiv_
 0003:000129C7       snd_interval_ratnum_
 0003:00012E3C       snd_interval_list_
 0003:00012F32       snd_pcm_hw_rule_add_
 0003:0001304A       snd_pcm_hw_constraint_mask_
 0003:00013077       snd_pcm_hw_constraint_mask64_
 0003:000130C4       snd_pcm_hw_constraint_integer_
 0003:000130E3       snd_pcm_hw_constraint_minmax_
 0003:0001314F       snd_pcm_hw_constraint_list_
 0003:000131D8       snd_pcm_hw_constraint_ratnums_
 0003:00013261       snd_pcm_hw_constraint_ratdens_
 0003:000132AE       snd_pcm_hw_constraint_msbits_
 0003:000132F3       snd_pcm_hw_constraint_step_
 0003:0001333A       snd_pcm_hw_constraint_pow2_
 0003:000133B6       _snd_pcm_hw_params_any_
 0003:000133FC       snd_pcm_hw_param_value_
 0003:00013473       _snd_pcm_hw_param_setempty_
 0003:0001353A       snd_pcm_hw_param_first_
 0003:000135D7       snd_pcm_hw_param_last_
 0003:0001360E       snd_pcm_hw_params_choose_
 0003:0001378D       snd_pcm_lib_ioctl_
 0003:000137CB       snd_pcm_period_elapsed_
 0003:00013C62       snd_pcm_lib_write_
 0003:00013DCD       snd_pcm_lib_writev_
 0003:000140B2       snd_pcm_lib_read_
 0003:000141E0       snd_pcm_lib_readv_
 0003:000144B2       snd_pcm_format_name_
 0003:000144BA       snd_pcm_new_stream_
 0003:000145E8       snd_pcm_new_
 0003:00014759       snd_pcm_attach_substream_
 0003:000149CA       snd_pcm_detach_substream_
 0003:00014C24       snd_pcm_notify_
 0003:00014D7F       pcm_info_
 0003:00014E1B       pcm_instances_
 0003:00014E81       snd_lookup_minor_data_
 0003:00014F8B       snd_register_device_for_dev_
 0003:00015079       snd_unregister_device_
 0003:000150C8       snd_add_device_sysfs_file_
 0003:000151C2       snd_minor_info_init_
 0003:00015203       snd_minor_info_done_
 0003:000152C2       snd_info_check_reserved_words_
 0003:00015A0E       snd_info_init_
 0003:00015AAA       snd_info_done_
 0003:00015AF8       snd_info_card_create_
 0003:00015B5A       snd_info_card_register_
 0003:00015B73       snd_info_card_id_change_
 0003:00015BB2       snd_info_card_disconnect_
 0003:00015C06       snd_info_card_free_
 0003:00015C26       snd_info_get_line_
 0003:00015CB1       snd_info_get_str_
 0003:00015D90       snd_info_create_module_entry_
 0003:00015DAA       snd_info_create_card_entry_
 0003:00015E3B       snd_card_proc_new_
 0003:00015E93       snd_info_free_entry_
 0003:00015ED6       snd_info_register_
 0003:00016064       snd_pcm_lib_preallocate_free_
 0003:0001606C       snd_pcm_lib_preallocate_free_for_all_
 0003:000160CE       snd_pcm_lib_preallocate_pages_
 0003:000160E6       snd_pcm_lib_preallocate_pages_for_all_
 0003:00016146       snd_pcm_sgbuf_ops_page_
 0003:00016164       snd_pcm_sgbuf_get_chunk_size_
 0003:000161BA       snd_pcm_lib_malloc_pages_
 0003:00016285       snd_pcm_lib_free_pages_
 0003:000162C5       _snd_pcm_lib_alloc_vmalloc_buffer_
 0003:0001630B       snd_pcm_lib_free_vmalloc_buffer_
 0003:00016328       snd_pcm_timer_resolution_change_
 0003:0001641D       snd_pcm_timer_init_
 0003:00016516       snd_pcm_timer_done_
 0003:0001691A       snd_pcm_info_
 0003:000169DB       snd_pcm_info_user_
 0003:00016A37       snd_pcm_hw_refine_
 0003:000172FB       snd_pcm_status_
 0003:000178DF       snd_pcm_start_
 0003:00017997       snd_pcm_stop_
 0003:000179A8       snd_pcm_drain_done_
 0003:00017B76       snd_pcm_suspend_
 0003:00017BC7       snd_pcm_suspend_all_
 0003:00018786       snd_pcm_hw_constraints_init_
 0003:00018AC9       snd_pcm_hw_constraints_complete_
 0003:00018C60       snd_pcm_release_substream_
 0003:00018CC9       snd_pcm_open_substream_
 0003:00019C07       snd_pcm_kernel_ioctl_
 0003:00019E37       snd_oss_info_register_
 0003:00019FDD       snd_info_minor_register_
 0003:0001A031       snd_info_minor_unregister_
 0003:0001A043       snd_lookup_oss_minor_data_
 0003:0001A11E       snd_register_oss_device_
 0003:0001A1A9       snd_unregister_oss_device_
 0003:0001A320       snd_minor_info_oss_init_
 0003:0001A363       snd_minor_info_oss_done_
 0003:0001A37B       snd_device_new_
 0003:0001A3CE       snd_device_free_
 0003:0001A465       snd_device_disconnect_
 0003:0001A4CF       snd_device_register_
 0003:0001A529       snd_device_register_all_
 0003:0001A567       snd_device_disconnect_all_
 0003:0001A59F       snd_device_free_all_
 0003:0001A80C       snd_ctl_notify_
 0003:0001A96E       snd_ctl_new1_
 0003:0001AA3F       snd_ctl_free_one_
 0003:0001AB08       snd_ctl_add_
 0003:0001AC1B       snd_ctl_remove_
 0003:0001AC86       snd_ctl_remove_id_
 0003:0001AD43       snd_ctl_rename_id_
 0003:0001AD9F       snd_ctl_find_numid_
 0003:0001ADCC       snd_ctl_find_id_
 0003:0001BF0A       snd_ctl_register_ioctl_
 0003:0001BF64       snd_ctl_unregister_ioctl_
 0003:0001C070       snd_ctl_create_
 0003:0001C088       snd_ctl_boolean_mono_info_
 0003:0001C0A7       snd_ctl_boolean_stereo_info_
 0003:0001C0E6       snd_malloc_pages_
 0003:0001C112       snd_free_pages_
 0003:0001C13C       snd_malloc_dev_pages_
 0003:0001C179       snd_free_dev_pages_
 0003:0001C1AE       snd_dma_alloc_pages_
 0003:0001C23D       snd_dma_alloc_pages_fallback_
 0003:0001C29D       snd_dma_free_pages_
 0003:0001C2F0       snd_dma_get_reserved_buf_
 0003:0001C3A1       snd_dma_reserve_buf_
 0003:0001C506       snd_card_create_
 0003:0001C76B       snd_card_locked_
 0003:0001C842       snd_card_disconnect_
 0003:0001C9F1       snd_card_free_when_closed_
 0003:0001CA41       snd_card_free_
 0003:0001CC2B       snd_card_set_id_
 0003:0001CC51       snd_card_register_
 0003:0001CD2F       snd_card_info_read_oss_
 0003:0001CDB8       snd_card_info_init_
 0003:0001CE36       snd_card_info_done_
 0003:0001CE4D       snd_component_add_
 0003:0001CF13       snd_card_file_add_
 0003:0001CF87       snd_card_file_remove_
 0003:0001D03A       snd_power_wait_
 0003:0001D0FA       snd_free_sgbuf_pages_
 0003:0001D140       snd_malloc_sgbuf_pages_
 0003:000336B2       ioread8_
 0003:000336CD       ioread16_
 0003:000336EA       ioread32_
 0003:00033700       iowrite8_
 0003:00033713       iowrite16_
 0003:00033728       iowrite32_
 0003:0003373B       ioport_map_
 0003:0003374B       ioport_unmap_
 0003:0003374C       pci_iomap_
 0003:000338D7       pci_iounmap_
 0003:000338FB       snd_ca0106_ptr_read_
 0003:00033935       snd_ca0106_ptr_write_
 0003:0003396F       snd_ca0106_spi_write_
 0003:00033A41       snd_ca0106_i2c_write_
 0003:000356B2       ca_midi_init_
 0003:000360AB       snd_ca0106_mixer_
 0003:0003624A       snd_ca0106_mixer_suspend_
 0003:00036283       snd_ca0106_mixer_resume_
 0003:00036AD6       snd_ca0106_proc_init_
 0003:0005060A       snd_hda_add_codec_preset_
 0003:0005063A       snd_hda_delete_codec_preset_
 0003:00050662       snd_hda_get_jack_location_
 0003:000506AB       snd_hda_get_jack_connectivity_
 0003:000506B9       snd_hda_get_jack_type_
 0003:000507D8       snd_hda_codec_read_
 0003:00050805       snd_hda_codec_write_
 0003:0005083E       snd_hda_sequence_write_
 0003:0005086B       snd_hda_get_sub_nodes_
 0003:000508A3       snd_hda_get_connections_
 0003:00050AC2       snd_hda_queue_unsol_event_
 0003:00050BA5       snd_hda_bus_new_
 0003:00051030       snd_hda_add_pincfg_
 0003:000510BC       snd_hda_codec_set_pincfg_
 0003:000510D1       snd_hda_codec_get_pincfg_
 0003:00051162       snd_hda_shutup_pins_
 0003:0005125C       snd_hda_codec_new_
 0003:000514E5       snd_hda_codec_configure_
 0003:000515AA       snd_hda_codec_setup_stream_
 0003:000515F0       snd_hda_codec_cleanup_stream_
 0003:000516DD       query_amp_caps_
 0003:0005174E       snd_hda_override_amp_caps_
 0003:000517CB       snd_hda_query_pin_caps_
 0003:000517E6       snd_hda_pin_sense_
 0003:0005183C       snd_hda_jack_detect_
 0003:00051936       snd_hda_codec_amp_read_
 0003:00051976       snd_hda_codec_amp_update_
 0003:00051A1D       snd_hda_codec_amp_stereo_
 0003:00051A68       snd_hda_codec_resume_amp_
 0003:00051B1B       snd_hda_mixer_amp_volume_info_
 0003:00051C00       snd_hda_mixer_amp_volume_get_
 0003:00051C9A       snd_hda_mixer_amp_volume_put_
 0003:00051D49       snd_hda_mixer_amp_tlv_
 0003:00051E0C       snd_hda_set_vmaster_tlv_
 0003:00051EA8       snd_hda_find_mixer_ctl_
 0003:00051EB2       snd_hda_ctl_add_
 0003:00051F1F       snd_hda_add_nid_
 0003:00051F60       snd_hda_ctls_clear_
 0003:00052000       snd_hda_codec_reset_
 0003:00052159       snd_hda_add_vmaster_
 0003:000521E5       snd_hda_mixer_amp_switch_info_
 0003:00052215       snd_hda_mixer_amp_switch_get_
 0003:000522AC       snd_hda_mixer_amp_switch_put_
 0003:00052367       snd_hda_mixer_bind_switch_get_
 0003:000523A2       snd_hda_mixer_bind_switch_put_
 0003:00052443       snd_hda_mixer_bind_ctls_info_
 0003:0005247B       snd_hda_mixer_bind_ctls_get_
 0003:000524B4       snd_hda_mixer_bind_ctls_put_
 0003:00052522       snd_hda_mixer_bind_tlv_
 0003:0005286E       snd_hda_create_spdif_out_ctls_
 0003:00052954       snd_hda_create_spdif_share_sw_
 0003:00052A45       snd_hda_create_spdif_in_ctls_
 0003:00052AEB       snd_hda_codec_write_cache_
 0003:00052B61       snd_hda_codec_update_cache_
 0003:00052BD7       snd_hda_codec_resume_cache_
 0003:00052C24       snd_hda_sequence_write_cache_
 0003:00052E20       snd_hda_build_controls_
 0003:00052E7D       snd_hda_codec_build_controls_
 0003:00052EB1       snd_hda_calc_stream_format_
 0003:00053204       snd_hda_is_supported_format_
 0003:0005344C       snd_hda_codec_build_pcms_
 0003:000534FF       snd_hda_build_pcms_
 0003:00053526       snd_hda_check_board_config_
 0003:000535A1       snd_hda_check_board_codec_sid_config_
 0003:000535E7       snd_hda_add_new_ctls_
 0003:00053654       snd_hda_ch_mode_info_
 0003:0005368B       snd_hda_ch_mode_get_
 0003:000536AF       snd_hda_ch_mode_put_
 0003:000536F8       snd_hda_input_mux_info_
 0003:00053747       snd_hda_input_mux_put_
 0003:00053883       snd_hda_bus_reboot_notify_
 0003:000538AC       snd_hda_multi_out_dig_open_
 0003:000538E6       snd_hda_multi_out_dig_prepare_
 0003:00053916       snd_hda_multi_out_dig_cleanup_
 0003:00053944       snd_hda_multi_out_dig_close_
 0003:00053966       snd_hda_multi_out_analog_open_
 0003:00053A7A       snd_hda_multi_out_analog_prepare_
 0003:00053C16       snd_hda_multi_out_analog_cleanup_
 0003:00053D59       snd_hda_parse_pin_def_config_
 0003:00054304       snd_hda_suspend_
 0003:00054327       snd_hda_resume_
 0003:0005434A       snd_array_new_
 0003:000543C8       snd_array_free_
 0003:000543E9       snd_print_pcm_rates_
 0003:00054444       snd_print_pcm_bits_
 0003:00054622       snd_hda_create_hwdep_
 0003:00055939       snd_hda_parse_generic_codec_
 0003:000559E5       ilog2_
 0003:00056C7B       snd_hda_codec_proc_new_
 0003:00056DA7       snd_seq_device_load_drivers_
 0003:00056DA8       snd_seq_device_new_
 0003:00056F79       snd_seq_device_register_driver_
 0003:000570B5       snd_seq_device_unregister_driver_
 0003:000573EA       snd_seq_info_init_
 0003:0005742B       snd_seq_info_done_
 0003:000574A4       snd_seq_system_broadcast_
 0003:000574D1       snd_seq_system_notify_
 0003:00057512       snd_seq_system_client_init_
 0003:0005763C       snd_seq_system_client_done_
 0003:000576AE       snd_seq_queue_get_cur_queues_
 0003:00057868       snd_seq_queues_init_
 0003:0005786B       snd_seq_queues_delete_
 0003:0005788B       snd_seq_queue_alloc_
 0003:000578CA       snd_seq_queue_delete_
 0003:000578F3       queueptr_
 0003:0005792C       snd_seq_queue_find_name_
 0003:00057969       snd_seq_check_queue_
 0003:00057A49       snd_seq_enqueue_event_
 0003:00057B42       snd_seq_queue_check_access_
 0003:00057B7C       snd_seq_queue_set_owner_
 0003:00057BCB       snd_seq_queue_timer_open_
 0003:00057C06       snd_seq_queue_timer_close_
 0003:00057C1D       snd_seq_queue_timer_set_tempo_
 0003:00057C8B       snd_seq_queue_use_
 0003:00057D1F       snd_seq_queue_is_used_
 0003:00057D53       snd_seq_queue_client_termination_
 0003:00057DB6       snd_seq_queue_client_leave_
 0003:00057E45       snd_seq_queue_client_leave_cells_
 0003:00057E83       snd_seq_queue_remove_cells_
 0003:00058035       snd_seq_control_queue_
 0003:0005808A       snd_seq_info_queues_read_
 0003:000581ED       snd_seq_dump_var_event_
 0003:000582DE       snd_seq_expand_var_event_
 0003:00058387       snd_seq_cell_free_
 0003:000584FA       snd_seq_event_dup_
 0003:000586D6       snd_seq_pool_poll_wait_
 0003:000586F6       snd_seq_pool_init_
 0003:00058794       snd_seq_pool_done_
 0003:0005884F       snd_seq_pool_new_
 0003:000588BB       snd_seq_pool_delete_
 0003:000588DA       snd_sequencer_memory_init_
 0003:000588DD       snd_sequencer_memory_done_
 0003:000588DE       snd_seq_info_pool_
 0003:000589CA       snd_seq_client_use_ptr_
 0003:00058A3D       client_init_data_
 0003:000592AD       snd_seq_dispatch_event_
 0003:00059B48       snd_seq_client_notify_subscription_
 0003:0005A0EB       snd_seq_set_queue_tempo_
 0003:0005A8A9       snd_seq_create_kernel_client_
 0003:0005A983       snd_seq_delete_kernel_client_
 0003:0005A9FF       snd_seq_kernel_client_enqueue_
 0003:0005AA0B       snd_seq_kernel_client_enqueue_blocking_
 0003:0005AA20       snd_seq_kernel_client_dispatch_
 0003:0005AA63       snd_seq_kernel_client_ctl_
 0003:0005AA76       snd_seq_kernel_client_write_poll_
 0003:0005ACB7       snd_seq_info_clients_read_
 0003:0005ADD9       snd_sequencer_device_init_
 0003:0005AE32       snd_sequencer_device_done_
 0003:0005AE77       snd_seq_port_use_ptr_
 0003:0005AED5       snd_seq_port_query_nearest_
 0003:0005AF72       snd_seq_create_port_
 0003:0005B1D7       snd_seq_delete_port_
 0003:0005B25E       snd_seq_delete_all_ports_
 0003:0005B311       snd_seq_set_port_info_
 0003:0005B39C       snd_seq_get_port_info_
 0003:0005B587       snd_seq_port_connect_
 0003:0005B7EB       snd_seq_port_disconnect_
 0003:0005B90B       snd_seq_port_get_subscription_
 0003:0005B94F       snd_seq_event_port_attach_
 0003:0005B9DD       snd_seq_event_port_detach_
 0003:0005BB06       snd_seq_timer_new_
 0003:0005BB4A       snd_seq_timer_delete_
 0003:0005BB83       snd_seq_timer_defaults_
 0003:0005BBE2       snd_seq_timer_reset_
 0003:0005BCA3       snd_seq_timer_set_tempo_
 0003:0005BCE0       snd_seq_timer_set_ppq_
 0003:0005BD41       snd_seq_timer_set_position_tick_
 0003:0005BD71       snd_seq_timer_set_position_time_
 0003:0005BDAB       snd_seq_timer_set_skew_
 0003:0005BDF1       snd_seq_timer_open_
 0003:0005BEED       snd_seq_timer_close_
 0003:0005BF10       snd_seq_timer_stop_
 0003:0005BFBB       snd_seq_timer_start_
 0003:0005C004       snd_seq_timer_continue_
 0003:0005C055       snd_seq_timer_get_cur_time_
 0003:0005C0E5       snd_seq_timer_get_cur_tick_
 0003:0005C0E9       snd_seq_info_timer_read_
 0003:0005C19B       snd_seq_prioq_new_
 0003:0005C1E5       snd_seq_prioq_delete_
 0003:0005C290       snd_seq_prioq_cell_in_
 0003:0005C35C       snd_seq_prioq_cell_out_
 0003:0005C3B3       snd_seq_prioq_avail_
 0003:0005C3D1       snd_seq_prioq_cell_peek_
 0003:0005C431       snd_seq_prioq_leave_
 0003:0005C5A9       snd_seq_prioq_remove_events_
 0003:0005C658       snd_seq_fifo_new_
 0003:0005C6DC       snd_seq_fifo_delete_
 0003:0005C725       snd_seq_fifo_clear_
 0003:0005C75D       snd_seq_fifo_event_in_
 0003:0005C80E       snd_seq_fifo_cell_out_
 0003:0005C899       snd_seq_fifo_cell_putback_
 0003:0005C8CD       snd_seq_fifo_poll_wait_
 0003:0005C8E8       snd_seq_fifo_resize_
 0003:0005C971       snd_opl3_synth_use_inc_
 0003:0005C98D       snd_opl3_synth_use_dec_
 0003:0005C98E       snd_opl3_synth_setup_
 0003:0005CA38       snd_opl3_synth_cleanup_
 0003:0005D15E       snd_opl3_interrupt_
 0003:0005D1D1       snd_opl3_new_
 0003:0005D254       snd_opl3_init_
 0003:0005D2C5       snd_opl3_create_
 0003:0005D40E       snd_opl3_timer_new_
 0003:0005D44B       snd_opl3_hwdep_new_
 0003:0005D7D1       snd_opl3_load_drums_
 0003:0005D842       snd_opl3_drum_switch_
 0003:0005D8EF       snd_opl3_calc_volume_
 0003:0005DB38       snd_opl3_timer_func_
 0003:0005DC40       snd_opl3_note_on_
 0003:0005E313       snd_opl3_note_off_
 0003:0005E343       snd_opl3_key_press_
 0003:0005E344       snd_opl3_terminate_note_
 0003:0005E472       snd_opl3_control_
 0003:0005E4D7       snd_opl3_nrpn_
 0003:0005E4D8       snd_opl3_sysex_
 0003:0005E4DB       snd_opl3_open_
 0003:0005E4DE       snd_opl3_ioctl_
 0003:0005E65A       snd_opl3_release_
 0003:0005E668       snd_opl3_write_
 0003:0005E75E       snd_opl3_load_patch_
 0003:0005E848       snd_opl3_find_patch_
 0003:0005E8BD       snd_opl3_clear_patches_
 0003:0005E8FB       snd_opl3_reset_
 0003:0005EDAF       snd_mpu401_uart_interrupt_
 0003:0005EDC1       snd_mpu401_uart_interrupt_tx_
 0003:0005F343       snd_mpu401_uart_new_
 0003:0005FC7F       snd_cs46xx_download_
 0003:0005FCB8       snd_cs46xx_download_image_
 0003:00060A42       snd_cs46xx_pcm_
 0003:00060CB5       snd_cs46xx_mixer_
 0003:000610BC       snd_cs46xx_midi_
 0003:00061173       snd_cs46xx_gameport_
 0003:00061547       snd_cs46xx_start_dsp_
 0003:000617DA       snd_cs46xx_suspend_
 0003:00061899       snd_cs46xx_resume_
 0003:000619D3       snd_cs46xx_create_
 0003:00062397       snd_cs5535audio_suspend_
 0003:0006243B       snd_cs5535audio_resume_
 0003:00062979       snd_cs5535audio_pcm_
 0003:00063650       snd_p16v_free_
 0003:00063661       snd_p16v_pcm_
 0003:00063A36       snd_p16v_mixer_
 0003:00063A75       snd_p16v_alloc_pm_buffer_
 0003:00063A97       snd_p16v_free_pm_buffer_
 0003:00063AA2       snd_p16v_suspend_
 0003:00063AD4       snd_p16v_resume_
 0003:00063BB1       snd_emu10k1_timer_
 0003:00063F32       snd_emu10k1_fx8010_register_irq_handler_
 0003:00063FD3       snd_emu10k1_fx8010_unregister_irq_handler_
 0003:0006412C       snd_emu10k1_efx_read_
 0003:0006A591       snd_emu10k1_init_efx_
 0003:0006A5C9       snd_emu10k1_free_efx_
 0003:0006A603       snd_emu10k1_fx8010_tram_setup_
 0003:0006AD8D       snd_emu10k1_fx8010_new_
 0003:0006AE3E       snd_emu10k1_efx_alloc_pm_buffer_
 0003:0006AEE5       snd_emu10k1_efx_free_pm_buffer_
 0003:0006AF16       snd_emu10k1_efx_suspend_
 0003:0006B039       snd_emu10k1_efx_resume_
 0003:0006C7D8       snd_emu10k1_mixer_
 0003:0006ED90       snd_emu10k1_pcm_
 0003:0006EEB0       snd_emu10k1_pcm_multi_
 0003:0006EF8D       snd_emu10k1_pcm_mic_
 0003:0006F729       snd_emu10k1_pcm_efx_
 0003:0006FE38       snd_emu10k1_midi_
 0003:0006FE85       snd_emu10k1_audigy_midi_
 0003:0006FF1D       snd_emu10k1_voice_init_
 0003:0007068F       snd_emu10k1_done_
 0003:000715D6       snd_emu10k1_create_
 0003:00071BD2       snd_emu10k1_suspend_regs_
 0003:00071C61       snd_emu10k1_resume_init_
 0003:00071CC5       snd_emu10k1_resume_regs_
 0003:00072698       snd_emu10k1_proc_init_
 0003:000728BF       snd_emu10k1_ptr_read_
 0003:0007297B       snd_emu10k1_ptr_write_
 0003:00072A4F       snd_emu10k1_ptr20_read_
 0003:00072A8F       snd_emu10k1_ptr20_write_
 0003:00072ACF       snd_emu10k1_spi_write_
 0003:00072BC5       snd_emu10k1_i2c_write_
 0003:00072CD0       snd_emu1010_fpga_write_
 0003:00072D5B       snd_emu1010_fpga_read_
 0003:00072DD2       snd_emu1010_fpga_link_dst_src_write_
 0003:00072E26       snd_emu10k1_intr_enable_
 0003:00072E5F       snd_emu10k1_intr_disable_
 0003:00072E9A       snd_emu10k1_voice_intr_enable_
 0003:00072EFF       snd_emu10k1_voice_intr_disable_
 0003:00072F66       snd_emu10k1_voice_intr_ack_
 0003:00072FC6       snd_emu10k1_voice_half_loop_intr_enable_
 0003:0007302B       snd_emu10k1_voice_half_loop_intr_disable_
 0003:00073092       snd_emu10k1_voice_half_loop_intr_ack_
 0003:000730F2       snd_emu10k1_voice_set_loop_stop_
 0003:00073157       snd_emu10k1_voice_clear_loop_stop_
 0003:000731BE       snd_emu10k1_wait_
 0003:00073219       snd_emu10k1_ac97_read_
 0003:0007325B       snd_emu10k1_ac97_write_
 0003:0007329D       snd_emu10k1_rate_to_pitch_
 0003:00073479       snd_emu10k1_voice_alloc_
 0003:00073507       snd_emu10k1_voice_free_
 0003:00073829       snd_emu10k1_memblk_map_
 0003:000738C9       snd_emu10k1_alloc_pages_
 0003:000739BA       snd_emu10k1_free_pages_
 0003:000739BF       snd_emu10k1_synth_alloc_
 0003:00073A1F       snd_emu10k1_synth_free_
 0003:00073C64       snd_emu10k1_synth_bzero_
 0003:00073CD8       snd_emu10k1_synth_copy_from_user_
 0003:00073D66       snd_emu10k1_interrupt_
 0003:00074183       snd_ymfpci_free_gameport_
 0003:00075C50       snd_ymfpci_pcm_
 0003:00075D21       snd_ymfpci_pcm2_
 0003:00075DDB       snd_ymfpci_pcm_spdif_
 0003:00075E9A       snd_ymfpci_pcm_4ch_
 0003:0007673D       snd_ymfpci_mixer_
 0003:000769F8       snd_ymfpci_timer_
 0003:00077107       snd_ymfpci_suspend_
 0003:000771D0       snd_ymfpci_resume_
 0003:000772BA       snd_ymfpci_create_
 0003:00079BA4       snd_trident_start_voice_
 0003:00079BCF       snd_trident_stop_voice_
 0003:00079CE0       snd_trident_write_voice_regs_
 0003:0007B2E8       snd_trident_pcm_
 0003:0007B43E       snd_trident_foldback_pcm_
 0003:0007B5E1       snd_trident_spdif_pcm_
 0003:0007C388       snd_trident_create_gameport_
 0003:0007C9BA       snd_trident_create_
 0003:0007CEEF       snd_trident_alloc_voice_
 0003:0007CF9F       snd_trident_free_voice_
 0003:0007D0DC       snd_trident_suspend_
 0003:0007D15E       snd_trident_resume_
 0003:0007D4C0       snd_trident_alloc_pages_
 0003:0007D4CF       snd_trident_free_pages_
 0003:0007EAAE       snd_sbmixer_write_
 0003:0007EAD9       snd_sbmixer_read_
 0003:0007F3B5       snd_sbmixer_add_ctl_
 0003:0007F4DA       snd_sbmixer_new_
 0003:0007F699       snd_sbmixer_suspend_
 0003:0007F710       snd_sbmixer_resume_
 0003:0007F787       snd_sbdsp_command_
 0003:0007F7DA       snd_sbdsp_get_byte_
 0003:0007F822       snd_sbdsp_reset_
 0003:0007FA1A       snd_sbdsp_create_
 0003:000806D7       _snd_pcm_hw_param_set_
 0003:00081502       snd_pcm_oss_write3_
 0003:00081561       snd_pcm_oss_read3_
 0003:000815F3       snd_pcm_oss_writev3_
 0003:00081652       snd_pcm_oss_readv3_
 0003:00083380       ACPIFindPCIDevice
 0003:00083422       InitACPICall
 0003:000834C0       StrLen
 0003:000834E0       StrNCmp
 0003:00083510       FindAddress
 0003:0008377C       init_MUTEX_
 0003:0008377D       init_MUTEX_LOCKED_
 0003:0008377E       down_
 0003:0008377F       up_
 0003:00083780       down_interruptible_
 0003:00083A6B       _snd_ctl_add_slave_
 0003:00083C24       snd_ctl_make_virtual_master_
 0003:00083CE6       release_and_free_resource_
 0003:00083CFB       snd_pci_quirk_lookup_id_
 0003:00083D3A       snd_pci_quirk_lookup_
 0003:00083D57       copy_to_user_fromio_
 0003:00083DC5       copy_from_user_toio_
 0003:0008403B       snd_ac97_set_rate_
 0003:000843F9       snd_ac97_pcm_assign_
 0003:00084774       snd_ac97_pcm_open_
 0003:00084A00       snd_ac97_pcm_close_
 0003:00084AC8       snd_ac97_pcm_double_rate_rules_
 0003:0008800B       snd_ac97_write_
 0003:00088068       snd_ac97_read_
 0003:000880E2       snd_ac97_write_cache_
 0003:00088138       snd_ac97_update_
 0003:000881B8       snd_ac97_update_bits_
 0003:00088202       snd_ac97_update_bits_nolock_
 0003:0008A1BF       snd_ac97_get_name_
 0003:0008A352       snd_ac97_get_short_name_
 0003:0008A435       snd_ac97_bus_
 0003:0008A4B8       snd_ac97_mixer_
 0003:0008AF36       snd_ac97_suspend_
 0003:0008B039       snd_ac97_resume_
 0003:0008B7A4       snd_ac97_tune_hardware_
 0003:0008C793       snd_ac97_proc_init_
 0003:0008C877       snd_ac97_proc_done_
 0003:0008C89A       snd_ac97_bus_proc_init_
 0003:0008C8F5       snd_ac97_bus_proc_done_
 0003:0008C909       snd_midi_process_event_
 0003:0008CEF1       snd_midi_channel_set_clear_
 0003:0008D399       snd_midi_channel_alloc_set_
 0003:0008D3F0       snd_midi_channel_free_set_
 0003:0008D417       snd_util_memhdr_new_
 0003:0008D44A       snd_util_memhdr_free_
 0003:0008D47E       __snd_util_mem_alloc_
 0003:0008D4D2       __snd_util_memblk_new_
 0003:0008D528       snd_util_mem_alloc_
 0003:0008D54B       __snd_util_mem_free_
 0003:0008D56C       snd_util_mem_free_
 0003:0008D58D       snd_util_mem_avail_
 0003:0008D5C0       __U8RS
 0003:0008D5DA       __I8RS
 0003:0008D5F5       __I8LS
 0003:0008D5F5       __U8LS
 0003:0008D610       __I8M
 0003:0008D610       __U8M
 0003:0008D630       strstr_
 0003:0008D6E0       strlcpy_
 0003:0008D770       vsscanf_
 0003:0008D7A0       sscanf_
 0003:0008D810       vsnprintf_
 0003:0008D870       snprintf_
 0003:0008D8A0       memset_
 0003:0008D8C0       memmove_
 0003:0008DB40       strtoul_
 0003:0008DB50       strtol_
 0003:0008DB60       __IsTable
 0003:0008DC70       __STOSB
 0003:0008DCA7       __STOSD
 0003:0008E880       __scnf_
 0003:0008EAF0       __prtf_
 0003:0008F7D4       __set_errno_
 0003:0008F7E2       __set_EDOM_
 0003:0008F7F0       __set_ERANGE_
 0003:0008F7FE       __set_EINVAL_
 0003:0008F811       __set_doserrno_
 0003:0008F820       tolower_
 0003:0008F830       __FDFS
 0003:0008F880       strupr_
 0003:0008F8A0       __Bits
 0003:0008F8FC       __threadstack_
 0003:0008F903       __threadid_
 0003:0008F90C       __OS2MainInit_
 0003:0008F97B       __OS2Init_
 0003:0008F9B9       __OS2Fini_
 0003:0008F9C1       __shutdown_stack_checking_
 0003:0008F9D6       __exit_
 0003:0008FA20       wctomb_
 0003:0008FA50       mbtowc_
 0003:0008FB10       _ismbblead_
 0003:0008FB30       ultoa_
 0003:0008FB80       ltoa_
 0003:0008FBB0       ulltoa_
 0003:0008FC20       lltoa_
 0003:0008FC50       utoa_
 0003:0008FCA0       itoa_
 0003:0008FCD0       __exit_with_msg_
 0003:0008FD20       __fatal_runtime_error_
 0003:0008FD50       __InitRtns
 0003:0008FDA0       __FiniRtns
 0003:0008FE00       __CommonInit_
 0003:0008FE45       __mbinit_
 0003:0008FF40       __EnterWVIDEO_
 0003:0008FF68       __OffFinalCS32
 0004:00000003       ___begtext
 0005:00000000       __OffBeginDS32
 0005:00000030       W?deviceOwner$nul
 0005:00000034       W?numOS2Opens$nul
 0005:00000038       _InitCompleteWas
 0005:0000003C       _rdOffset
 0005:00000040       _wrOffset
 0005:00000044       _szprintBuf
 0005:00000048       _fVerbose
 0005:0000004C       _fDebug
 0005:00000050       _idc16_PddHandler
 0005:00000058       W?RM_Help$npn()i
 0005:0000005C       W?RM_Help0$npn()i
 0005:00000060       W?RM_Help3$npn()i
 0005:00000064       W?RMFlags$nul
 0005:000000B0       _sISRHigh
 0005:000000E8       _SaveIRQCounter
 0005:000000EC       W?fnCardExitCall$n[]pn()v
 0005:0000010C       _nrCardsDetected
 0005:00000110       _fStrategyInit
 0005:00000114       _DebugLevel
 0005:0000011C       _ulget_free_pagesMemUsed
 0005:00000560       W?pmbUsed$npn$_MEMBLOCK$$
 0005:00000564       W?pmbFree$npn$_MEMBLOCK$$
 0005:00000568       W?uMemFree$nui
 0005:0000056C       W?acHeap$npnuc
 0005:00000570       W?ulnAlloc$nul
 0005:00000574       W?ulcAlloc$nul
 0005:00000578       W?ulnAllocCalls$nul
 0005:0000057C       W?ulnFree$nul
 0005:00000580       W?ulcFree$nul
 0005:00000584       W?ulnFreeCalls$nul
 0005:00000588       W?ulnCompact$nul
 0005:000005B4       _snd_pcm_devices_os2
 0005:00000ABC       _snd_ecards_limit
 0005:00000AC0       _snd_major
 0005:00000ACC       _snd_oss_root
 0005:00000AD0       _snd_seq_root
 0005:00000DC0       _snd_cards
 0005:00001538       ___Is_DLL
 0005:0000153C       ___saved_CS
 0005:00001640       ___MBCSIsTable
 0005:00001744       ___IsDBCS
 0005:00001748       ___hmodule
 0005:0000176C       BootCode
 0005:0000177C       stackbase
 0005:00001780       stacksel
 0005:00001784       __OffsetFinalCS16
 0005:00001786       __OffsetFinalDS16
 0005:00001788       _MSG_TABLE32
 0005:0000178C       PDDName
 0005:00001790       RMAllocResource1632
 0005:00001798       RMDeallocResource1632
 0005:000017A0       RMCreateDevice1632
 0005:000017A8       RMCreateAdapter1632
 0005:000017B0       RMCreateDriver1632
 0005:000017B8       RMDestroyDriver1632
 0005:000017C0       RMGetNodeInfo1632
 0005:000017C8       RMDevIDToHandleList1632
 0005:000017D0       RMHandleToResourceHandleList1632
 0005:000017D8       _TimerHandler16
 0005:000017DE       _ISR00
 0005:000017E2       _ISR01
 0005:000017E6       _ISR02
 0005:000017EA       _ISR03
 0005:000017EE       _ISR04
 0005:000017F2       _ISR05
 0005:000017F6       _ISR06
 0005:000017FA       _ISR07
 0005:00001800       DevHelp32
 0005:00001804       intSwitchStack
 0005:00001808       _TKSSBase
 0005:00001810       W?StratDispatch$n[]pn(pf$RP$$)ul
 0005:000018A4       W?ForceCard$ni
 0005:000018D4       _jiffies
 0005:000018D8       _current_task
 0005:000018FC       _current
 0005:00001900       _system_utsname
 0005:00001A86       _ioport_resource
 0005:00001AA2       _iomem_resource
 0005:00001ABE       _mem_map
 0005:00001AC2       _this_module
 0005:00001BC2       _szLastALSAError1
 0005:00001C42       _szOverrunTest1
 0005:00001C43       _szLastALSAError2
 0005:00001CC3       _szOverrunTest2
 0005:00001CC4       _iLastError
 0005:00001CC8       _proc_root
 0005:00001D14       _cardcalls
 0005:00001E1C       _midi_port
 0005:00001F88       _szRecSources
 0005:00002014       _oss_devices
 0005:00002154       _alsa_fops
 0005:00002158       _per_bytes
 0005:0000215C       _prev_size
 0005:00002160       _pcm_device
 0005:00002164       _total
 0005:00002168       _opened_handles
 0005:000081E4       _CountWv
 0005:000081E8       _LockAdd
 0005:000081EC       _hextab
 0005:000081FD       _MAGIC_COMM_PORT
 0005:00008200       _pcmcaps
 0005:00008220       _substream_int
 0005:0000A220       _control_id_changed
 0005:0000A224       _card_id_changed
 0005:0000A228       _unlock_all
 0005:0000A22C       _fInInterrupt
 0005:0000AA8C       _pci_devices
 0005:0000D4CC       _fSuspended
 0005:0000E8D0       W?ulcTotalHeap$nul
 0005:0000E934       ___initcall_alsa_hwdep_init
 0005:0000E938       ___exitcall_alsa_hwdep_exit
 0005:0000E9E0       ___initcall_alsa_timer_init
 0005:0000E9E4       ___exitcall_alsa_timer_exit
 0005:0000EA70       ___initcall_alsa_rawmidi_init
 0005:0000EA74       ___exitcall_alsa_rawmidi_exit
 0005:0000EE00       ___initcall_alsa_pcm_init
 0005:0000EE04       ___exitcall_alsa_pcm_exit
 0005:0000EE5C       ___initcall_alsa_sound_init
 0005:0000EE60       ___exitcall_alsa_sound_exit
 0005:0000EEE4       _snd_pcm_link_rwlock
 0005:0000EFA8       _snd_pcm_f_ops
 0005:0000F0B4       ___initcall_snd_mem_init
 0005:0000F0B8       ___exitcall_snd_mem_exit
 0005:0000F370       ___initcall_alsa_card_bt87x_init
 0005:0000F374       ___exitcall_alsa_card_bt87x_exit
 0005:0000F4D4       ___initcall_alsa_card_als4000_init
 0005:0000F4D8       ___exitcall_alsa_card_als4000_exit
 0005:00010255       ___initcall_alsa_card_cmipci_init
 0005:00010259       ___exitcall_alsa_card_cmipci_exit
 0005:00010578       ___initcall_alsa_card_atiixp_init
 0005:0001057C       ___exitcall_alsa_card_atiixp_exit
 0005:000109E4       ___initcall_alsa_card_fm801_init
 0005:000109E8       ___exitcall_alsa_card_fm801_exit
 0005:00010FB8       ___initcall_alsa_card_via82xx_init
 0005:00010FBC       ___exitcall_alsa_card_via82xx_exit
 0005:000114E0       ___initcall_alsa_card_m3_init
 0005:000114E4       ___exitcall_alsa_card_m3_exit
 0005:000121F0       ___initcall_alsa_card_intel8x0_init
 0005:000121F4       ___exitcall_alsa_card_intel8x0_exit
 0005:00012434       ___initcall_alsa_card_es1968_init
 0005:00012438       ___exitcall_alsa_card_es1968_exit
 0005:00012C95       ___initcall_alsa_card_es1938_init
 0005:00012C99       ___exitcall_alsa_card_es1938_exit
 0005:00012F30       ___initcall_alsa_card_cs4281_init
 0005:00012F34       ___exitcall_alsa_card_cs4281_exit
 0005:0001333C       ___initcall_alsa_card_ens137x_init
 0005:00013340       ___exitcall_alsa_card_ens137x_exit
 0005:000137F0       ___initcall_alsa_card_ca0106_init
 0005:000137F4       ___exitcall_alsa_card_ca0106_exit
 0005:00016870       ___initcall_patch_via_init
 0005:00016874       ___exitcall_patch_via_exit
 0005:00018FDC       ___initcall_patch_conexant_init
 0005:00018FE0       ___exitcall_patch_conexant_exit
 0005:0001913C       ___initcall_patch_atihdmi_init
 0005:00019140       ___exitcall_patch_atihdmi_exit
 0005:0001B93C       ___initcall_patch_sigmatel_init
 0005:0001B940       ___exitcall_patch_sigmatel_exit
 0005:000230C4       ___initcall_patch_analog_init
 0005:000230C8       ___exitcall_patch_analog_exit
 0005:00023858       ___initcall_patch_cmedia_init
 0005:0002385C       ___exitcall_patch_cmedia_exit
 0005:0004253B       ___initcall_patch_realtek_init
 0005:0004253F       ___exitcall_patch_realtek_exit
 0005:00042814       ___initcall_alsa_card_azx_init
 0005:00042818       ___exitcall_alsa_card_azx_exit
 0005:0004296B       _snd_hda_bind_vol
 0005:0004297B       _snd_hda_bind_sw
 0005:00042BD7       _snd_hda_pcm_type_name
 0005:00042C37       _auto_pin_cfg_labels
 0005:00042E04       _seq_client_load
 0005:00042E40       _seq_default_timer_class
 0005:00042E44       _seq_default_timer_sclass
 0005:00042E48       _seq_default_timer_card
 0005:00042E4C       _seq_default_timer_device
 0005:00042E50       _seq_default_timer_subdevice
 0005:00042E54       _seq_default_timer_resolution
 0005:00042E58       ___initcall_alsa_seq_init
 0005:00042E5C       ___exitcall_alsa_seq_exit
 0005:00042E80       ___initcall_alsa_seq_device_init
 0005:00042E84       ___exitcall_alsa_seq_device_exit
 0005:00042FD4       _use_internal_drums
 0005:00042FD8       _opl3_ops
 0005:00042FFC       ___initcall_alsa_opl3_seq_init
 0005:00043000       ___exitcall_alsa_opl3_seq_exit
 0005:00043070       ___initcall_alsa_opl3_init
 0005:00043074       ___exitcall_alsa_opl3_exit
 0005:00043208       _snd_opl3_regmap
 0005:0004324C       ___initcall_alsa_mpu401_uart_init
 0005:00043250       ___exitcall_alsa_mpu401_uart_exit
 0005:000432F8       ___initcall_alsa_card_cs46xx_init
 0005:000432FC       ___exitcall_alsa_card_cs46xx_exit
 0005:00050F80       ___initcall_alsa_card_cs5535audio_init
 0005:00050F84       ___exitcall_alsa_card_cs5535audio_exit
 0005:0005117C       ___initcall_alsa_card_emu10k1_init
 0005:00051180       ___exitcall_alsa_card_emu10k1_exit
 0005:00053E54       ___initcall_alsa_card_ymfpci_init
 0005:00053E58       ___exitcall_alsa_card_ymfpci_exit
 0005:000547DC       ___initcall_alsa_card_ali_init
 0005:000547E0       ___exitcall_alsa_card_ali_exit
 0005:000548A8       ___initcall_alsa_card_trident_init
 0005:000548AC       ___exitcall_alsa_card_trident_exit
 0005:0006152C       ___initcall_alsa_card_nm256_init
 0005:00061530       ___exitcall_alsa_card_nm256_exit
 0005:000619F8       ___initcall_alsa_sb_common_init
 0005:000619FC       ___exitcall_alsa_sb_common_exit
 0005:00061A78       ___initcall_alsa_pcm_oss_init
 0005:00061A7C       ___exitcall_alsa_pcm_oss_exit
 0005:00061B0C       ___EFG_printf
 0005:00061B10       ___EFG_scanf
 0005:00061B14       ___FirstThreadData
 0005:00061B18       ___GetThreadPtr
 0005:00061B1C       __AccessFileH
 0005:00061B20       __ReleaseFileH
 0005:00061B24       __AccessIOB
 0005:00061B28       __ReleaseIOB
 0005:00061B2C       __AccessNHeap
 0005:00061B30       __AccessFHeap
 0005:00061B34       __ReleaseNHeap
 0005:00061B38       __ReleaseFHeap
 0005:00061B3C       __AccessTDList
 0005:00061B40       __ReleaseTDList
 0005:00061B44       ___sig_init_rtn
 0005:00061B48       ___sig_fini_rtn
 0005:00061B4C       __threadstksize
 0005:00061B50       ___process_fini
 0005:00061B54       __dynend
 0005:00061B58       __curbrk
 0005:00061B5C       __LpCmdLine
 0005:00061B60       __LpPgmName
 0005:00061B64       __LpDllName
 0005:00061B68       __LpwCmdLine
 0005:00061B6C       __LpwPgmName
 0005:00061B70       __LpwDllName
 0005:00061B74       __STACKLOW
 0005:00061B78       __STACKTOP
 0005:00061B7C       __ASTACKSIZ
 0005:00061B80       __ASTACKPTR
 0005:00061B84       __cbyte
 0005:00061B88       __cbyte2
 0005:00061B8C       __child
 0005:00061B90       __no87
 0005:00061B92       __Envptr
 0005:00061B96       __Envseg
 0005:00061B98       __osmajor
 0005:00061B99       __osminor
 0005:00061B9A       ___FPE_handler
 0005:00061BA0       ___MBCodePage
 0005:00061BA4       ___WD_Present
 0005:00061BA8       __amblksiz
 0005:000623FA       ___initcall_alsa_ac97_init
 0005:000623FE       ___exitcall_alsa_ac97_exit
 0005:00062524       ___initcall_alsa_seq_midi_emul_init
 0005:00062528       ___exitcall_alsa_seq_midi_emul_exit
 0005:0006252C       ___initcall_alsa_util_mem_init
 0005:00062530       ___exitcall_alsa_util_mem_exit
 0005:00072188       ___Alphabet
 0005:00074E40       _snd_pcm_known_rates
 0005:0007B3DC       __OffFinalDS32
 0005:0007B3E0       __Start_XI
 0005:0007B3E6       __Start_YI
 0005:0007B3E6       __End_XI
 0005:0007B3E6       __End_YI
 0005:0007B430       __nullarea
 0005:0008B440       _end
 0005:0008B440       _edata
